:020000040800F2
:104000000050002029EA0008C5C10008C9C1000805
:10401000CDC10008D1C10008D5C1000800000000D2
:10402000000000000000000000000000DDC10008EA
:10403000D9C1000800000000E1C100080D9100088E
:10404000E5C10008E9C10008EDC10008F1C10008A0
:10405000F5C10008F9C10008FDC1000801C200084F
:1040600005C2000809C200080DC2000800000000D7
:104070000000000000000000000000000000000040
:1040800000000000000000002DC2000831C200083E
:1040900041C2000851C2000861C2000871C2000894
:1040A00075C2000879C200087DC2000881C20008FC
:1040B00085C2000889C200088DC2000891C20008AC
:1040C00095C2000899C200089DC20008A1C200085C
:1040D000A5C20008818D0008BD8C0008B1C200088F
:1040E000B5C20008B9C20008BDC200080000000047
:1040F00000000000000000000000000000000000C0
:0C41000000000000000000005FF800005C
:1041100030BF704720BF704740BF7047BFF36F8FFD
:104120007047BFF34F8F7047BFF35F8F704701DF5A
:104130007047EFF31480704780F31488BFF36F8FDC
:104140007047EFF30980704780F309887047EFF3F9
:104150000880704780F30888704772B6704762B66F
:10416000704771B6704761B6704780F31188704729
:10417000EFF31280704740BA704700BA70470000F2
:1041800037B509F023F9554B00254FF480301D70E9
:1041900009F03CF909F0A0FA0128044626D11020C4
:1041A00008F0FEFB284609F081F9284609F092F94B
:1041B000284609F085F94FF480304FF4802109F04A
:1041C00051F9204609F05AF9392009F06FFA002810
:1041D000FAD0012008F0CCFB012009F055F909F0D4
:1041E0005DF90428FBD13D4B01221A700420012106
:1041F00009F012FA03238DF80630153301A9384867
:104200008DF807304FF48073ADF8043008F0FCFDF2
:10421000062009F045FA0120014609F0FDF94FF0AA
:10422000C050012109F006FA4FF480414FF00060C0
:1042300008F0EEFF4FF4407008F04CFF00F04CFB2C
:1042400000F08AFC2749284A284B1160284A294D4A
:10425000136001222A70284A284C136000F0C8F825
:1042600005F038F804F09AFF04F002FC00F04AF878
:10427000207804F097FEE07804F088FC207804F0C1
:10428000D7FDE07804F0AAFC2B780BB105F064FBB5
:1042900006F0FCF800F0BAF907F066FD01F014FF33
:1042A00005F074FB06F038F9154B4FF480625A6143
:1042B00004F06EFF03F056FD06F03CF905F0BAFB82
:1042C00000F006F900F0F8F80028F3D006F0DEF868
:1042D00001F0FAFE06F020F9ECE700BF540C0020D4
:1042E00000080140F9970008640C002009910008BB
:1042F000F40B0020740B0020940B00200800002019
:10430000000C0140144B82B01B7813B3134B4FF4D5
:1043100000725A614FF480721A61002301E0019B20
:1043200001330193019A4AF69B539A42F7D90B4BFA
:104330004FF400721A614FF480725A61002301E059
:10434000019B01330193019A4AF69B539A42DDD8AF
:10435000F6E702B0704700BFA00B0020000C014040
:1043600010B1012805D101E0082200E00422014B30
:104370005A617047000C014010B1012805D101E0DD
:10438000082200E00422014B1A617047000C014032
:1043900038B50546002455FA04F2E3B212F0010FD5
:1043A000184602D0FFF7E8FF01E0FFF7D9FF01341C
:1043B000082CF0D138BD00BF18B1012806D000206C
:1043C00008E0054BD868C0F3C00003E0024BD86892
:1043D000C0F38000704700BF000C014008B100200E
:1043E00003E0024B9868C0F3C030704700080140FA
:1043F00062B6704772B6704718B9024B4FF48062CC
:104400005A617047000C014018B9024B4FF48062AA
:104410001A617047000C014020B1054B4FF4005267
:104420001A6103E0024B4FF400525A61704700BF1B
:1044300000100140074B9A88C2F30722042A06D1D4
:104440009A88D2B2892A02D1188980B200E000206D
:10445000704700BF006C004020B1054B4FF4804214
:104460001A6103E0024B4FF480425A61704700BF6B
:104470000010014010B9024B09011960704700BFDC
:104480000400002008B9014B197070473002002069
:1044900008B1002001E0014B58787047300200203D
:1044A000044B98780138C0B201288CBF002001204D
:1044B000704700BF30020020044B9878012801D0DB
:1044C000002001E002229A70704700BF30020020F5
:1044D000082008B504F078FE592804D9064B9A78CC
:1044E0004AB9013206E0082004F06EFE542802D8D2
:1044F000014B00229A7008BD3002002008B5032845
:1045000003D8DFE800F0040D1217002016E00020A9
:1045100004F05AFEB0F5006F94BF002001200DE0BA
:10452000074B9868C0F3801008E0054B9868C0F30B
:10453000C01003E0024B9868C0F3401008BD00BFF4
:10454000000C014038B500242546E0B2FFF7D6FF45
:1045500020B10123A34043EA0505EDB20134082C44
:10456000F3D1284638BD00BFF8B51E4D01212846BD
:1045700009F01EFF1C4C08B9606831E0FF210022E1
:10458000032000F06DFAFF2101220646032000F00F
:1045900067FA4CF2215307460121AB84284647EACB
:1045A000062609F00BFF002316F0020F637001D0FE
:1045B00001336370B60816F4805F04D00A4B5A7852
:1045C00042F002025A7016F4005F04D0064B5A788B
:1045D00042F004025A70044B986820EA06005860C2
:1045E000F8BD00BF000800403002002008B5FFF70A
:1045F000BBFF052801D8012007E0FFF7B5FF40F217
:10460000F933984294BF0020012008BD38B5234CEF
:10461000002021694909FFF72DFF2169002001F0E1
:104620001F01FFF72FFFFE210022032000F018FAE0
:1046300040210122032000F013FA00210A46032042
:1046400000F00EFA002104460122032000F008FACF
:10465000082C134B05D14FF40062DA6040F6FF726C
:1046600004E04FF40072DA6040F2FF329A60E72112
:104670000022032000F0F4F900210122032000F0C1
:10468000EFF9FFF771FF064B040224464FEAE47589
:10469000C3E90845C3E90645186138BDF80B002099
:1046A000300200202DE9F84304F072FD624CA06254
:1046B000FFF75AFF2369E06298423EDDE268C11AC3
:1046C00091420BDA5D4B256B1A684D195143D4E9C1
:1046D0000867721847EBE17325632BE094F800C07C
:1046E000564A1CF0040F12D0A3681668C31A5E4322
:1046F0002CF0040C36464FEAE677236300220023B1
:10470000C4E9086784F800C0C4E906234EE0A56840
:1047100016685A190132121A7243D4E90867236BDA
:10472000ED43ED18B6EB020867EBE27942464B46E3
:1047300069182163C4E9082338E037DAE1681A1AF6
:104740008A420EDA3D4D216B2D68C91A6A43D4E9BD
:104750000867B6EB020867EBE27942464B46091858
:10476000E7E72178354A11F0040F0FD0126821F0E5
:104770000401424312464FEAE273C4E908230022CF
:1047800000232170C4E9062320630FE0A1681268AA
:104790000131CB1A1B185A43D4E90867B61847EB06
:1047A000E277226BC4E908679B182363224B1D6BD9
:1047B0005A6B996BAA1A82EAE27CACEBE27C8C45DC
:1047C0002CD942F210714A439E6ADC6B3C21341BA7
:1047D00092FBF4F251434FF4807C91FBFCF181EAAF
:1047E000E172A2EBE172596440F6B8318A42DE63AD
:1047F0005D631C6401DDC82219E0B2F57A7F01DD3A
:10480000642214E0322A01DD0A2210E00A2A01DDC6
:1048100005220CE0012A0BDD012208E0996ADA6B1F
:104820008A1AB2F5FA6F03D900225A6401329A63E8
:10483000014B1861BDE8F88330020020040000201D
:1048400038B50D4618BB124CFFF72CFFD4E9080110
:10485000002901DBA26803E0A268404261EB41014C
:10486000120212464FEAE2730CF0FEFEC4E9062380
:1048700028464FEAE071064C0B02020243EA10633D
:10488000D4E90601801841EB0301C4E9080138BDF1
:104890003002002008B508B100200CE0FFF702FF4D
:1048A000054BD3E90601D3E90823121A63EB010390
:1048B000100A40EA036008BD3002002008B510B1BC
:1048C00008F0B0FC01E008F0B5FC08BD08B510B96F
:1048D000C90805F04DFA08BD2DE9F0455A4885B0E4
:1048E000DFF87481012108F01FFB03AE04200121D1
:1048F00008F092FE03251024404642F2122331466E
:10490000ADF80C308DF80E508DF80F4008F07CFAA1
:1049100002234E4F40464FF0040AC8F8104031467B
:10492000C8F814304CF20043ADF80C308DF80E503E
:104930008DF80FA008F068FA0820012108F06CFE3D
:1049400041F61C7338463146ADF80C308DF80E50E8
:104950008DF80F4008F058FA4FF4F8533B610C23E0
:10496000384631467B614FF0E00308F50068ADF84A
:104970000C308DF80E508DF80FA008F045FA204647
:10498000012108F049FE4EF2000331464046ADF8E1
:104990000C308DF80E508DF80F4008F035FA4FF4BA
:1049A0002043C8F81030A3F5C0430121C8F81430E3
:1049B000504608F03FFE264809F00EFE684609F012
:1049C00001FA4FF00003ADF800304FF0FF336946B5
:1049D0001F48ADF804304FF00003ADF80630ADF8D5
:1049E000023009F097F81A48012109F013FA012161
:1049F000184808F099FA00231A461946164C4FF445
:104A0000005565612046A468013314F4804F4FF4CB
:104A100000540461806808BF013110F4804F18BF52
:104A200001320A2BEAD10A2903D10A2A01D1012233
:104A300000E00022094B04481A70012108F074FAC2
:104A400005B0BDE8F08500BF00023000000C014059
:104A5000000800400004300000080140A00B0020C6
:104A600070B504460D461646032868D8DFE800F006
:104A700002070A0E334B4FF480525A6112E01022A3
:104A8000314B0DE04FF400622E4B09E02F4A1388A2
:104A900023F002031B041B0C13802D4B4FF4004228
:104AA0005A6110E02B48022108F018FF0028F9D0C5
:104AB0002946284808F0B6FE2648012108F00EFFD6
:104AC0000028F9D00FE02148022108F007FF002854
:104AD000F9D029461D4808F0A5FE1C48012108F020
:104AE000FDFE0028F9D0EEB1032C28D8DFE804F051
:104AF00002070A0F134B4FF480521A6118E010227C
:104B0000114B02E00F4B4FF400621A6112E0104AA1
:104B10000E4B4FF4004111611A8892B242F002022A
:104B20001A8007E0032C0AD8DFE804F0020404042A
:104B3000084800E0054808F077FEC0B200E0002019
:104B400070BD00BF000C0140000801400030014072
:104B500000100140003800402DE9F04F01218BB0DA
:104B60004FF4804008F066FD494C012009AF014632
:104B700008F052FD03264FF0180B204639464AF242
:104B80000003DFF81491ADF824304FF0040A8DF8DB
:104B900026608DF827B008F037F9204639464FF4E3
:104BA00080430DF11008ADF824308DF826608DF8A3
:104BB00027A008F029F94FF48273002402224FF451
:104BC000007C012548464146ADF812304FF00803FD
:104BD000ADF81620ADF81AC00392CDF808C0ADF8B4
:104BE0001C30ADF81040ADF81440ADF81850ADF8D9
:104BF0001E40ADF8204008F0A1FD4846294608F0C7
:104C0000D9FD29464FF4805008F006FD09F55049BA
:104C10002846214608F088F9484639464FF0A00357
:104C2000ADF824308DF827B08DF8266008F0ECF848
:104C3000484639464FF04003ADF824308DF82660E1
:104C40008DF827A008F0E0F8039ADDF808C04FF4CB
:104C500082734146ADF812300E484FF01003ADF8A4
:104C60001620ADF81AC0ADF82040ADF81040ADF8F0
:104C70001440ADF81850ADF81C30ADF81E4008F0E7
:104C80005DFD0448294608F095FD0BB0BDE8F08FA6
:104C9000000C01400030014000380040014B187802
:104CA000704700BF780200202DE9F84505461446FC
:104CB0000E4600294BD0002849D0814247D04FEA08
:104CC00042185FFA88F848F006073946002006F0D7
:104CD00047FD48F00C018246002006F041FD804669
:104CE00028460CF083FA054630460CF07FFA014660
:104CF00028460CF087FB064650460CF077FA314602
:104D00000CF080FB0CF090FC054640460CF06EFA6F
:104D100031460CF077FB0CF087FC0E49002814BFDD
:104D200080464FF001083046002D08BF01250CF0E9
:104D300053FC18B14146204606F08CFF39462A46FE
:104D4000002006F0BFFD044BE41801232371BDE8E9
:104D5000F88500BF0000A0417802002070B50D4D1D
:104D6000044645192B799BB1C6B20B4B710141F03A
:104D7000060153F8202001F0E601002006F036FE7F
:104D8000064B304653F8241006F064FF00232B71C5
:104D900070BD00BF78020020700B00206C0700205F
:104DA00037B5A24B5B789A1FD2B2012A02D98C2B5D
:104DB00000D0C02B9D4A92780AB1042279E3A42B3B
:104DC00000F0AC825CD8842B00F0D48028D8062B6D
:104DD00000F0348110D8022B00F0CC8006D8002BD4
:104DE00000F0AE80012B40F06383B4E0042B00F0B0
:104DF000F18000F20681E0E0802B00F0A18009D86C
:104E00000C2B00F03D810D2B00F05181072B40F061
:104E10004F8323E1822B00F0618100F2DB809AE076
:104E2000942B00F02D8116D88A2B00F0738108D8BE
:104E3000862B00F0E680C0F0C080872B40F03883DE
:104E40005BE18D2B00F08D81932B00F030818C2B5A
:104E500040F02E8378E1A02B00F0428209D8992BF4
:104E600000F0AE819A2B00F0C581952B40F0208395
:104E700084E1A22B00F047826C4C00F24A823DE2B2
:104E8000B52B00F0C38229D8AB2B00F08A8211D851
:104E9000A72B00F0708206D8A52B00F04E82A62B1F
:104EA00040F0068358E2A92B00F070825F4C00F2BC
:104EB000738266E2AF2B00F0918206D8AD2B00F032
:104EC00081825A4C00F2848271E2B12B00F092820E
:104ED000C0F08A82B22B40F0EB8291E2C72B00F047
:104EE000AD8015D8C02B00F0B98008D8B72B00F0E2
:104EF000B182C0F09682B82B40F0DA82B2E2C22BC7
:104F000000F09E81C0F09481C32B40F0D182A1E1DA
:104F1000D22B00F0B68209D8CC2B00F0B881D12B6F
:104F200000F0A682C82B40F0C3829EE1D52B00F092
:104F3000C481D62B00F0C981D42B40F0B982B1E1F5
:104F40003A4B002099785A68DB78490143EA0222FB
:104F500001F0E0010BE0354B002099785A684901D7
:104F6000DB7841F0020143EA022201F0E20106F09F
:104F7000A9FCA0E22D4C0020A178E37849016268E9
:104F800041F0080143EA022201F0E80106F02EFD9B
:104F9000E378A1786268490143EA0222002A41F0DD
:104FA0000601B8BF524201F0E601002006F01EFDE6
:104FB0001F4AA378D318012252E21C4B0020997893
:104FC0005A684901DB7841F00A0143EA022201F004
:104FD000EA018FE0154C0020A178E378626849016E
:104FE00041F0060143EA022201F0E60106F0FEFC70
:104FF000E2786068A37842EA00200D4A0D499A18C9
:105000000FE00A4CE3786168A07843EA012106F0DA
:1050100021FEE2786068A37842EA0020044A06494B
:105020009A1841F823000023137144E2E806002097
:1050300078020020700B00206C070020AB4BAC4ABC
:105040009878D978AB4BAC4C1B5C02EB40124FF01C
:10505000010C04F800C0022B517215E1A34BA44AC5
:105060009878D978A34BA44C1B5C02EB40124FF00C
:10507000010C04F800C09172002B40F01C82E6E1A4
:105080009A4C0020A17801AA490141F0140101F0D5
:10509000F40106F0B7FB6168E2789DF8053052EA4A
:1050A000012114BF43F0020323F002037CE08F4C84
:1050B0000020A17801AA490141F0140101F0F40196
:1050C00006F0A0FB6168E2789DF8053052EA012104
:1050D00014BF43F0010323F0010365E0834B00207C
:1050E00099785A684901DB7841F0040143EA0222C9
:1050F00001F0E40106F07AFCDDE17C4B00209978B8
:105100005A684901DB7841F00E0143EA022201F0BE
:10511000EE01EFE7754C01ADA1782A46490141F057
:10512000140101F0F401002006F06CFBA178E37893
:10513000490141F0140101F0F4012A4600208DF8E4
:10514000063006F0FBFCB6E1684AD3789078684AEE
:10515000C3F1080102EB4012C9B2D37205F01AF98B
:10516000A9E1624B002099785A684901DB7841F047
:105170001A0143EA022201F0FA01BBE75B4C00206E
:10518000A17801AA490141F0140101F0F40106F0EF
:1051900039FB6168E2789DF8053052EA012114BFBD
:1051A00043F0040323F004038DF805304F4B002037
:1051B000997801AA490141F0140101F0F401C0E716
:1051C0004A4C01ADA1782A46490141F0180101F08D
:1051D000F801002006F016FBA1789DF80530E27872
:1051E000490102F00F0223F00F0341F0180142EAD7
:1051F000030316E03D4C01ADA1782A46490141F078
:10520000180101F0F801002006F0FCFAA1789DF8E1
:105210000530E278490103F00F0341F0180143EA39
:10522000021301F0F8012A4600208DF8053088E7C6
:105230002E4B9978DA782E4B03EB41131A723AE130
:105240002A4B59689A78DB78520143EA0121284BAE
:10525000D15030E1254B59689878DA78244B42EAEE
:10526000012203EB40135A6025E1204B204A987835
:10527000D978204B204C1B5C02EB40124FF0010C04
:1052800004F800C0032BD17740F01581DFE0174B05
:1052900059689878DA78164B42EA012203EB4013FA
:1052A000DA8108E1114B59689878DA78104B42EAB4
:1052B000012203EB40135A61FDE00C4B9978DA7838
:1052C0000B4B03EB41139A77F5E0084B596898783C
:1052D000DA78074B42EA012203EB40139A83EAE0B3
:1052E000024BD978987805F047F8E4E0E80600200A
:1052F000F80B0020600C00205C0C0020E178A07806
:1053000005F030F8D7E06C4BD978987804F00AFFB4
:10531000D1E0E178A07804F0F9FECCE0664CA0780A
:1053200004F0BEFBE178A37818B9184604F0D6FE65
:10533000C1E0184604F0A2FEBDE05F4CA07804F086
:10534000AFFB20B9E178A07804F0BCFEB3E0E178CF
:10535000A07804F07BFEAEE0574CA07804F0A0FBF0
:10536000E178A37818B9184604F0A0FEA3E0184627
:1053700004F078FE9FE0504BD978987804F08AFECC
:1053800099E0E178A07804F097FD94E04A4BD97851
:10539000987804F085FD8EE0E178A07804F074FD43
:1053A00089E0454BD978987804F062FD83E0E17894
:1053B000A07804F051FDA178404BE27803EBC103E3
:1053C0005A7178E03C4BD978987804F0E9FC72E0A7
:1053D00094F90310A07804F0D7FC6CE0364BD97830
:1053E000987804F063FF66E0334BD978987804F03E
:1053F00051FF60E0304BD978987804F03FFF5AE0D5
:105400002D4BD978987804F02DFF54E02A4B596839
:105410009878DA782A4B42EA012203EB40139A612A
:1054200049E0254B254A5C68D978987841EA0423FD
:1054300042F8303023B902EBC002517904F00CFD80
:105440001D4B204A9878125C012A34D1D978FFF795
:105450003DFA30E0184B9978DA78184B03EBC1032A
:105460001A7128E0144BD978987804F043FE22E0B2
:10547000114AD3785168907843EA0121FFF7E0F9A7
:1054800019E00D4C0E4BA078E178626803EB4013F5
:1054900041EA02221A6101F01F01FEF7F3FFE378EF
:1054A0006168A07843EA01214911FEF7E3FF02E0B9
:1054B0000322054B1A703EBDE8060020840B002035
:1054C000F80B0020600C00206007002037B5A74BC8
:1054D0005B789A1FD2B2012A02D98C2B00D0C02B44
:1054E000A24A92781AB1A24B04221A7043E3A52B68
:1054F00000F080829E4C7BD8842B00F00B8138D842
:10550000082B00F03D8115D8032B00F00C8105D845
:10551000012B00F0F38000F2FD80E8E0052B00F0A5
:105520001181C0F00B81062B00F01281072B40F097
:105530000F8314E10D2B00F03C810BD80A2B00F0F7
:105540005D81C0F044810B2B00F046810C2B40F0B4
:10555000FF821EE1812B00F0D18003D8802B40F028
:10556000F782C4E0822B00F05881832B40F0F08258
:10557000E4E0992B00F093811ED88C2B00F06D8114
:105580000BD8862B00F0DE80C0F0CD80872B00F09A
:105590004D818A2B40F0DC8251E1932B00F0098190
:1055A00003D88D2B40F0D4825EE1942B00F0F18083
:1055B000952B40F0CD8262E1A02B00F0F8810BD852
:1055C0009B2B00F00981C0F07A819C2B00F01681A2
:1055D0009D2B40F0BD82D3E0A22B00F0F281C0F001
:1055E000EB81A32B00F0F281A42B40F0B182F2E119
:1055F000C02B00F0B4803BD8AF2B00F059821BD8F1
:10560000AA2B00F039820BD8A72B00F02682C0F01D
:105610001582A82B00F02682A92B40F0998226E261
:10562000AC2B00F03382C0F02C82AD2B00F0358221
:10563000AE2B40F08D8235E2B42B00F052820BD8B5
:10564000B12B00F03F82C0F03882B22B00F03F82D5
:10565000B32B40F07D823FE2B62B00F04E82C0F0CB
:105660004582B72B00F05082B82B40F0718252E295
:10567000CF2B00F063811ED8C52B00F047810BD8DB
:10568000C22B00F03281C0F02981C32B00F033819E
:10569000C42B40F05D8235E1C82B00F03B8103D87C
:1056A000C72B40F0558253E0CC2B00F03A81CE2B33
:1056B00040F04E823CE1D52B00F064810BD8D12B19
:1056C00000F02E82C0F05281D22B00F02E82D42B1B
:1056D00040F03E824FE1D72B00F03082C0F059817C
:1056E000DB2B00F02E82FE2B40F0328258E11F4B64
:1056F00000209978490101F0E00107E01B4B0020F0
:105700009978490141F0020101F0E20106F028F820
:1057100060601FE2154B00209978490141F00801B3
:1057200001F0E801A8E0114B00209978490141F00F
:105730000A0101F0EA0106F04DF8E9E70B4B9A780F
:105740000C4B02E0094B9A780B4B53F82230D9E10D
:10575000064B9A78094B03EB42135B7AD2E1034B79
:105760009A78064B03EB42139B7ACBE1E8060020C4
:1057700060070020700B00206C070020F80B002051
:10578000002005F003FFA14B9B785B0050FA03F368
:1057900040E09E4B0020997801AA490141F0140194
:1057A00001F0F40106F02EF89DF80530C3F3400334
:1057B000A8E1964B0020997801AA490141F0140113
:1057C00001F0F40106F01EF89DF8053022E0904B40
:1057D0009A68C2F34012AEE17C21002001AA06F0D3
:1057E00011F88A4B02219A789DF80630520011FA7E
:1057F00002F21A420CBF0023012383E101AA002018
:105800007C2105F0FFFF814B9DF806209B785B0013
:1058100052FA03F303F0010374E17C4B0020997802
:10582000490141F0040101F0E40125E0774B00203B
:105830009978490141F00E0101F0EE011CE0734B33
:1058400001AA99780020490141F0140101F0F40106
:1058500005F0D8FF9DF806206DE16C4B987804F0B8
:10586000FFF8C0F1080053E7684B00209978490120
:1058700041F01A0101F0FA0105F0ACFF65E1634B5C
:1058800001AA99780020490141F0140101F0F401C6
:1058900005F0B8FF9DF80520C2F380024BE15B4B99
:1058A0000020997801AA490141F0180101F0F8019E
:1058B00005F0A8FF9DF8053003F00F0322E1534BDC
:1058C00001AA99780020490141F0180101F0F8017E
:1058D00005F098FF9DF8052012092CE14B4B9A78B2
:1058E0004C4B03EB42131A7A25E1484B9A78494B0B
:1058F0005201D35806E1454B9A78464B03EB4213CD
:105900005A6818E1414B9A78434B14E03F4B9A7820
:10591000424B1AE73D4B9A783E4B03EB4213DB7F39
:10592000F0E03A4B9A783B4B03EB4213DA8902E101
:10593000364B9A783A4B53F82220FCE0334B394AE5
:105940009B780021D25C61600AB101226260364A14
:105950003449D25C0020C85422B1344A516841F025
:1059600002015160304A0021D154F3E0274B304A04
:105970009B78D25CDFE0254B9A78264B03EB4213F1
:105980005A69D8E0214B9A78224B03EB42139B7F54
:10599000B8E01E4B9A781F4B03EB42139A8BCAE078
:1059A0001A4B9A781B4B03EB42131A7BC3E0174B3D
:1059B000987804F05DF8ABE6144B987804F060F842
:1059C000C3E0124B987804F063F8A1E60F4B987887
:1059D00004F066F8B9E00D4D144CA87804F060F8B6
:1059E000AB7818B9184604F06BF891E6184604F045
:1059F00087F88DE6054D0D4CA87804F051F8AB788A
:105A0000C0B9184604F064F882E600BFE80600203A
:105A1000000C0140F80B0020780B00201C0C00202B
:105A20009C0B0020EC0B0020900B00206007002056
:105A3000F00B0020184604F073F869E64E4D4F4C09
:105A4000A87804F02DF8AB7818B9184604F048F897
:105A50005EE6184604F05CF85AE6474B987804F086
:105A600047F855E6444B987804F062F86DE0424BF5
:105A7000987804F065F868E03F4B987804F068F88F
:105A800046E63D4B987804F06BF85EE03A4B9A7826
:105A90003B4B03EBC2035B7934E0374B987804F05F
:105AA0006FF852E0344B987804F072F840B24CE052
:105AB000314B987804F07EF82AE62F4B987804F062
:105AC00081F842E02C4B987804F084F820E62A4BC9
:105AD000987804F087F838E0274B987804F092F82B
:105AE00033E0254B274A9B78D35C0BE0224B9A7816
:105AF000254B03EB42139A691DE01F4B9A78204B0C
:105B000053F83230636025E01B4B9A781C4B03EB53
:105B1000C2031A790FE0184B987803F0C9FF14E01C
:105B2000154B9878FEF7B6FEF2E5134B9A78164BB4
:105B300003EB42131A69114B5A600BE0FEF714FD98
:105B4000E6E50D4B9878FEF7A3FC0C4B586001E09E
:105B5000032323700D4B1B786BB1084B0C495A681B
:105B60000C4B0A601AB91A6842F0080202E01A687F
:105B700022F008021A603EBDE806002060070020FF
:105B8000840B0020800B0020F80B00205A07002017
:105B900048070020F006002008B58B4A5378991F6B
:105BA000C9B201290AD98C2B08D0C02B06D0C72B2B
:105BB00004D003F13401C9B2322900D8824A927864
:105BC0000AB10422FDE09A2B20D8992B73D2822BA4
:105BD00065D00BD8062B44D003D8042B3DD0052B21
:105BE0000AE0072B4BD00C3B012B0CE08C2B58D040
:105BF00005D8832B31D0862B40F0E2802FE08D2B0F
:105C000057D0933B022B00F2DB8046E0C82B00F01C
:105C10008A800FD8C12B5FD005D8B52B51D0C02BAF
:105C200040F0CE802BE0C32B72D068D3C72B40F05E
:105C3000C78016E0D42B00F0928005D8CC2B7CD006
:105C4000D22B40F0BD8082E0D62B00F09C80C0F0CB
:105C50008E80FE2B40F0B480A1E006212CE00C21C8
:105C60002AE0594B59499A7853010833CB1803EB72
:105C70004210413001EB4212801A59783CE0524BFD
:105C800052499A7853010833CB1803EB4210423043
:105C900001EB4212801A99782EE014210CE00421C5
:105CA0000AE0494B49489B78012200EB43110B3134
:105CB0007CE01A2100E01821434B987805F0E0FDC4
:105CC00081E0414B414893F802C004224FEA4C1353
:105CD00003F11801411853E03B4A3C4B91788A008C
:105CE000013201F1020C03EBC20003EB411100EBA6
:105CF0004C10401A13F8321002F070FD63E0324B82
:105D000032499B780422981C01EB4311400154E076
:105D10002D4B042299782D4B881C03EB41139918C5
:105D200001EB401048E0284B284893F802C00122BC
:105D30004FEA4C1319181F3122E0234B23489B785C
:105D4000022200EB43110E3103EB020C30E01E4B3C
:105D50001E489B78042259011031411826E01A4B45
:105D60001A489B78042200EB431114311EE0164BB5
:105D7000164893F802C001224FEA4C1319181E313D
:105D80000CF1020C09E0104B104893F802C00222FB
:105D90004FEA4C1319181C319444C3180AE00A4BFB
:105DA0000A489B78012200EB43110C3103F1020CED
:105DB00000EB431301EB4C10C01A02F091FC02E01F
:105DC0000322034B1A7008BDE8060020F80B0020E0
:105DD0006007002038B59E4A5378991FC9B201293F
:105DE0000AD98C2B08D0C02B06D0C72B04D003F1C6
:105DF0003401C9B2322900D8954A92780AB10422F6
:105E000058E19A2B25D8992B80F0C280822B00F084
:105E10009E800CD8062B78D003D8042B42D0052BBB
:105E20000CE0072B00F081800C3B012B0EE08C2B4B
:105E300000F0938005D8832B34D0862B40F0398135
:105E400047E08D2B00F0A280933B022B00F23181C2
:105E50007BE0C72B59D011D8C12B00F0A68006D803
:105E6000B52B00F09780C02B40F023815DE0C22B62
:105E700000F0AD80C32B40F01C81B1E0D42B00F0CA
:105E8000CE8006D8C82B00F0B680CC2B40F0118114
:105E9000BBE0D62B00F0E680C0F0CD80FE2B40F0BA
:105EA0000881F0E06A4C0621A07805F0B1FEA578E3
:105EB0000020690141F0060101F0E60105F08AFCCD
:105EC000644AA378D318644A42F8250000221A7164
:105ED000F2E05F4C0C21A07805F09AFEA578002036
:105EE000690141F00C0101F0EC0105F073FCA378AD
:105EF0005A4A584942F8250018465B1852F82010B3
:105F000000221A7105F0A6FED6E0514B544A9B7848
:105F10005C010834141904EB4310413002EB4313C5
:105F2000C01A02F0C5FB6070C6E0494B4C4A9B7832
:105F30005C010834141904EB4310423002EB4313A4
:105F4000C01A02F0B5FBA070B6E0142100E00421F5
:105F50003F4B987805F05CFEAEE03D4D404CAB7891
:105F6000012204EB43110B31981C01EB401004EBB0
:105F70004313C01A02F078FBA87804EB4014E17ACE
:105F8000C1F10801C9B204F005FA95E01A21DFE772
:105F90001821DDE72E4B324893F802C004224FEA65
:105FA0004C1303F1180141184EE0294B2C4C9B78FF
:105FB0009D000135981C04EBC50202EB401004EB78
:105FC0004313C01A02F074FB04F8350074E0204B50
:105FD00023499B780422981C01EB431140014FE0B8
:105FE0001B4B042299781E4B881C03EB4113991814
:105FF00001EB401043E0164B194893F802C0012210
:106000004FEA4C1319181F311EE0114B14489B78AE
:10601000022200EB43110E3103EB020C08E00C4BA3
:106020000F489B78042200EB4311143103F1020C5A
:1060300000EB431321E0064B094893F802C001220C
:106040004FEA4C1319181E310CF1020C14E000BF7A
:10605000E806002078020020700B00206C0700206A
:10606000F80B0020154B164893F802C002224FEAA5
:106070004C1319181C319444C31801EB4C10C01A6E
:1060800002F0F2FA18E00D4D0D4CAB78012204EB52
:1060900043110C31981C01EB401004EB4313C01A60
:1060A00002F0E2FAAB7804EB4314207BFEF7D4F95C
:1060B00002E00322034B1A7038BD00BFE80600203F
:1060C000F80B002060070020374938B500230B602B
:1060D0003649374A0B60374993740B609360D3603D
:1060E00013745374344A4FF0FF3142F82310334A8B
:1060F0000024D45401332F2BF4D10731204605F06E
:106100002FFB2F4B0C211860204605F029FB2D4D4D
:106110002D4BE97A1860C1F108012046C9B204F09C
:1061200039F9287BFEF798F9284B0022E250043415
:10613000B4F5806FF8D1264B9B7E5BB104F50674F5
:106140002449204609190422043402F08DFAB4F5DA
:10615000CD6FF5D11E4BDB7E5BB94FF4A7641E49B2
:10616000204609190422043402F07EFAB4F5C36F04
:10617000F5D1174B1B79012B03D0112B01D0212B0B
:1061800001D1012200E00022094B83F8D020104BFE
:106190005B7D23B1FEF784F908B1012200E0002203
:1061A000034B83F8D12038BD480700206807002042
:1061B00078020020F00600208C020020700C0020E5
:1061C000700B0020F80B00206C07002070070020E7
:1061D00008000020E00000203802002010B5994B94
:1061E0009A78022A00F05181032A00F05781002A90
:1061F00040F0E7815A784D2A00F0BC8023D8452A28
:1062000070D00ED8422A56D005D8402A45D0412A0F
:1062100040F0D58146E0432A53D0442A40F0CF8154
:1062200056E0482A7BD005D8462A61D0472A40F05C
:10623000C6816AE04B2A00F0848000F29480492AEB
:1062400040F0BD8171E0542A00F0DA8011D8512A63
:1062500000F0B08006D84F2A00F09280502A40F01B
:10626000AE81A0E0522A00F0B780532A40F0A78107
:10627000BCE0832A00F0EC8006D8552A00F0CD80DF
:10628000572A40F09C81D5E0852A00F0F180C0F0CB
:10629000E780FF2A40F09381F3E06A4B40F2FF7001
:1062A000D97805E0674B684ADB78002019461370FF
:1062B00002F094FA88E1DB78634A194601205370B2
:1062C000F6E7604B604ADB78042019461371EFE76C
:1062D0005C4B5D495A68DB781C2043EA022341F895
:1062E0001C3F0EE0DB78584A194605205371DFE762
:1062F000544B55495A68DB780C2043EA022341F895
:106300000C3F042202F0ECF95EE14E4B4E495A6814
:10631000DB78082043EA022341F8083FF1E7DB7805
:106320004949262001F8263F75E0464A464BD27877
:1063300012B1464901224A60DA75434B1720D97DD4
:10634000B6E7404B404CDB7803201946E37002F07F
:1063500045FAE07802F01AFCE07802F017FCE078E9
:1063600002F03CFC30E1374B374ADB78022019461B
:1063700093709DE7DB78344A19461520537597E7EB
:10638000304B314CDB7819201946637602F026FA3F
:10639000607E10F0010002D00020012100E00146E3
:1063A00005F012FB10E1274B274ADB78162019462F
:1063B00093757DE7244A127D12F0010F05D0DB783A
:1063C00013F0010F01D102F0CDFA1E4B1E4ADB780B
:1063D0001420194613756BE71A4B1B495A68DB7872
:1063E000202043EA022341F8203F8AE7154B164953
:1063F0005A68DB78102043EA022341F8103F80E717
:106400005A68DB7843EA0222012A00F2DA800E4958
:106410001A2001F81A3F012274E70A4B5A68DB7808
:1064200043EA0222012A00F2CC8007491B2001F82E
:106430001B3FF0E7034B0449DB78272001F8273F97
:10644000E9E700BFE8060020080000206007002000
:106450005A68DB7843EA02225C4BC3F8D420B3E0ED
:106460005B4B5A68DB7843EA02225A4B1A60ABE076
:10647000574B5A68DB7843EA0222544BC3F8D820C2
:10648000A2E0534BDA78544B9DE05868D9785A789B
:10649000524B41EA002143F8221095E05A78272A0E
:1064A00059D00ED8022A33D004D8CAB1012A40F0FC
:1064B000868021E01B2A3ED01C2A44D0092A7ED1A6
:1064C00032E02B2A5FD005D8292A50D0D978444A07
:1064D00054D847E02D2A64D05CD32E2A6FD167E0D0
:1064E0005A68DB7843EA02223D4B1A6002F050FE04
:1064F000364BC3F8DC0067E05A68DB7843EA0222D7
:10650000374B5A6002F044FE304BC3F8E0005BE0CA
:106510005A68DB7843EA0222314B9A6002F038FE77
:106520002A4BC3F8E4004FE05A68DB7843EA0222C2
:106530002B4BDA6048E05968DB78002043EA012100
:1065400005F03CFB40E05968DB78002043EA01217C
:1065500005F008FB38E05A68DB7843EA0222204B5A
:106560001A6131E05B6841EA032151612CE05A680D
:10657000DB7843EA02221A4B9A6125E05B6841EA24
:106580000321D16120E05A68DB7843EA0222144BF0
:106590001A6219E05A68DB7843EA0222104B5A6209
:1065A00012E05A68DB7843EA02220D4B9A620BE054
:1065B0005A68DB7843EA0222094BDA6204E00322DC
:1065C00000E00422074B1A7010BD00BF78020020C3
:1065D000E80600205C070020590700207007002013
:1065E000200C00206007002008B5824B9A78022A10
:1065F00000F0B980032A00F0BB80002A40F01E8121
:106600005B78502B6ED022D8462B54D00ED8422B1C
:1066100047D005D8402B3DD0412B40F00D813EE0C6
:10662000442B43D0744B754A43D83DE04B2B4DD09F
:1066300006D8482B43D040D3492B40F0FD8042E0A0
:106640004D2B49D045D34F2B40F0F68047E0812BAE
:106650005FD010D8542B4ED005D8522B47D0664B64
:10666000664A46D841E0572B4BD0802B4DD0552B56
:1066700040F0E28042E0852B5DD004D8832B53D0DC
:106680005D4B55D84DE0FE2B64D066D8F02B40F022
:10669000D3805FE040F2FF7002F00AF89CE0574BB5
:1066A00059E0564B5A78C4E01279C3E0534BDA698B
:1066B000BFE05279BEE0514B85E0504B80E04F4B3C
:1066C00093F82620B5E04D4BDA7D48E04B4BDA7865
:1066D000AFE04A4B9A78ACE0484B5A7DA9E0474B73
:1066E0005A7EA6E0454B9A7DA3E0127DA2E0434B83
:1066F00095E012699EE0414B9A7E9AE03F4BDA7E2C
:1067000097E03E4B93F8272093E03D4B93F8D12040
:106710008FE03B4B93F8D120042A14BF00220122C2
:1067200087E0374A926885E0354BD3F8D42080E083
:10673000344A12687EE0324A334BD2F8D8104B43C9
:1067400003F5405339332C4923F000404860C2F828
:10675000D83076E02D4B1A786BE02D4B1A78003A42
:1067600018BF012265E05A782A4B53F8222060E0D6
:106770005B78272B33D00DD8022B20D003D8C3B1A0
:10678000012B59D118E01B2B1FD01C2B21D0092B1A
:1067900052D117E02B2B41D005D8292B24D0164BF2
:1067A0001D4A24D81EE02D2B3ED03AD32E2B43D1A8
:1067B0003DE0194B1A683CE0174B5A6839E0164B1C
:1067C0009A6836E0144BDA6833E0002005F044F8AC
:1067D00002E0002005F02CF8074B586031E00E4B2A
:1067E0001A6926E0526925E00B4B9A6921E0D269CB
:1067F00020E000BFE806002060070020080000201D
:10680000780200205C0700206D4EC641540C002029
:106810005907002070070020200C0020124B1A6A34
:1068200007E0114B5A6A04E00F4B9A6A01E00E4BE5
:10683000DA6A0E4B5A6004E0032200E004220B4B9C
:106840001A700B4B1B786BB1084B0A495A680A4BFC
:106850000A601AB91A6842F0080202E01A6822F0C7
:1068600008021A6008BD00BF200C0020600700204D
:106870005A07002048070020F006002037B5504B8B
:106880001A7CA2B94F494868CA7842EA0022B2F19C
:10689000FF3F04BF4C4A12680A214A43C3F8E8206C
:1068A00002F076FC464B01221A74C3F8EC00454B0B
:1068B0005B78042B00F28280DFE803F003353F4F62
:1068C000130002F065FC3E4BD3F8EC10D3F8E8203F
:1068D000411A0029B8BF494291426CD900221A746A
:1068E0006CE0384B364C987804F0F8FA30B9374AF7
:1068F0002074136823F0100313605FE0D4F8E830CD
:10690000002B57D002F044FCD4F8EC20D4F8E83047
:10691000821A002AB8BF52429A424BD92B4B00210F
:106920001A68217442E0002004F030FE254B244C0C
:106930009D786D0050FA05F51CE000207C2101AA2D
:1069400004F060FF1F4B02229D789DF806306D0019
:1069500012FA05F51A4C1D400EE001AA00207C2118
:1069600004F050FF174A9DF806309578144C6D00DE
:1069700053FA05F515F0010506D0144B00211A68ED
:10698000217422F0100213E0D4F8E83093B102F041
:10699000FFFBD4F8EC20D4F8E830821A002AB8BF04
:1069A00052429A4206D9094B25741A6842F01002E5
:1069B0001A6003E0024B9A68013A9A603EBD00BF3C
:1069C00078020020E806002048070020F00600209A
:1069D00008B5184B9A7812B1022A26D106E05868F9
:1069E000DB7843EA0020FDF717FD21E058780728FF
:1069F0000AD85A68DB7853EA022202D1FDF7B0FCCC
:106A000016E0FDF7B9FC13E0FF280CD15868DB78DD
:106A100043EA0020B0F1FF3F0ABF074BC0B218782D
:106A2000FDF7B6FC04E0032200E00422034B1A70D9
:106A300008BD00BFE80600204807002060070020CE
:106A400010B5224B9A78012A23D003D3022A204C76
:106A500028D122E05878082802D8FDF74FFD15E02C
:106A60000A2801D100220AE00B2802D1FDF7BEFD61
:106A70000CE00C2806D1174B9A68C2F34012144B55
:106A80005A6011E0FF280FD1FDF75CFD104B5860F4
:106A90000AE0587802F098FBF8E75878FDF78CFC8C
:106AA000606001E0042323700B4B1B786BB1084B33
:106AB0000A495A680A4B0A601AB91A6842F0080271
:106AC00002E01A6822F008021A6010BDE8060020F1
:106AD00060070020000C01405A07002048070020F2
:106AE000F006002010B5204B5A78812A3AD19A78C6
:106AF000922A37D19A79A32A34D15A79B42A31D13A
:106B00001A79C52A2ED1DB78D62B2BD1174B4FF40F
:106B100080621A6102F0E0FE02F03AFB044602F0E5
:106B200037FB001B0028B8BF4042B0F57A7FF6DB88
:106B3000FDF760FC06F09CFA002006F0C9FF00217A
:106B40000B4805F04BFE0A4805F0A8FD094805F082
:106B50007BFD05F093FE4FF0804007F03DFD0020E7
:106B6000FDF7ACFE10BD00BFE8060020000C0140A0
:106B700008000240002401402DE9FF479C4C9D4D38
:106B8000E07862682378642140EA0220222B297091
:106B90006B70686000F0D58554D80F2B00F0CE8262
:106BA00024D8072B00F0388210D8032B00F0F8808F
:106BB00006D8012B00F0A680022B41F04080C8E0EF
:106BC000052B00F0218200F2238201E10B2B00F063
:106BD000338205D8092B00F0278200F229821FE2B8
:106BE0000D2B00F05E8200F2A5823EE2192B00F030
:106BF0004B8412D8152B00F03B8306D8132B00F0E2
:106C0000A182142B41F01B8004E3172B00F01C849D
:106C1000794B00F22C8400F010BC1E2B00F05E8437
:106C200009D81B2B00F05284C0F03E841C2B41F08D
:106C3000068000F04EBC202B00F0E28400F22B8591
:106C400000F088BC812B00F03C862ED8412B00F050
:106C50001E8615D8252B00F0BA8507D8232B00F007
:106C60007C85242B40F0EB8700F083BD272B00F0C0
:106C7000E585C0F0B785402B40F0E18700F004BE09
:106C8000452B00F0108606D8432B00F0068600F254
:106C9000078600F0FFBD472B00F00B86C0F006868C
:106CA000802B40F0CC8700F007BE882B00F09A863E
:106CB00012D8842B00F03F8607D8822B00F019866B
:106CC000832B40F0BC8700F019BE862B00F04D8668
:106CD00000F2A88600F044BE8C2B00F0228706D874
:106CE0008A2B00F0FF8600F2178700F0C9BEF22B56
:106CF00000F09487FF2B00F094878D2B40F09F8746
:106D000000F037BFA378FBB93B4B4FF0010C83F881
:106D100004C03A4B00241C70394B21461C7020469D
:106D2000022204F0F7FC2046062140F2FF7204F034
:106D30005DFE2F4B20465A68DB78082143EA022289
:106D400004F054FE00F07EBF2A4B04221A7000F0BB
:106D500079BF274DAC78F4B9274B4FF0010C83F87D
:106D600004C0264B21461C70254B20461C70022275
:106D700004F0D0FC2046062140F2FF7204F036FEFB
:106D80006A68EB78204643EA02225242082104F066
:106D90002DFE00F057BF174B04221A7000F052BFAF
:106DA000A4788CB9154B20461C70154B1C7004F050
:106DB0008DF820462146022204F0ACFC2046082132
:106DC00004F028FE00F03EBF04232B7000F03ABF11
:106DD000074B9A78002A40F012815B78032B00F26F
:106DE0000981DFE813F00F005800AE00DE0000BF9D
:106DF000E80600206007002078020020EC0B00204D
:106E0000900B0020AD4D0020FDF7A8FFAB784FF0B0
:106E1000010C0CFA03FCAA4EAA4F002496F800E0DD
:106E20006868EA78FC54A84F59012EEA0C0C42EA33
:106E30000022FC5401F0E001204686F800C004F076
:106E400041FDA9782246204604F064FCA9789F4AB7
:106E500002EB41139B7F002B00F0F486002900F029
:106E6000F186927F9A4240F0ED862046FDF776FF4C
:106E700033786968EA7823F0010342EA0122204668
:106E80002146337004F01EFD20462146224604F0C0
:106E900041FC00F0D7BE894D0020FDF75FFFAB78C5
:106EA000884A00245901D454874A41F00201D4543D
:106EB00001F0E201204604F053FCA97801238B4045
:106EC000EA786F687E4E42EA07273278C71922EACD
:106ED00003034901337001F0E0013A46204604F013
:106EE000F1FC2046A978224604F014FCA878774AE1
:106EF000774902EB40139B7F4F60002B00F0A28686
:106F0000002800F09F86927F9A4240F09B86FDF712
:106F100025FF0221204604F023FC6968EA783378D3
:106F200042EA012223F001038218214620463370F1
:106F300004F0C8FC20462146224604F0EBFB00F09A
:106F400081BE5E4CE378626843EA0223142B23DCA3
:106F5000604A002052F82370FDF700FFA3784FF03D
:106F6000010C0CFA03FC564E00253278590122EA36
:106F70000C0C86F800C0534E3A46F554524E284643
:106F800001F0E001F55404F09DFC2846A1782A4662
:106F900004F0C0FB00F056BE4D4B04221A7000F006
:106FA00051BE464C0020E3786268454E43EA022217
:106FB000484B002553F82270FDF7D0FEA3784FF020
:106FC000010C0CFA03FC3278590122EA0C0C86F809
:106FD00000C03C4E3A46F5543B4E284601F0E001D5
:106FE000F55404F06FFC2846A1782A4604F092FB81
:106FF00000F028BE364B03221A7000F023BE344B3B
:1070000004221A7000F01EBEFDF7CAFE00F01ABE80
:10701000FEF75CFA00F016BEFEF7BEFD00F012BEF1
:10702000FEF7D8FE00F00EBEFFF7D8F800F00ABE5B
:10703000FFF7DAFA00F006BEA378022B11D16378CD
:10704000372B0AD8244903F5A77001EB8301800090
:10705000042201F045FB00F0F5BD03232B7000F086
:10706000F1BD04232B7000F0EDBD144B9A78022A79
:1070700012D15B78372B0AD8174903F5A77001EBBB
:1070800083018000023201F0EFFA00F0DBBD104B0B
:1070900003221A7000F0D6BD0D4B04221A7000F0C6
:1070A000D1BDA378002B40D1044C6378012B2DD0A7
:1070B00014D3022B064C34D12DE000BFE80600208B
:1070C0007D0B0020900B0020EC0B0020F80B002023
:1070D00060070020F406002070070020002003F065
:1070E000EDFEA17851B1994A937F002B00F0AA855B
:1070F00002EB4112927F9A4240F0A485944B012208
:107100001A71944B013A1A7000F09CBD002003F0F4
:10711000DDFE00F097BD002003F0E0FE606000F0AF
:1071200091BD0323237000F08DBD8B4B04221A7098
:1071300000F088BDFFF74CFC00F084BDFFF780FC39
:1071400000F080BD6278854B092A53D8DFE802F051
:10715000050D151D26313941494C814A1968506881
:10716000D27842EA0022521843E07D4A19685068FA
:10717000D27842EA00228A1A3BE0794A19685068BC
:10718000D27842EA00224A4333E0754A19685068CF
:10719000D27842EA002291FBF2F22AE070481968A4
:1071A0004468C27842EA042291FBF2F002FB10121A
:1071B0001FE06B4A19685068D27842EA00220A4000
:1071C00017E0674A19685068D27842EA00220A43F9
:1071D0000FE0634A19685068D27842EA00224A40B8
:1071E00007E01A68D24304E05D4A5168D27842EA67
:1071F00001221A60594A5B4B12682AB91A6842F098
:1072000008021A6000F01EBD1A6822F008021A6017
:1072100000F018BD524B514A5968DB78126843EAB6
:1072200001239A4206DD4F4B1A6842F0040222F015
:1072300003020CE04B4B05D11A6822F0060242F023
:10724000010204E01A6822F0070242F002021A600A
:10725000424A444B12682AB91A6842F008021A607E
:1072600000F0F0BC1A6822F008021A6000F0EABCD4
:1072700063780C2B00F2E684DFE813F00D001C00AD
:107280002B003A0049005800760085009400A300C6
:10729000B200C100D000334B1B6813F0080F00F0A0
:1072A000D1842F4B5A68DB7843EA0222284B9A603C
:1072B00000F0C8BC2B4B1B6813F0080F40F0C284D1
:1072C000274B5A68DB7843EA0222214B9A6000F090
:1072D000B9BC244B1B6813F0010F00F0B384204BA2
:1072E0005A68DB7843EA0222194B9A6000F0AABC84
:1072F0001C4B1B6813F0010F40F0A484184B5A6814
:10730000DB7843EA0222124B9A6000F09BBC154BDB
:107310001B6813F0040F00F09584114B5A68DB785A
:1073200043EA02220A4B9A6000F08CBC0D4B1B68AA
:1073300013F0050F00F08684094B5A68DB7843EAA6
:107340000222034B9A6000F07DBC00BFF80B0020C6
:1073500078020020900B00206007002048070020E2
:10736000E8060020F00600209B4B1B6813F0020F7C
:1073700000F06884994B5A68DB7843EA0222984B04
:107380009A6000F05FBC944B1B6813F0030F00F091
:107390005984924B5A68DB7843EA0222904B9A60F8
:1073A00000F050BC8C4B1B6813F0100F00F04A84A7
:1073B0008A4B5A68DB7843EA0222894B9A6000F0D4
:1073C00041BC854B1B6813F0200F00F03B84834BBE
:1073D0005A68DB7843EA0222814B9A6000F032BCA3
:1073E0007D4B1B6813F0400F00F02C847B4B5A68D8
:1073F000DB7843EA02227A4B9A6000F023BC764B9A
:107400001B6813F0800F00F01D84744B5A68DB7802
:1074100043EA0222724B9A6000F014BC6E4B1B6868
:1074200013F4807F00F00E846C4B5A68DB7843EADB
:1074300002226B4B9A6000F005BC684A5168D27812
:1074400042EA01229A60FDE3654BDA68072A00F2FE
:10745000F98362499C684868C97841EA0020511C58
:1074600003EB8202C2F8F0409860D960EAE3DA6880
:107470005B4B002A00F0E683013A03EB8201D1F86E
:10748000F010DA609960DDE363782E2B03D8554A5B
:107490000121D154D6E3FF2B03D1514B01225A7461
:1074A000D0E303232B70CDE34C4B5B782E2B03D81A
:1074B0004C4A0021D154C5E3FF2B03D1484B002295
:1074C0005A74BFE3484B03221A70BBE3FFF7D6F9A7
:1074D000B8E3434B002283F8D120B3E36378142B45
:1074E00035D8A278A2B9414A4149927E41F8230099
:1074F000002A00F0A783002B00F0A48303F5C270DC
:10750000013001EB83018000042201F0E9F899E3E6
:10751000FF2A18D163B94FF4C364364920460919CC
:107520000422043401F0DCF8B4F5CD6FF5D189E321
:1075300003F5C2702E49013001EB83018000042263
:1075400001F0CEF87EE3284B04221A707AE303237D
:107550002B7077E36378142B39D8204A9278BAB924
:10756000234A214952F82320234B4A601B78002BE1
:1075700000F068832149184B0A6022B91A6842F06A
:1075800008021A605EE31A6822F008021A6059E3E2
:10759000FF2A18D163B94FF4C3641649204609196C
:1075A0000422043401F060F8B4F5CD6FF5D149E35D
:1075B00003F5C2700E49013001EB83018000042203
:1075C00001F052F83EE3084B04221A703AE3064BEE
:1075D00003221A7036E300BFF0060020E806002000
:1075E00078020020700C00206007002008000020B6
:1075F000F4060020E00000205A0700204807002081
:107600006578142D43D8934CA07810F0800F1ED0CD
:1076100010F0010F06D00020022104F0A1F88E4BDB
:1076200043F825008D4B9B7E002B00F00B83894B8C
:107630005B78002B00F0068303F5C27086490130A9
:1076400001EB83018000042201F04AF8FAE2D0B98C
:10765000022104F085F8814A7F4B927E43F8250091
:10766000002A00F0EF826178002900F0EB82A07818
:107670000422091801F5C270013003EB810180007A
:1076800001F02EF8DEE2764B04221A70DAE2744B37
:1076900003221A70D6E26278724B0A2A43D8DFE8D6
:1076A00002F0060B11161C242A30363A3D006E49B2
:1076B0001A6809688A1803E06B4A196812688A1AFE
:1076C0001A6030E0684A196812684A43F8E7664A67
:1076D0001968126891FBF2F2F2E7634A19681268BE
:1076E00091FBF2F002FB1012EAE75F491A680968A1
:1076F00001EA0202E4E75C491A68096841EA020209
:10770000DEE759491A68096881EA0202D8E7564B50
:107710001A68D243D4E71A68534BD1E7524A186823
:107720001168106019604F4A504B126822B91A68EC
:1077300042F008021A6085E21A6822F008021A6014
:1077400080E2484B02F07F4219681B7842EA11221E
:107750006260E370FDF724FB74E2424B02F07F426B
:1077600019681B7842EA11226260E370FEF736FD69
:1077700068E2384B5B78052B00F26482DFE803F0A7
:1077800003090F151B21394B1A6802F00F021A600A
:1077900058E2364B1A6822F010021A6052E2334B5C
:1077A0001A6822F020021A604CE2304B1A6822F06C
:1077B00040021A6046E22D4B1A6822F080021A60DD
:1077C00040E22A4B1A6822F480721A603AE2637827
:1077D0002E2B04D8264A02EB8303586132E203239E
:1077E0002B702FE2224BDFF87CC0D3F81091214997
:1077F00093F82C21D3F814A1CCF80090DFF868C0DE
:10780000D3F81871D3F81C81D3F82061D3F8245130
:10781000D3F82841CCF800A0885CDFF850C09F6006
:10782000CCF800801E74C3F8EC50C3F8E84008B1EF
:1078300001238B540E4B00229A7403E2A378FBB908
:10784000044B5B78142B17D8064A1168024A42F899
:107850002310F7E1E8060020F406002008000020CD
:10786000600700204807002068070020F00600207D
:1078700078020020700C00208F4B03221A70E1E187
:107880008D4B04221A70DDE102F082F8DAE102F099
:1078900081F8D7E102F080F8D4E102F07FF8D1E17D
:1078A00002F098F8CEE102F097F8CBE102F096F8FA
:1078B000C8E102F095F8C5E1804B002283F8D120A1
:1078C000C0E1637813B1012B10D104E07B4B01229E
:1078D00083F8D120B6E1B0F5006F04D2774A90600A
:1078E00082F8D130AEE104232B70ABE103232B707F
:1078F000A8E1724B022283F8D120A3E16F4B002153
:10790000997459746D4A4FF0FF3402F1140040F835
:1079100021406B480023435401312F29F2D169499A
:1079200013740B60684982F8D1300B60674993602B
:107930000B60D36086E1664B1B7D13F0020F0CD108
:10794000B0F5006F06D25D4B0422C3F8300183F816
:10795000D12077E104232B7074E108232B7071E1AF
:10796000564B002283F8D1206CE1594B01219A78C3
:10797000584BB0F5006F1970574B1A7028D2544B02
:107980001C7D0C4024D101A901F030F8524B9DF828
:1079900004709DF805609DF806509DF80AC09DF89A
:1079A00009009DF808109DF807201C725F709E70FA
:1079B000DD7083F804C058719971DA710123464A69
:1079C000985C117A01334118082B1172F7D139E113
:1079D0000123414A002199540133082BF9D113782E
:1079E00013722FE163788BB9394A012091783B4AB1
:1079F0001468384A1070384A11700133E21812F8CE
:107A0000011C354A082B9954F7D11BE1012B40F09A
:107A100019811D222A710422EA716FF07602AA717F
:107A20006B710FE12E4B5B78032B00F20B81DFE8CB
:107A300003F002101D22214A1F4BD2F8301192F898
:107A4000D1C0107C0A0A197183F807C098715A7165
:107A5000F8E01A4A184B916892F8D1C0107C0A0AD3
:107A6000197183F807C098715A71EBE0164B1A68C8
:107A7000114B5A60E6E0154B1A680F4B5A60E1E073
:107A8000174B5A78002A40F0DD809978002940F0A1
:107A9000D9805A68DB7843EA022240F2D2439A4204
:107AA00040F0D08040F2FF7000F098FE00F05AFFE6
:107AB0000120FCF703FFC5E06007002078020020EA
:107AC000700C0020F0060020480700206807002006
:107AD000080000204C070020500700200000002074
:107AE000E80600206278584B02B1012257491A700B
:107AF000574B0878DA78574B42EA000093F834C1C4
:107B0000554C0870554984F800C00A70544C554AC9
:107B100000232370137095E04E4B012283F835212A
:107B200090E0667816B1012E20D111E0042240F2D7
:107B3000FB7003A900F098FDE378626843EA022233
:107B4000039B9A4202D101236B607BE06E6079E077
:107B5000A3782A2B06D140F2FB704349042200F09F
:107B6000BFFD6FE0414B03221A706BE003232B70C3
:107B700068E0374B5B78032B4CD8DFE803F00C024E
:107B80003C47334B33495A68DB78D1F8381143EA24
:107B9000022C00232BE02F4BD3F83821092A0CD8D4
:107BA0002B49501C4C68C97803EB820241EA04213E
:107BB000C2F83C11C3F8380144E02C4B09221A707A
:107BC00040E052F82340581C64450FD102EB80027C
:107BD000013904E052F8040C013342F8080C043275
:107BE0008B42F7D31B4BC3F838112BE003468B4273
:107BF0001F4AE6D326E0174A0023C2F838311C4A50
:107C00000021D1500433282BF9D11BE0174B0A2255
:107C10005A6017E0154B03221A7013E0FEF762FF5B
:107C200010E00B4B5A68DB7843EA022240F2D24361
:107C30009A4207D1074B012283F8642102E00B4BE3
:107C400002221A70BDE8FF877C0B00207D0B00200C
:107C5000E8060020780200205E0C0020980B00202F
:107C60009F0C0020910B0020EB06002060070020F5
:107C7000B403002073B5204B024640781F4D1870A6
:107C8000907800265870D078EC46987010790C46A1
:107C900098715079587192F806E095E8030083F8DE
:107CA00004E0D2798CE80300DA70154B1E70FEF701
:107CB00063FF144B1B7873B9637023702B78A37028
:107CC0006B78E370EB792371AB7963716B79A37196
:107CD0002B79E37108E0012B06D10B4B9B195B78E4
:107CE000A3550136082EF8D1044B6A4692E80300EA
:107CF00083E803007CBD00BFE80600206007002089
:107D00005A0700204C07002050070020F7B5114DFE
:107D1000114C6F684FF0000C07F07F4747EA1327BC
:107D20006F600E4F6E4687F800C028706970AA70A9
:107D300094E80300EB7086E80300FEF71DFF96E869
:107D400003006368227884E80300054918460A7036
:107D5000FEBD00BFE8060020600700205A07002093
:107D6000780200202DE9F04F7E4B93B01B781BB9B1
:107D70007D4B93F865316BB17C4B1B78062B09D09A
:107D80000A2B07D00F2B05D01F2B03D0764B0022D8
:107D900083F83421744A92F83431032B25D192F8B8
:107DA000D040002C40F0D980714B1B7893B9714DB5
:107DB000714CA8786E78227863788619B618E279C3
:107DC000F618A379B6186279F6182379B618F6185A
:107DD000F6B219E0012B40F0FE80684BE05C013404
:107DE00000F040FF092CF8D1F5E0042B27D1614DBC
:107DF000614CAB786E7818469E190136002301223B
:107E000022706360F6B2637000F02CFF687800F0B7
:107E100029FF207800F026FF607800F023FFE0794A
:107E200000F020FFA07900F01DFF607900F01AFF3C
:107E3000207900F017FF304600F014FFCBE0052B4F
:107E400025D192F8D040002C40F08780484B1B7819
:107E500093B9484D484CA8786E7822786378861993
:107E6000B618E279F618A379B6186279F61823796C
:107E7000B618F618F6B219E0012B40F0AC803F4B73
:107E8000E05C013400F0D2FE092CF8D1A3E0062B0F
:107E900027D1384D384CAB786E7818469E1901368C
:107EA0000023012222706360F6B2637000F0BEFE10
:107EB000687800F0BBFE207800F0B8FE607800F033
:107EC000B5FEE07900F0B2FEA07900F0AFFE607977
:107ED00000F0ACFE207900F0A9FE304600F0A6FECE
:107EE00079E0072B4ED192F8D030002B35D1204AC3
:107EF000127822BB1F4A204B557896781C7893F84D
:107F000001C0AF19D879E719997967445A79C71927
:107F10001B79CF19D719DF198DF838708DF83060BB
:107F20008DF831508DF832408DF833C08DF8340023
:107F30008DF835108DF836208DF8373008E0012A9D
:107F400006D10E4A995C0CAAD1540133092BF8D101
:107F50000B4B1B78002B3ED039E0074803F094FF11
:107F600039E000BF5907002078020020E806002011
:107F70004C07002008000020600700205007002068
:107F8000740B0020082B26D1954B00225978987845
:107F9000944B45181C78944B4FF0010C01355A60F6
:107FA0008DF832C08DF8332016468DF834208DF8C8
:107FB00035208DF836208DF837208DF838505A70DE
:107FC00083F800C08DF830008DF831101CB10CA87A
:107FD000092101F04FFB854B1B78002B56D0844BB9
:107FE0001B78032B02D0072B4BD123E07C4C814D17
:107FF000A07866782B7886190A36F61800F032FEDB
:10800000607800F02FFE802000F02CFE8A2000F027
:1080100029FE002000F026FE002000F023FE0020B4
:1080200000F020FEF6B2287800F01CFE304600F08A
:1080300019FE26E06A4B6FF07F05597898786D4BF2
:1080400000EB010C1A78674B0CF10A0C1C78944475
:1080500000238DF826500A358DF827508DF82A30E8
:108060008DF82CC08DF824008DF825108DF828305F
:108070008DF829308DF82B201CB109A8092101F0B9
:10808000F9FA5A4A002313705A4A13705A4B5B4844
:1080900093F864110022027083F8652183F834217B
:1080A00011B10120FCF70AFC534B93F8352152B172
:1080B00093F8D0200021D2F1010238BF002283F8CA
:1080C000351183F8D0204C4C94F8D050002D72D14B
:1080D0000DF1470000F044FD00286CD000F05CFD7D
:1080E00008B184F86651444B9DF8470093F8661137
:1080F0004A1CD2B2C918092A81F8680183F866219E
:1081000040F07681364993F8682148784FF0000CAA
:10811000904283F866C107D091F82730002B00F019
:1081200067819A4240F064812D4B93F82730934247
:1081300003D1314B012283F8652100231A462E4CCE
:1081400004F5B471C95C01335218082BD2B2F6D1D0
:1081500094F8703193422CD1294B94F86D1194F816
:108160006E2194F86F5194F8696194F86AE194F87B
:108170006BC194F86C01DD7059711A711E7083F82F
:1081800001E083F802C0987101F002F81D4D94F8E7
:10819000D1302860591E1C480022C9B20270032049
:1081A000012984F8340184F8662140F2EE80052B21
:1081B000A0E00423EDE0104C94F8D03033B3104825
:1081C00003F0A8FE10B300F0E3FF0E4994F8D1309D
:1081D00008600D495A1E00200870D2B20321CEE07B
:1081E00008000020740B0020600700209F0C002076
:1081F0005E0C0020910B0020780200204C0700202C
:10820000E8060020580C00205D0C00206F4C94F80C
:10821000D050002D73D10DF1470000F0C7FC0028AD
:108220006DD000F0E1FC08B184F86651674B9DF811
:10823000470093F866114A1CD2B2C918092A81F87E
:10824000680183F8662140F0D380614993F8682182
:1082500048784FF0000C904283F866C107D091F83F
:108260002730002B00F0C4809A4240F0C180584B68
:1082700093F82730934203D1544B012283F86521B0
:1082800000231A46514C04F5B471C95C01335218ED
:10829000082BD2B2F6D194F8703193422DD14D4BC8
:1082A00094F86D1194F86E2194F86F5194F8696107
:1082B00094F86AE194F86BC194F86C01DD7059711F
:1082C0001A711E7083F801E083F802C0987100F003
:1082D0005FFF414D94F8D1302860591E3F4800227D
:1082E000C9B202700520012984F8340184F866219E
:1082F0004BD9834249D0013248E0062349E0334B51
:1083000093F8D040002C47D1354B1B78002B43D03D
:108310000FA801F099F900283ED0234622460FA964
:10832000C95C01335218082BD2B2F8D19DF8441021
:10833000264C91422DD1274B9DF841109DF84220AB
:108340009DF83D609DF83EE09DF83FC09DF84000DF
:108350009DF8435059711A711E70DD7083F801E069
:1083600083F802C0987100F013FF1B4994F8D130D4
:1083700008601A495A1E00200870D2B20721012A4B
:1083800084F8341101D9052B1ED10022154B1A7027
:108390002EE084F834312BE00C4C94F8D130013BC2
:1083A000DBB2012B24D8A368B3F5006F1CD2FCF715
:1083B00077F8C8B1A368074918460133A36000F0F5
:1083C00015FB092384F834310122DFE7780200200D
:1083D00008000020E8060020580C00205D0C00205A
:1083E000740B00205A070020964B002283F8D120FE
:1083F000944C94F8D130042B05D1934E327812F07E
:10840000800F00F0EF808F4B93F834313BB1042B99
:1084100005D0082B03D0062B01D0FEF7ADFB894C0D
:1084200094F83431092B40F0B28000F0B1FED4F85A
:10843000DC30864AC31A002B1268B8BF5B429342F5
:108440000AD9834B1A78012A01D101321A7000F03F
:108450009FFE7C4BC3F8DC0000F09AFE794BD3F80A
:10846000E0207A4B821A002A5B68B8BF52429A42D7
:108470000AD9774B5A78012A01D101325A7000F09B
:1084800087FE704BC3F8E00000F082FE6D4BD3F81E
:10849000E4206E4B821A002A9B68B8BF52429A426F
:1084A0000AD96B4B9A78012A01D101329A7000F0F7
:1084B0006FFE644BC3F8E400624A537C002B66D025
:1084C000937C002B63D19C46624B92F82C011B6875
:1084D00002900793604BD2F8E8001B680390069364
:1084E0005E4BD2F810811B68D2F814710593D2F854
:1084F000EC30D2F818410493D2F81C619368107CD8
:10850000D2F82051D2F824B1D2F828210192624643
:10851000DFF83C91194619F802A0BAF1020F18D100
:108520004F4951F82210B1F1FF3F0ED00546D0B2AD
:1085300002900398DDF810B00190059E069FDDF8CB
:108540001C804FF0010C002004E0002109F802100B
:108550001946234601322F2A02D01C460B46D7E784
:10856000384AC2F818311074019B029882F812C080
:10857000C2F81081C2F814719160C2F81C61C2F88F
:108580002051C2F824B1C2F8283182F82C012D4BB9
:1085900093F83421092A06D193F8D120022A02D176
:1085A000033283F8D120274BD3F83811002946D065
:1085B00093F83421092A42D193F8D120012A3ED1DF
:1085C0009868002308E054F823400133A04203D107
:1085D000052382F8D13032E01A4A8B4202F59E74AC
:1085E000F1D32CE094F834314BB3042B27D0082B73
:1085F00025D0062B23D0F3787168D4F83001194DBB
:1086000043EA0123B0F5006F6A706B6012D2314605
:1086100000F01CF93146D4F8300100F03FF930B1D8
:10862000D4F830310133C4F83031652300E007233A
:108630002B7004E007232B70002384F8D13013B093
:10864000BDE8F08F78020020E8060020200C002012
:10865000700C00204807002068070020F00600206A
:108660008C0200206007002070B5044600200E46F2
:10867000154603210246FCF7F3F90020C4F3072155
:108680000246FCF7EDF90020E1B20246FCF7E8F9FA
:10869000002407E0944214BF00220122FCF7E0F915
:1086A0003055013400206A1EAC420146F2D370BD41
:1086B00010B50446002003210246FCF7D1F9002042
:1086C000C4F307210246FCF7CBF90020E1B20246D1
:1086D000FCF7C6F9002001460122FCF7C1F910BDE4
:1086E0002DE9F04104460F461646002006210122DE
:1086F000FCF7B6F9002005210246FCF7B1F900208D
:1087000001220146FCF7ACF910F0020FF2D0002074
:1087100002210246FCF7A4F90020C4F30721024617
:10872000FCF79EF90020E1B20246FCF799F900251A
:1087300043E0013414F03F08795D01D1012204E0E7
:10874000721E954214BF002201220020FCF788F916
:10875000B8F1000F30D1731E9D422DD200200521AB
:108760000246FCF77DF9002001220146FCF778F96A
:1087700010F00100F2D106210122FCF771F900206E
:1087800005210246FCF76CF9002001220146FCF7A6
:1087900067F910F0020FF2D0002002210246FCF728
:1087A0005FF90020C4F307210246FCF759F90020C5
:1087B000E1B20246FCF754F90135B542B9D30020C5
:1087C00005210246FCF74CF9002001220146FCF786
:1087D00047F910F0010FF2D1BDE8F08138B5012260
:1087E00004460D4600200621FCF73AF90020052139
:1087F0000246FCF735F9002001220146FCF730F96A
:1088000010F0020FF2D0002002210246FCF728F9F6
:108810000020C4F307210246FCF722F90020E1B250
:108820000246FCF71DF9294600200122FCF718F941
:10883000002005210246FCF713F900200122014621
:10884000FCF70EF910F0010FF2D138BD38B507254D
:10885000454305F500650C46284609780135FFF7C4
:10886000BDFF284661780135FFF7B8FF2846A1789B
:108870000135FFF7B3FF2846E1780135FFF7AEFF7A
:10888000284621790135FFF7A9FF28466179FFF7CE
:10889000A5FF681CA179FFF7A1FF38BD2DE9F347BB
:1088A0000725454300200C4602460321FCF7D8F873
:1088B00005F500650020C5F307210246FCF7D0F856
:1088C0000020E9B20246FCF7CBF800200146024640
:1088D000FCF7C6F88246002001460246FCF7C0F8C5
:1088E0008046002001460246FCF7BAF80746002001
:1088F00001460246FCF7B4F88146002001460246D4
:10890000FCF7AEF80646002001460246FCF7A8F840
:108910000546002001220146FCF7A2F823785345C2
:108920001DD1637843451AD1A378BB4217D1E378B0
:1089300021798DF804608DF805508DF80600627974
:1089400043EA012343EA0243A079019A43EA006023
:1089500049EA0229814514BF0020012000E00020DF
:10896000BDE8FC8738B54FF40064002006210122E1
:10897000FCF776F8002005210246FCF771F800208C
:1089800001220146FCF76CF810F0020FF2D0002033
:1089900002210246FCF764F80020C4F307210246D6
:1089A000FCF75EF80020E1B20246FCF759F800251A
:1089B00000203F2D14BF0022012201460135FCF7A3
:1089C0004FF8402DF4D1002005210246FCF748F86D
:1089D000002001220146FCF743F810F0010FF2D10C
:1089E0004034B4F5804FC0D138BD00BF38B507253D
:1089F000454300200C4602460321FCF731F805F5FB
:108A000000650020C5F307210246FCF729F8002085
:108A1000E9B20246FCF724F8002001460246FCF7C2
:108A20001FF82070002001460246FCF719F860701C
:108A3000002001460246FCF713F8A0700020014612
:108A40000246FCF70DF8E070002001460246FCF7F4
:108A500007F82071002001460246FCF701F860711A
:108A6000002001460122FBF7FBFFA07138BD00BFCB
:108A700037B5002005210246FBF7F2FF0020012256
:108A80000146FBF7EDFF10F07104F2D100F080FB1E
:108A9000054605E0FFF70CFE422814BF0024012420
:108AA00000F076FB431B002BB8BF5B42B3F5FA6FB7
:108AB00040F2FF7002DA002CECD000E01CB1234B36
:108AC0001B78002B36D040F2FF700021FFF786FEA6
:108AD000FFF748FF00201E494022FFF701FE4FF438
:108AE00080701C49B422FFF7FBFD40201A49202268
:108AF000FFF7F6FD002301934FF4C36401AD204658
:108B0000042204342946FFF7EBFDB4F5FF6FF5D1DD
:108B100000230193A4F5307420460422043429462E
:108B2000FFF7DEFDB4F5C36FF6D140F2FF704221CE
:108B3000FFF754FE002040220549FFF795FD402035
:108B400006492022FFF790FD3EBD00BFA00B00208C
:108B500008000020581D0108881D0108F80B00209E
:108B6000094B19685A68914201D100200BE01A683C
:108B7000D118097A013201701A601A68202A01D1CD
:108B800000221A6001207047EC030020014B98621C
:108B9000704700BFEC030020034B1A78104612B157
:108BA00000221A7001207047B00C00200A4BD96ACD
:108BB0001A6B914201D100200CE0DA6AD11891F8C9
:108BC000341001320170DA62DA6A202A01D10022FF
:108BD000DA620120704700BFEC030020014B5865AA
:108BE000704700BFEC030020034B1A78104612B107
:108BF00000221A7001207047B10C002008B5FBF765
:108C0000F9FB034B0022DA621A63FBF7F1FB08BDA4
:108C1000EC03002008B5FBF7EDFB034B00221A60C4
:108C20005A60FBF7E5FB08BDEC03002038B50B4BA1
:108C300084469C6DDA6D0134202C08BF00249442D8
:108C40000AD09D6D0648ED1885F860C040F2277186
:108C500001229C6505F058FD38BD00BFEC030020E3
:108C60000044004038B50D4B8446D3F88040D3F81B
:108C700084200134202C08BF002494420CD0D3F867
:108C800080500748ED1885F888C040F2277101220E
:108C9000C3F8804005F038FD38BD00BFEC0300206C
:108CA0000038014038B50546002401E0FFF7DAFF3F
:108CB0002B5D01341846002BF8D138BD2B4910B577
:108CC0000B8813F0200F1DD0294BDB6813F0020F27
:108CD00001D08B8816E0274B1A6BD86A0132202A04
:108CE00008BF0022824206D01C6B8888E118C0B2FF
:108CF00081F834001A63204B0A221A601D4B5A6D0A
:108D00001E4B1A601948038813F0800F1BD01B4BB1
:108D10001A68C2B9174B9C6DD96D8C420FD014499B
:108D200002240C61D96DCC1894F860C00131A0F810
:108D300004C0D965D96D202905D1DA6503E040F278
:108D4000277105F0E1FC0948038813F0400F0BD0B0
:108D500040F2266105F0D0FD064BDA6D9B6D9A421C
:108D600002D1034B02225A6110BD00BF00440040F3
:108D700000080140EC030020A00C0020A80C0020FB
:108D8000274910B50B8813F0200F15D0254B5A68D2
:108D900018680132202A08BF0022824205D05C6890
:108DA0008888E118C0B208725A601F4B0A221A6004
:108DB0001C4B9A6A1D4B1A601948038813F0800FE8
:108DC0001ED01A4B1A68DAB9164BD3F88040D3F884
:108DD00084108C4210D0D3F88410CC1894F888C03A
:108DE0000131A0F804C0C3F88410D3F884102029FE
:108DF00006D1C3F8842003E040F2277105F084FC1B
:108E00000748038813F0400F08D040F2266105F0B0
:108E100073FD044BD3F88420D3F8803010BD00BF1D
:108E200000380140EC030020AC0C0020A40C002012
:108E300030B5054687B0564805F0AEFD4FF400301A
:108E4000012104F0F7FB0420012104F0E5FB0420DC
:108E5000002104F0FDFB0820002104F065F806ACB9
:108E60004FF0040324F8083D03234A4821468DF8B7
:108E7000123015338DF8133003F0C6FF48234548F0
:108E80008DF8133021464FF00803ADF8103003F091
:108E9000BBFF684605F002FC0B2D25D8DFE805F086
:108EA0002406090C0F1215181B1E20224FF46153C3
:108EB0001CE04FF4964319E04FF4E14316E04FF401
:108EC000164313E04FF4614310E04FF496330DE086
:108ED0004FF4E1330AE04FF4613307E02E4B05E035
:108EE0002E4B03E02E4B01E04FF416530093009BF2
:108EF00006A95B0841F8183D2548694605F004FDC0
:108F000026230024012505A88DF8143007238DF8A9
:108F100015308DF816408DF8175004F0E5F81C4810
:108F200040F2FF3105F0C4FC28212246184805F024
:108F3000EBFB2A46164840F2277105F0E5FB2A466E
:108F4000134840F2266105F0DFFB2A46104840F244
:108F5000255105F0D9FB22460D4840F2244105F089
:108F6000D3FB22460A4840F6460105F0CDFB2246D7
:108F7000074840F66A1105F0C7FB60212246044805
:108F800005F0C2FB2946024805F0B0FB07B030BD32
:108F9000004400400008014090D0030020A10700D9
:108FA00040420F0030B5054687B0524805F0F4FC4A
:108FB0004FF48040012104F02FFB0420002103F036
:108FC000B3FF06AC4FF4007324F8083D03234A486E
:108FD00021468DF8123015338DF8133003F014FF4D
:108FE000482345488DF8133021464FF48063ADF88F
:108FF000103003F009FF684605F050FB0B2D25D813
:10900000DFE805F02406090C0F1215181B1E20229C
:109010004FF461531CE04FF4964319E04FF4E143E1
:1090200016E04FF4164313E04FF4614310E04FF4A1
:1090300096330DE04FF4E1330AE04FF4613307E07B
:109040002E4B05E02E4B03E02E4B01E04FF4165360
:109050000093009B06A95B0841F8183D2548694626
:1090600005F052FC25230024012505A88DF81430B5
:1090700007238DF815308DF816408DF8175004F041
:1090800033F81C4840F2FF3105F012FC282122463B
:10909000184805F039FB2A46164840F2277105F0BA
:1090A00033FB2A46134840F2266105F02DFB2A4681
:1090B000104840F2255105F027FB22460D4840F2AA
:1090C000244105F021FB22460A4840F6460105F0FE
:1090D0001BFB2246074840F66A1105F015FB60218C
:1090E0002246044805F010FB2946024805F0FEFA26
:1090F00007B030BD003801400008014090D00300A7
:1091000020A1070040420F00704700BF184B1A789B
:10911000AAB15968174A013159601168164B0131DB
:1091200011601A6812B11A68013A1A60134B1A6872
:1091300012B11A68013A1A6000220D4B00E00122B8
:109140001A700F4B1A683AB11A68013A1A601B6814
:1091500013B90C4B01221A700B4B1A683AB11A68FA
:10916000013A1A601B6813B9084B01221A70704744
:10917000940400205C070020A40C0020A80C002010
:10918000AC0C0020B00C0020A00C0020B10C002082
:10919000014B5868704700BF9404002008B50420B4
:1091A00004F06AFC4FF4FA5004F076FC012004F05D
:1091B00079FC04480321002204F064F8012004F043
:1091C00087FC08BD9AC302000828F8B508D0092812
:1091D0000ED008B100205AE03B4B188880B256E010
:1091E000394B588840F26B1380B2584300134EE05D
:1091F000354B988880B207F0F9FF07F0DBFB0022BF
:10920000324B07F02BFC22A3D3E9002306460F467E
:1092100007F024FC20A3D3E9002307F06DFA1EA376
:10922000D3E9002304460D463046394607F016FCC4
:109230001BA3D3E9002307F03BFD02460B46204663
:10924000294607F035FD07F0CBFE07F0B3FB0022FF
:109250001F4B07F02DFD06F055FE13A3D3E90023A5
:1092600007F0FCFB12A3D3E9002307F045FA0246FE
:109270000B4611A1D1E9000107F01AFD10A3D3E9B3
:10928000002307F037FA07F0ABFE08F0CDF9F8BD80
:109290006666666666660AC06666666666660A40F2
:1092A0009A99999999990140C3F5285C8FA27240C7
:1092B0000000000000FEAA409A999999FD6F2F4185
:1092C000C3F5285C8F1271409C0400200000303FE1
:1092D00000002440F0B593B011AF0124002503260F
:1092E00040483946ADF844408DF846608DF8475007
:1092F00003F08AFD39463C48ADF844608DF846607D
:109300008DF8475003F080FD2046214604F076F9A1
:1093100021464FF4007004F07FF9344803F0BEF9A1
:10932000334B32480193334B01A9029380230693B8
:10933000DB18079303F540730893A3F5787309933B
:1093400003F5FF530A930395049605950B9503F0D7
:1093500015FA2648214603F041FA4FF460232648C7
:109360000CA90E938DF834400C958DF835400F956F
:109370008DF8406002F0C6FF1F48082122463346A0
:1093800003F042F81C4829460222334603F03CF819
:10939000334632461848092103F036F82A46164863
:1093A0004FF4FC6102F0F2FF1348214602F0E4FFA3
:1093B0001148214602F0D6FF0F4802F0F1FF0E4897
:1093C00002F0F4FF0028FAD10B4802F0F3FF0A483C
:1093D00002F0F6FF0028FAD10748012102F0F4FF5D
:1093E00013B0F0BD00080140000C0140080002402D
:1093F0004C2401409C04002000240140AFF3008075
:10940000014B03221A607047A4040020044A054B54
:10941000927A0AB1052200E001221A60704700BF6B
:10942000C00C0020A4040020704700BF014B0022A4
:109430005A607047A404002008B5074B1A6892B21E
:1094400042F008021A601A6892B242F004021A60EE
:10945000FFF7D6FF08BD00BF405C004010B5064CCA
:109460004FF6FB73226802EA03032360FFF7CEFF87
:109470004FF40643236010BD405C0040072818BF2E
:109480001F4B10B51E4C18BF18702378052B33D80E
:10949000DFE803F003060A0E1621FFF7DFFF2BE0DB
:1094A000FFF7DCFF042328E002236370013324E08C
:1094B0006378013BDBB263706378FBB9042218E088
:1094C000104B1A6892B242F010021A600523237002
:1094D000DB18637012E06378013BDBB26370637882
:1094E00063B9084A4FF6EF73116801EA030313608A
:1094F0000622034B1A7001E00623237010BD00BF43
:10950000240D0020405C0040034B9B7A13B1034BB9
:1095100005221A60704700BFC00C0020A404002080
:10952000014B04221A607047A4040020034B1A7AEE
:10953000202A01D100221A72704700BFA404002023
:10954000704700BF212808B508D1124B1B681B7853
:1095500003F07F03212B1AD10F4B0EE0202816D1E8
:109560000C4B0E4A1B681B7810720D4A03F07F03E8
:10957000212B0CBF134600234BB1064A4FF00001CC
:1095800012680020518293619847002000E0022079
:1095900008BD00BF200D0020D9950008A4040020BC
:1095A000F5950008074B1B681B7803F07F03212B00
:1095B00005D1022801D0222801D1002000E002209C
:1095C000704700BF200D002019B9012801D80846B6
:1095D00000E00220704700BF28B9044B4FF008029A
:1095E0001B681A8200E00248704700BF200D00206F
:1095F0004800002028B9044B4FF008021B681A826B
:1096000000E00248704700BF200D00204800002005
:109610000B4B10B5DA6882B11B68052B01D0002214
:109620000BE0002303E00749595CC15401330449AE
:10963000CC68A342F7D30023CB60104610BD00BF17
:10964000A4040020280D0020084BDB68082B01D85B
:1096500000200AE00023064A9A5CC2540133092B19
:10966000F9D1024B0022DA6001207047A4040020E7
:10967000280D002010B5074C0B468AB2C02163604C
:1096800005F066FF0120A18806F070F9012006F0C0
:109690003BF810BDA404002007B5142200238DF868
:1096A000042001A801228DF806308DF807208DF8DE
:1096B000053003F019FD0EBD07B5142200238DF807
:1096C000042001A801228DF806308DF807208DF8BE
:1096D000053003F009FD0EBD08B5064B1B68DB78AD
:1096E000042B01D9002004E0034901EBC30105F07C
:1096F000D7FA08BD200D00205000002008B502490F
:1097000005F0CEFA08BD00BF7000002008B5024980
:1097100005F0C6FA08BD00BF78000020334B10B535
:109720001B686FF03F0200245A72DC729C72204664
:1097300005F062FF20464FF4007105F07BFF102119
:10974000204605F08DFF4021204606F0E3F88021F9
:10975000204606F0CFF8204606F00CF8244B2046B1
:1097600093F8641006F024F9204605F0DBFF012091
:10977000214605F05FFF0120C02106F0BBF8012063
:10978000202105F06DFF0120214605F081FF022018
:109790004FF4C06105F04EFF02204FF4807106F0D7
:1097A000A9F80220214605F073FF0220202105F0D0
:1097B00057FF0320214605F03DFF03204FF4887139
:1097C00006F0A8F80320402106F0F2F803204FF439
:1097D000405105F05DFF2146032005F041FF204682
:1097E00005F06CFA034B01221A6010BD200D002019
:1097F00048000020A404002008B5174B174A196838
:1098000089B2118016491288098801EA020212F40D
:10981000806F05D04FF6FF321A60124BDB6B984712
:109820000E4B1A880E4B1B8803EA020212F4007FCB
:1098300008D009490C4A4FF6FF500860117C0131ED
:10984000C9B21174054A1288134013F4004F01D0B5
:1098500005F0BAFD08BD00BF445C0040B60C002016
:10986000680D002048000020A404002010B503204B
:1098700006F0CEF8064C034602464FF488710548C0
:10988000E36005F07DFE032005F04CFF10BD00BF36
:10989000A4040020280D002008B520B104481021A0
:1098A00003F018FB03E00248102103F015FB08BD8C
:1098B000000C014038B5064D01232B60054B0024F8
:1098C00020461C60FFF7E8FF03232B60204638BDCD
:1098D000405C0040445C004008B5FFF7EBFF08BD6A
:1098E00008B50120FFF7D8FF064B01211960064992
:1098F0004FF4E0520A8005490020186008601A60A1
:1099000008BD00BF405C0040680D0020445C004082
:10991000084B10B51B6800249C72FFF7E1FF064A54
:109920004FF406431460043A1360044A1460044A76
:10993000138010BD200D0020445C0040A4040020D2
:10994000680D0020012008B503F0DCFD4FF4000095
:10995000012103F06FFE08BD07B5FFF7F3FFFFF726
:10996000ABFE05F0D3FC0820012103F055FE1023C7
:109970000322054801A98DF806208DF80730ADF8BF
:10998000043003F041FA0EBD000C0140704700BFE7
:10999000704700BF704700BF704700BF0A4B0B4ABB
:1099A000D978187993F805C041EA0020997940EAFE
:1099B0000C4353EA01610BBF054B054B9B881B8988
:1099C0009BB25360704700BFE8060020600700208C
:1099D000006C0040704700BF704700BF704700BF79
:1099E00008B5FAF7C1FD052805D9FAF7BDFD40F223
:1099F000F933984201D9012200E00022094B5A6054
:109A0000094B1B786BB1074B08495A68084B0A6031
:109A10001AB91A6842F0080202E01A6822F0080235
:109A20001A6008BD600700205A0700204807002080
:109A3000F006002010B5FFF7ABFB074C2368C31AF4
:109A4000B3F5FA7F07D9054BDA6882F40072DA6061
:109A5000FFF79EFB206010BD6C0D0020000C014044
:109A6000024B03EBC003D879704700BFB804002055
:109A7000024B03EBC0035879704700BFB8040020C5
:109A8000024B03EBC0039879704700BFB804002075
:109A9000024B0B2202FB0033187A7047B8040020F7
:109AA000024B0B2202FB0033587A7047B8040020A7
:109AB000024B0B2202FB0033D87A7047B804002017
:109AC000024B0B2202FB0033987A7047B804002047
:109AD000024B0B2202FB0033187B7047B8040020B6
:109AE000024B0B2202FB0033587B7047B804002066
:109AF000024B0B2202FB0033987B7047B804002016
:109B0000024B0B2202FB0033187C7047B804002084
:109B1000024B0B2202FB0033587C7047B804002034
:109B2000024B0B2202FB0033987C7047B8040020E4
:109B3000024B052202FB0033187D7047B804002059
:109B4000024B052202FB0033587D7047B804002009
:109B5000024B052202FB0033987D7047B8040020B9
:109B6000024B052202FB0033D87D7047B804002069
:109B7000024B052202FB0033187E7047B804002018
:109B8000024B032202FB0033187F7047B804002009
:109B9000034B032202FB003393F91D00704700BF03
:109BA000B8040020024B032202FB0033987F704769
:109BB000B8040020024B03EBC00393F82000704769
:109BC000B8040020024B03EBC00393F82100704758
:109BD000B8040020024B03EBC00393F82200704747
:109BE000B8040020024B03EBC00393F82300704736
:109BF000B8040020024B03EBC00393F82400704725
:109C0000B8040020024B03EBC00393F82500704713
:109C1000B8040020024B03EBC00393F82600704702
:109C2000B8040020024B03EBC00393F827007047F1
:109C3000B804002006281AD8DFE800F004070A0D4F
:109C4000101316000A4B9B6A10E0094BDB6A0DE00B
:109C5000074B1B6B0AE0064B5B6B07E0044B9B6BEF
:109C600004E0034BDB6B01E0014BDB7B0B607047D7
:109C7000B804002070B5C0F307410546002201205A
:109C8000FAF7EEFE0A4C0602C5F307210022012076
:109C9000A662FAF7E5FE064301203602E9B2024663
:109CA000A662FAF7DDFE06433609A66270BD00BF64
:109CB000B80400202D4B032202FB003310B51C33E7
:109CC00093F901203F2A01DD3F225A70274B0322DE
:109CD00002FB00331C3393F9012012F13F0FBCBF8C
:109CE0006FF03E025A70214B032202FB00331C33FB
:109CF0009A781F2A01D91F229A701C4B032202FB5B
:109D000000324FF440211964127F012A04BF4FF43E
:109D100050221A64154B03EBC00292F827203AB97F
:109D2000033202FB0032527F196C02F07F020BE01B
:109D3000032101FB003191F81DC002F003020CF079
:109D40007C0C196C4CEA0202084C41EA02221A64AB
:109D5000032303FB0040236C827F42EA030318467F
:109D60002364FFF787FF236CA36310BDB8040020B2
:109D700008B5044B032202FB00339977FFF79AFFE3
:109D800008BD00BFB804002008B5044B032202FB45
:109D900000335977FFF78EFF08BD00BFB8040020DD
:109DA00008B5044B032202FB00331977FFF782FF4B
:109DB00008BD00BFB8040020264B052210B502FBE9
:109DC00000331A7D012A01D901221A75214B05227F
:109DD00002FB003314335A78032A01D903225A7044
:109DE0001C4B052202FB003314339A780F2A01D949
:109DF0000F229A70174B052202FB00331433DA78D6
:109E0000032A01D90322DA70124B052202FB003328
:109E100014331A790F2A01D90F221A710D4C052318
:109E200003FB004000F114021379017D43F4202369
:109E3000507843EAC133917843EA4033D27843EA19
:109E4000012343EA421318462364FFF713FF236CF0
:109E5000636310BDB804002008B5044B052202FB63
:109E600000331976FFF7A8FF08BD00BFB804002033
:109E700008B5044B052202FB0033D975FFF79CFFA0
:109E800008BD00BFB804002008B5044B052202FB42
:109E900000339975FFF790FF08BD00BFB80400209C
:109EA00008B5044B052202FB00335975FFF784FF08
:109EB00008BD00BFB804002008B5044B052202FB12
:109EC00000331975FFF778FF08BD00BFB804002004
:109ED000514B0B2210B502FB00331A7A032A01D929
:109EE00003221A724C4B0B2202FB003308339A7880
:109EF000032A01D903229A70474B0B2202FB00333D
:109F000008331A790F2A01D90F221A71424B0B22FA
:109F100002FB003308335A79072A01D907225A7104
:109F20003D4B0B2202FB003308339A790F2A01D9EB
:109F30000F229A71384B0B2202FB003310335A78F0
:109F40000F2A01D90F225A70334B0B2202FB003328
:109F500010339A780F2A01D90F229A702E4B0B22B8
:109F600002FB0032117AC90341F400241C64527AC6
:109F700012B141F404211964274B0B2101FB00317C
:109F8000C97A19B1196C41F400511964224B8AB98C
:109F90000B3202FB0032083292F804C091784FEA8B
:109FA000CC1C1C6C4CEAC12C51794CEA040242EAEC
:109FB00001121DE00B2202FB0032127C1AB11A6C56
:109FC00042F480521A64144B0B2101FB0031103112
:109FD00091F801E01A6C897842EACE1201F0070C80
:109FE00042EA0C1211F0080F1A6402D042F4006227
:109FF0001A64094B0B2202FB00300830C27922B9E7
:10A0000081791A6C41EA02021A64034C206CFFF752
:10A0100031FE236C236310BDB804002008B528B9B5
:10A02000034BD97B11B1D873FFF752FF08BD00BFB6
:10A03000B804002008B530B9034BDA7B1AB90132F5
:10A04000DA73FFF745FF08BDB804002008B5044BDC
:10A050000B2202FB00339974FFF73AFF08BD00BFE3
:10A06000B804002008B5044B0B2202FB00335974DE
:10A07000FFF72EFF08BD00BFB804002008B5044B51
:10A080000B2202FB00331974FFF722FF08BD00BF4B
:10A09000B804002008B5044B0B2202FB003399736F
:10A0A000FFF716FF08BD00BFB804002008B5044B39
:10A0B0000B2202FB00335973FFF70AFF08BD00BFF4
:10A0C000B804002008B5044B0B2202FB00331973BF
:10A0D000FFF7FEFE08BD00BFB804002008B5044B22
:10A0E0000B2202FB00339972FFF7F2FE08BD00BF9E
:10A0F000B804002008B5044B0B2202FB0033D972D0
:10A10000FFF7E6FE08BD00BFB804002008B5044B09
:10A110000B2202FB00335972FFF7DAFE08BD00BFC5
:10A12000B804002008B5044B0B2202FB003319725F
:10A13000FFF7CEFE08BD00BFB804002010B5254BC8
:10A140004FF460221A6403EBC00292F8272012B188
:10A150004FF470221A641F4B03EBC00292F82110D7
:10A1600092F820C01C6C090341EA8C312143196428
:10A1700092F82220012A04BF41F480611964154B32
:10A1800003EBC00191F823C01A6C42EA0C221A6456
:10A1900091F82410012904BF42F080021A640D4B8B
:10A1A00003EBC00292F82520012A03D11A6C42F079
:10A1B00040021A64074C04EBC00090F82620236C80
:10A1C00043EA021318462364FFF754FD236CE3634C
:10A1D00010BD00BFB804002008B5044B03EBC0035A
:10A1E00083F82610FFF7AAFF08BD00BFB8040020BF
:10A1F00070B50F4B064603EBC00393F82650032DB2
:10A2000002D00321FFF7E8FF3046FFF797FF084B26
:10A210009C6A14F4002F1CBF6FEA04346FEA1434F4
:10A22000032D03D030462946FFF7D6FF204670BDE8
:10A23000B804002008B5044B03EBC00383F82510D5
:10A24000FFF77CFF08BD00BFB804002008B5044B31
:10A2500003EBC00383F82410FFF770FF08BD00BFB5
:10A26000B804002008B5044B03EBC00383F82310A7
:10A27000FFF764FF08BD00BFB804002008B5044B19
:10A2800003EBC00383F82210FFF758FF08BD00BF9F
:10A29000B804002008B5044B03EBC00383F8211079
:10A2A000FFF74CFF08BD00BFB804002008B5044B01
:10A2B00003EBC00383F82010FFF740FF08BD00BF89
:10A2C000B8040020064B10B503EBC003044683F826
:10A2D0002710FFF733FF2046FFF7ECFC10BD00BF4F
:10A2E000B804002010B5144B00221A6403EBC0021E
:10A2F000527912B14FF400721A640F4B03EBC00293
:10A3000092791AB11A6C42F480721A640A4B03EB08
:10A31000C003DA790F2A01D90F22DA71064C04EB57
:10A32000C000C279236C42EA030318462364FFF796
:10A33000A1FC236CE36210BDB804002070B5084D89
:10A340009DF810E09DF8146005EBC0042671627062
:10A35000A37084F803E005F83010FFF7C3FF70BD69
:10A36000B804002008B5034B03EBC0039971FFF755
:10A37000B9FF08BDB804002008B5054B03EBC003C6
:10A38000597109B10422DA71FFF7ACFF08BD00BFB3
:10A39000B804002008B5054B042903EBC003D971AC
:10A3A00001D000225A71FFF79DFF08BDB8040020BC
:10A3B0002DE9F047344D0446401990F844000E460C
:10A3C00017469846DDF82090DDF824A004281FD811
:10A3D000DFE800F003090F151B002046FFF778FDAA
:10A3E0006519012316E02046FFF7A8FE6519022330
:10A3F00010E02046FFF7E0FC651903230AE0204641
:10A40000FFF758FC6519042304E02046FFF76AFFB4
:10A410006519002385F844301B4B03EBC40494F802
:10A420002620012A0DD002D3022A23D111E016B131
:10A430009B6A9B0C3370EFB1134B9B6A9B0A3B707A
:10A4400018E0B8F1000F15D09B6A9B0AC8F80030DD
:10A4500010E0B8F1000F04D09B6ADB0B5B01C8F879
:10A460000030B9F1000F05D0074B9B6AC3F384237A
:10A4700089F80030BAF1000F03D0034B9B6A8AF8C9
:10A480000030BDE8F08700BFB8040020214B10B5B4
:10A49000032200244FF0050C02214FF0010E83F837
:10A4A00025E0197383F80EC09A745C7483F81CE07D
:10A4B00083F81DC083F81EC083F8202083F8212074
:10A4C00083F8224083F8234083F8244083F8261041
:10A4D00083F827401C755C759C75DC751C765C7177
:10A4E0009C71DC7119725C72DC729C725A73DC7341
:10A4F0001C742046FFF760FC2046FFF7DBFB20467C
:10A50000FFF71CFE2046FFF7EDFE2046FFF7E0FCBC
:10A5100010BD00BFB804002008B5044A0023917A9A
:10A52000034A18461370FAF7D1F908BDF80B00205A
:10A53000600C00202DE9FF417F4B1A7822B90132CF
:10A540001A706FF000425A607B4B1C7A5CB9E0B223
:10A55000F9F7D4FF784B03F10C0210550134082CA5
:10A56000F5D101221A7227240025E8B2F9F7C6FFB7
:10A57000724A535D834219D0714B291D53F8213023
:10A580005055022B05D0032B0AD0012B0ED168B1F8
:10A5900006E058B96B4A115D012907D1135505E052
:10A5A000684B1A5D012A01D101321A550135013477
:10A5B000082DDAD1644EF36993B1644C25787DB9E6
:10A5C000FEF7E6FD624AF3691268821A002AB8BFF4
:10A5D00052429A4204D9284601F03AFA01232370E4
:10A5E000594E336A93B15B4C25787DB9FEF7D0FDA7
:10A5F000594A336A1268821A002AB8BF52429A42F4
:10A6000004D9284601F024FA012323704A4D534C03
:10A610002A7D930004EBC3010E7B002E00F02881FD
:10A620004F48504F504E0021C318BF18B61810465F
:10A630000A4600970196FFF7BBFE2B7D04EB4314FF
:10A64000227B013A042A00F20281DFE812F00500C1
:10A650004E00D3004E00D300444A374D926812F0AA
:10A66000200F1BD05D192A7E022A04D1404AD25CF9
:10A67000002A00F0EC80394A2F4C02EB43121846B6
:10A68000517AFAF723F9207DFFF7C8FC237D384A79
:10A690000021E418D15402232376D8E05D192A7EE4
:10A6A000012A04D1324AD25C002A00F0D0802B4C1F
:10A6B000184604EB4313997AFAF708F91E4B187DF4
:10A6C00004EB4014A37A13B9FFF7B4FC04E0284B61
:10A6D0001B5C0BB1FFF7A2FC174A2549137D002034
:10A6E000D218C85401231376B1E01F4A124DD25636
:10A6F000002A3FDB5D192A7E022A02D11C4AD25C65
:10A700008AB1164A0C4C02EB43121846517AFAF7FA
:10A71000DDF8207DFFF782FC237D154A0021E41837
:10A72000D15402232376044C257DFEF731FD04EB42
:10A730008504606056E000BF000500200C05002085
:10A74000200C0020700C0020080000205D0C002070
:10A75000580C0020750B0020500C0020F80B002036
:10A760009C0B0020800B0020F00B0020000C01400F
:10A770005C0C00205B191B7E012B11D0FEF708FD3D
:10A780002B7D8A4A05EB830502EB43139B8B0A2240
:10A7900053436A68821A002AB8BF52429A4204DCC4
:10A7A000834B844A1B7DD35CE3B1814D7F4C287D74
:10A7B00004EB4013997AFAF789F8287D04EB4014EA
:10A7C000A37A13B9FFF736FC04E07A4B1B5C0BB19C
:10A7D000FFF724FC764A7749137D0020D218C8542D
:10A7E00001231376724B1A7D704B03EB42131B7BD4
:10A7F000042B20E06E4A9A18127E022A02D16D4A7A
:10A80000D25C8AB1694A6A4C02EB43121846517A0B
:10A81000FAF75CF8207DFFF701FC237D654A0021F3
:10A82000E418D15402232376614B1A7D5F4B03EB6E
:10A8300042131B7B052B0AD15F4B9A6812F0200F45
:10A8400015BF4FF480624FF480625A611A61FEF7BF
:10A850009FFC574CE369C31A002BB8BF5B420A2B1D
:10A8600040F31383F9F71EFFFEF792FCE0610CE35F
:10A87000F9F718FFFEF78CFCEB69C31A002BB8BF81
:10A880005B420A2B40F30183297D3046490141F0A8
:10A890000A0101F0EA0100F09DFF0446287D00282E
:10A8A00040F00B8201F0F8F82B7D0C20584343490F
:10A8B0004218157A0DB1455800E05568404AD25CFF
:10A8C000032A00F2DA80DFE802F0027F1C4B002C42
:10A8D00000F0D380354A364D02EB4311C97F384E24
:10A8E00029B11846F9F7F2FF2B7D032207E002EBAE
:10A8F00043121846517AF9F7E9FF2B7D0222F254F0
:10A90000BBE04CB95B0143F0080101F0E8012046CF
:10A9100000F060FF002861D0254E244B307D03EB12
:10A920004013D97F002900F0A180002D84EAE47251
:10A93000B8BF6D42A2EBE472AA4202D0002C40F0F4
:10A940008F80204B53F830108A4280F08F8003EBC9
:10A95000C0031979F9F7BAFF154B01211B7D83E07C
:10A96000002D84EAE471B8BF6D42A1EBE471A94205
:10A9700001D0002C7AD1134A0D4D52F83300104EFD
:10A98000814208D202EBC30218461179F9F79EFF03
:10A990002B7D012208E0054A184602EB4313597A41
:10A9A000F9F794FF2B7D0222F2545FE0F80B0020B0
:10A9B000000500205C0C0020000C0140A40B0020CE
:10A9C000600C0020840B002044BB5B0143F00801B5
:10A9D00001F0E801204600F0FDFEF8B9FEF7D8FBD3
:10A9E0007D4D7E4A2B7D4FF00A0E02EB4311B1F8EC
:10A9F0001CC099004E1976680EFB0CFC861B002EBD
:10AA0000B8BF7642664538DD02EBC1021846917A3E
:10AA1000F9F75CFF2B7D724AD4542EE06E4E6F4ADC
:10AA2000337D02EB4312D17F01B3002D84EAE4723F
:10AA3000B8BF6D42A2EBE472AA4200D07CB969496A
:10AA400051F833108A4211D3644A184602EB43137B
:10AA5000597AF9F73BFF604B02211B7D04E0184651
:10AA6000F9F734FF337D03215D4AD1545A4D2E7DD1
:10AA7000FEF78EFB05EB86056860574D5A4F2B7D20
:10AA80005A4E1846F618FF18594B002103EB800365
:10AA90000A4601960097514EFFF78AFC287D06EB87
:10AAA00040139B6943B3F9F799FC28B3287D84EAE6
:10AAB000E47206EB40139B69A2EBE4729A421BD945
:10AAC00000F0C6FF2A7D4B4906EB42139B7F012015
:10AAD000885443B1B27F9A4205D1013800F0B8FFE3
:10AAE000002000F0F3F93C4B434A1B7D0F33D15C4F
:10AAF000012901D10131D154374F384E3B7D06EB4E
:10AB000043125269002A7BD03C4AD55C002D77D194
:10AB1000002C76D05B0143F0020101F0E2012846EF
:10AB200000F01EFE8046387DF9F7B4FE397DC0EB9B
:10AB3000080806EB41135B69B8F1000F83EAE37282
:10AB4000B8BFC8F10008A2EBE372904562DD002BAC
:10AB50000EDD084600F07CFF3B7D06EB43139B7F38
:10AB60003BB3B27F9A4224D1284600F071FF1DE02A
:10AB70002846022200F0CEFD397D2846490141F0E9
:10AB8000080101F0E80100F045FF3B7D06EB4313AF
:10AB90009B7F73B1B27F9A420BD12946284602228D
:10ABA00000F0B8FD2846082100F034FF284600F0E8
:10ABB0008DF9094B104A1B7D1533D15C012901D158
:10ABC0000131D154044B0D4A1B7D01211846D1544B
:10ABD00000F07CF91EE000BF00050020F80B00200B
:10ABE000600C0020840B0020800B0020F00B002064
:10ABF0009C0B0020EC0B0020700C0020900B002020
:10AC000044B95B0143F0080101F0E801002000F0C5
:10AC1000E1FD20B19E4D9F4B2E7D9B5D43B39C4B30
:10AC20009D4A1B7D02EB4312D28912B9994AD35C2B
:10AC30001BB3FEF7ADFA964D97492B7D4FF00A0CEA
:10AC40009A0001EBC201C9895219126A0CFB01F189
:10AC5000821A002AB8BF52428A420EDD8F4EF25C41
:10AC60005AB91846FFF7E6F92B7D0122F25404E0A9
:10AC7000FEF78EFA05EB86052862854E884D307DFD
:10AC8000002C55F83030B8BF64429C420AD2FEF71F
:10AC90006FFF337D05EBC3056A7982420DD11846FB
:10ACA000002108E0FEF764FF337D05EBC3056979F9
:10ACB000884202D01846FFF7CFF8002000F066FC6B
:10ACC000734B10F0010F93F8242002F0F80283F880
:10ACD00024201CBF42F0010283F8242010F0040F4E
:10ACE00006D06B4B93F8242042F0020283F8242014
:10ACF00010F0100F06D0664B93F8242042F00402A7
:10AD000083F82420674B1A7812F0010F1FD0604A95
:10AD100092F8242012F0010F19D0634C94F800C06F
:10AD20001CF0010F13D16149614A91F800E04CF029
:10AD3000010C4EF0010E81F800E012785D4984F8B4
:10AD400000C04FF0010C81F800C002B91A70504BDE
:10AD500093F8242012F0010F0AD093F8253013F055
:10AD6000010F05D1544BDA78012A01D10132DA7092
:10AD7000474B93F8242012F0020F0AD093F82530A5
:10AD800013F0020F05D14C4B1A79012A01D101327F
:10AD90001A713F4B93F8242012F0040F0AD093F855
:10ADA000253013F0040F05D1434B5A79012A01D104
:10ADB00001325A71364C0322237D04A9B3FBF2F20F
:10ADC0008A188DF80C0012F9042C94F82410002A2B
:10ADD00084F825104ADA5B0143F01601002001F0E7
:10ADE000F60102AA00F00EFD9DF80A3013F0400FA4
:10ADF00008D0227D304952001B32885C012801D1E5
:10AE00000130885413F0800F0AD021492A4A097D65
:10AE10000E3112F81100012802D1013002F81100A0
:10AE200013F0100F09D01A4A2349127D52001B3229
:10AE3000885C012801D10130885413F0200F0AD01A
:10AE4000134A1D4B127D0E3213F81210012902D144
:10AE5000013103F812100E4B0020197D02AA49019E
:10AE600041F0160101F0F60100F068FE084C207D6B
:10AE700000F03AF8237D0133DBB223750BB10023D8
:10AE80002375FEF785F9024BD861BDE8FF8100BF4D
:10AE900000050020680C0020F80B00206C0C00203E
:10AEA000840B0020980B00207D0B0020910B0020CC
:10AEB0007C0B00209F0C0020700C0020024B1A5CC1
:10AEC0000AB901321A54704728050020024B1A5C57
:10AED0000AB10F221A54704728050020014B185C54
:10AEE000704700BF280500202DE9F3474601F5B261
:10AEF000044645F07C01002001AA00F083FCB74A1B
:10AF0000610002EB4413187A06EB020710F0400FC1
:10AF10009DF8063012D04FF001084FF0020C08FAED
:10AF200001F80CFA01FCB1587E680CEA030208EA49
:10AF30000307C1F10009C6F1000A0FE04FF0010C50
:10AF40004FF002080CFA01FC08FA01F156F80290E1
:10AF5000D7F804A00CEA030201EA030710F0800FFF
:10AF600000F03F0606D09E4B9B6883F02008C8F394
:10AF7000401803E09A4B9B68C3F34018731E072BDD
:10AF800000F2D182DFE813F0080008000800080092
:10AF90006E016E016E016E01924B1B5D013B0E2B2B
:10AFA00000F2C182DFE813F00F003D0053006200A1
:10AFB0007A0082008E00A000D10014012401BF029B
:10AFC00043014E01A60201AA45F014010020854F5D
:10AFD00000F018FC9DF8053045F0060507EB8408E5
:10AFE000C8F804302946002000F0F4FB0222C8F81B
:10AFF00008002146002000F08DFB023E002029467B
:10B0000040F2FF7200F0F2FCF6B20020032221466B
:10B0100000F05AFB012E01D8022300E004233B5527
:10B0200081E2704E002006EB84035A68214602F04C
:10B030000402824214BF0522012200F045FB45F0C4
:10B0400008014A46002000F0D1FC032324E0002A36
:10B0500000F0698245F00201002000F081FB614BA5
:10B0600004221A55604B43F824005CE25D4E002038
:10B0700006EB84035A68214602F00402824214BFA0
:10B080000622022200F020FB45F00801C9F100026F
:10B09000002000F0ABFC0523335544E2002F00F004
:10B0A0004282204600F0D4FC06222FE200202146F6
:10B0B000032200F009FB45F008015246002000F091
:10B0C00095FC68E1002F40F02E8245F008053A46D5
:10B0D0003846294600F08AFCCAF100023846294663
:10B0E00000F084FC082211E2002F00F01C8245F0E1
:10B0F0000201002000F034FB06460020024645F025
:10B10000080100F073FC384B002053F824702146EE
:10B11000BF1B43F82470032200F0D6FA8AEAEA72D1
:10B1200045F00601A2EBEA72002000F05FFC61012D
:10B1300001F0E0013246002000F0C4FB002002468E
:10B14000214600F0E7FA0922E0E1002000F01EFAB3
:10B15000630050FA03F313F0010F00F0E48145F0AF
:10B1600002073946002000F0FBFA204B45F00805A5
:10B1700043F8240000200246294600F037FC002056
:10B180000222214600F0C6FA00200246394600F0AD
:10B1900099FB00206101024601F0E001033E00F04E
:10B1A00091FBF6B200212046F9F74AFB012E0D4E25
:10B1B0000CD800202146022200F0ACFA2946CAF140
:10B1C0000002002000F012FC0A2365E70E2363E76B
:10B1D000002F00F0A8810B2298E100BFF80B00209F
:10B1E000000C014028050020780B00201C0C0020DA
:10B1F000002F40F0988145F00201384600F0B0FA87
:10B2000045F0080106463A46384600F0EFFB61017A
:10B21000022296FBF2F201F0E001384600F052FB08
:10B220003A463846214600F075FA0D226EE10020BC
:10B2300000F0ACF9630050FA03F313F0010F00F0D3
:10B24000728162E1A84E45F0060106EB84050020FC
:10B25000AA6800F0CBFB2A790020214600F034FADE
:10B26000002319E7A04B1B5D013B0E2B00F25B8115
:10B27000DFE813F00F003400520062008100590132
:10B28000930059015901CC00DC00AD0008014F01C9
:10B29000400145F0140101AA0020934F00F0B2FADA
:10B2A0009DF805C007EB840300200222C3F804C008
:10B2B000214600F02FFA002045F0060140F2FF720F
:10B2C00000F094FB00200322214600F0FDF9062E39
:10B2D00002D0082E7FF4A2AE022217E1062E0CD176
:10B2E000814B002003EB84035A68214602F00402DC
:10B2F000824214BF0522012204E0082E04D100205E
:10B300002146032200F0E0F94A4645F008010020FA
:10B3100000F06CFB0322F9E0731FDBB2012B05D8B0
:10B3200022B1062E704E30D10423B5E6B8F1000FDD
:10B3300000F0F9800C22E9E0052E0CD16A4B0020C8
:10B3400003EB84035A68214602F00402824214BFD0
:10B350000622022204E0072E04D100202146032207
:10B3600000F0B2F9C9F1000245F00801002000F038
:10B370003DFB0522CAE0731FDBB2012B07D837B1B2
:10B38000052E594E01D1022386E60F2384E6B8F13B
:10B39000000F00F0C8800722B8E0B8F1000F40F0BD
:10B3A000C280073EF6B2012E0DD94F4B404603EB4B
:10B3B00084035A68214602F00402002A14BF0522C1
:10B3C000012200F081F945F00801524619E0B8F178
:10B3D000000F40F0A880073EF6B2012E0DD9424B77
:10B3E000404603EB84035A68214602F00402002A17
:10B3F00014BF0622022200F067F945F00801CAF1E5
:10B400000002002000F0F2FA0A227FE0B8F1000FFB
:10B4100000F0898045F00201002000F0A1F9324BD4
:10B420000B2103EB84021955D0607CE0B8F1000FCA
:10B4300079D145F00201404600F092F92B4BA7006C
:10B44000294E03EBC7038AEAEA72814645F00601FA
:10B45000A2EBEA72404683F80D80BF1900F032FA81
:10B46000FB6861019944022399FBF3F201F0E001CA
:10B47000404600F027FA40462146424600F04AF98D
:10B480000D2309E6002000F081F8630050FA03F371
:10B4900013F0010F47D0144B0E2245F002061A5547
:10B4A0003146002000F05CF9114B45F0080143F8EB
:10B4B00024000020024600F099FA214600200222D2
:10B4C00000F028F900203146024600F0FBF9002088
:10B4D0006101024601F0E00100F0F4F9204600218C
:10B4E000F9F7AEF91FE000BF28050020F80B002097
:10B4F0001C0C002000202146022200F00BF9002045
:10B5000045F00801024600F071FA0E22074B1A5569
:10B5100009E0064D002005EB84031A79214600F06E
:10B52000D3F800232B55BDE8FC8700BF2805002079
:10B53000154B10B503EB0012926891420EDD8A1A8A
:10B54000C2F18074A2424FEA001C03DC63445C68D1
:10B5500012190EE063445A68141B0FE00FDA521AF6
:10B56000C2F18074A2424FEA001C04DC63445C68B0
:10B57000A21A5A6003E063445A68A4185C60024B44
:10B5800003EB0010816010BD700D0020012108B593
:10B5900002200A46F9F764FA08BD00BFF8B513782F
:10B5A000144613F0600F06460D4627D1414A127B20
:10B5B00022BB13F0010F21D15F2B1FD83E4A127816
:10B5C000E2B913F09F0301D0082B17D13B4F387815
:10B5D00060B9384BD97F19B1F9F778F9032304E042
:10B5E0000846597AF9F772F902233B70344F3B78D9
:10B5F00023B10020FEF712FD00233B7000222178CA
:10B600000220F9F72DFA2870002261780220F9F75C
:10B6100027FA68700022A1780220F9F721FAA870B1
:10B6200001220220E178F9F71BFAE870237813F081
:10B63000010F3ED15F2B3CD803F01E02082A04D034
:10B64000142A2CD0062A34D11BE0242171435B0933
:10B650000C2000FB0313A57894F803C0194A4CEAA8
:10B6600005259D50A37813F0080F22D0267876097F
:10B6700000FB0616B3586FEA03536FEA1353B35037
:10B6800017E0242256435B090C22A17802FB0363D6
:10B69000E27842EA01220B495B185A6009E0242251
:10B6A00056435B090C2202FB03630649E2785B18F0
:10B6B0001A72F8BDF80B0020680C0020600C002006
:10B6C0006C0C0020A40B00202DE9F3414901CEB2FF
:10B6D00001AC46F015031746694622468DF8043042
:10B6E0008046FFF75BFF9DF801C09DF8033046F0F0
:10B6F00014064046694622466D468DF804608DF872
:10B7000005C08DF806708DF80730FFF747FFBDE8DC
:10B71000FC8100BF2DE9F3414901CEB201AC46F0F6
:10B7200015031746694622468DF804308046FFF718
:10B7300035FF9DF801C09DF8023046F014064046E2
:10B74000694622466D468DF804608DF805C08DF877
:10B7500006308DF80770FFF721FFBDE8FC8100BFC0
:10B7600037B541F001030C466A4601A98DF8003057
:10B770000546FFF713FF9DF806009DF8052000021F
:10B780009DF8073040EA0240184310F4000F18BF3C
:10B7900040F07F405F2C1AD8C4F3411314F01E040C
:10B7A00002D0022C13D106E0032202FB0535084A21
:10B7B0002D01A8580BE0032202FB053520F07F4144
:10B7C000E8B2FFF7B5FE024B03EB051568683EBD16
:10B7D000700D002007B541F001036A4601A98DF8FC
:10B7E0000030FFF7DBFE9DF806009DF8073043EAC6
:10B7F000002010F4006F1CBF6FEA00506FEA105079
:10B800000EBD00BF13B541F00103144601A96A46FD
:10B810008DF80030FFF7C2FE9DF805109DF8063048
:10B820009DF807202170A27063709DF804001CBD74
:10B8300007B5410141F0160101F0F601002001AA0F
:10B84000FFF7E0FF9DF80530D80913F0200F18BF6F
:10B8500040F002000EBD00BF07B5410141F01601E6
:10B8600001F0F601002001AAFFF7CCFF9DF805309A
:10B87000C3F3801013F0100F18BF40F002000EBD8C
:10B8800037B50C4641EA401101AA0546C9B200206D
:10B89000FFF7B8FFB4235D436408032305F5807503
:10B8A00003FB04549DF804102046FCF797FF601C2E
:10B8B0009DF80510FCF792FFA01C9DF80610FCF700
:10B8C0008DFF3EBD5F292DE9F3410D460646144626
:10B8D00062D8C1F3411811F01E0102D002295BD1D8
:10B8E0001EE0032202FB0088344A4FEA0810831846
:10B8F0005B688450E01A0028B8BF4042B0F5000FE2
:10B900000ADB9C42CCBF2E4C2E4C2C4A1C1902EB5D
:10B910000812012313733FE002EB081211733BE09E
:10B92000032707FB0087254B3801C1587A00C4EB79
:10B93000010C0132BCF1000FB8BFCCF1000C00EBE0
:10B94000030EBCF5000F24F07F40CEF8044043F80E
:10B9500032001DDBA142CCBF194B1A4B4FEA4818ED
:10B96000E3184FEA234E4FEA232C3046694601AADA
:10B970008DF807308DF804808DF805E08DF806C04D
:10B98000FFF70CFE0D4B03EB071701233B7303E09E
:10B9900003EBC20300221A714FEA244C23123046F3
:10B9A000694601AA8DF804508DF805C08DF806305F
:10B9B0008DF80740FFF7F2FDBDE8FC81700D002017
:10B9C000FFFF7F00010080FF38B50D466821044667
:10B9D000FFF7C6FE15B140F0010201E020F00102C0
:10B9E00020466821FFF76EFF38BD00BF07B513463C
:10B9F0004FEA222C8DF804104FF0000E694601AA80
:10BA00008DF805E08DF806C08DF80730FFF7C6FD0C
:10BA10000EBD00BF07B50B4611F01E01024601D056
:10BA2000022905D1104619460022FFF74BFF0DE011
:10BA30004FF0000C694601AA8DF804308DF807C05C
:10BA40008DF805C08DF806C0FFF7A8FD0EBD00BF3C
:10BA500010B5C4B22146640100200222E4B2FFF70F
:10BA600059FE002044F00801FFF7D4FF44F00A011A
:10BA70000020FFF7CFFF10BD07B59DF810C08DF86F
:10BA800004108DF80520694601AA8DF806308DF85E
:10BA900007C0FFF783FD0EBD30B5430185B00446F6
:10BAA00043F00303002003A902AA8DF80830FFF732
:10BAB00075FD9DF80E109DF80D209DF80F300902C0
:10BAC00041EA024119432046FFF732FD174B03EBD1
:10BAD000041108310A7932B3154A0C2000FB042204
:10BAE000107A00BB2201D518D2586B68C3EB020C48
:10BAF000BCF1000FB8BFCCF1000CBCF5000F05DBAA
:10BB00009A42CCBF0B4A0C4A9A1800E008716101B6
:10BB1000C2F30723D4B201F0E0010020C2F30742D0
:10BB20000094FFF7A9FF05B030BD00BF700D0020E5
:10BB3000A40B0020FFFF7F00010080FF07B5937872
:10BB400092F800E092F801C08DF8041001AA69464D
:10BB50008DF805E08DF806C08DF80730FFF71EFD63
:10BB60000EBD00BF37B5440144F01604E4B20D46E3
:10BB700001AA21460020FFF745FE9DF8053015F08B
:10BB8000010F1ABF6FEA43636FEA536303F07F0349
:10BB90008DF805309DF8053015F0020F14BF43F005
:10BBA000200323F020038DF805300023184621469A
:10BBB00001AA8DF80630FFF7C1FF3EBD37B544013D
:10BBC00044F01604E4B20D4601AA21460020FFF716
:10BBD00019FE9DF8053015F0010F14BF43F0400326
:10BBE00023F040038DF805309DF8053015F0020F65
:10BBF00014BF43F0100323F010038DF80530002329
:10BC00001846214601AA8DF80630FFF797FF3EBD82
:10BC100073B5B42545434B08032205F5807502FB37
:10BC20000355044628460E46FCF742FD8DF80400F5
:10BC3000681CFCF73DFD8DF80500A81CFCF738FDDD
:10BC400046EA44148DF80600E1B2002001AAFFF78D
:10BC500075FF7CBD2DE9F74F4001C7B24C050020B0
:10BC600047F0180101AAFFF7CDFD9DF80560640DAE
:10BC700006F00F053609B5420EDB204604F078FECB
:10BC8000AD1B80460120A840894604F081FE0022B9
:10BC9000334B04F0E3FE0FE0204604F069FE751B11
:10BCA00080460120A840894604F072FE02460B46F9
:10BCB00000202B4904F0FCFF02460B464046494653
:10BCC00004F0F6FF05F08CF904F074FE22A3D3E92A
:10BCD000002304F0C3FE05F083F904F06BFE00229C
:10BCE000204B04F0BBFE4FF0FF36B04600258246E5
:10BCF0008B460120A84004F04BFE02460B465046FE
:10BD0000594604F0ABFE05F043F9A0F180027F2A0A
:10BD100098BF2E46034605F1010588BF43460E2D08
:10BD200001D09846E5E7002547F0120101AA284610
:10BD30008DF805308DF806608DF80450FFF7FEFE93
:10BD4000284647F00C012246FFF750FE2846BDE882
:10BD5000FE8F00BFAFF3008004560E2DB29DEF3F63
:10BD6000000060400000204013B5154B587E10F0D5
:10BD7000010003D000206821212201E06821202257
:10BD80000024FFF79FFD20467E21202223460094B9
:10BD9000FFF772FEE1B200200134FFF739FF1D2CDE
:10BDA000F8D10C210020FFF7DBFC01460020FFF753
:10BDB00051FF0020162143F2FF12FFF717FE1CBDB2
:10BDC00008000020AFF30080084B1868034605E028
:10BDD0002C2A02D100221A7003E001331A78002ABB
:10BDE000F6D1024A01331360704700BF38050020C6
:10BDF00010B50E4B02461B78ABB10D4B1C7994B1BC
:10BE00009C68601CE4180D2A2273986002D03F28B9
:10BE100000D851B9064C014604F10C00FDF72AFC8C
:10BE20000023A36001E0FCF71DFF10BD740B002090
:10BE30003805002030B50121044687B02020FFF7E7
:10BE4000D7FF002C04DA2D200121FFF7D1FF644237
:10BE500000230A2194FBF1F201FB124101AD3031C4
:10BE6000E954591C141E01DD0B46F2E7ED181C467F
:10BE70000121013C15F80109FFF7BAFFB4F1FF3FBA
:10BE8000F6D107B030BD00BF38B50C4D0446A878D8
:10BE900001214030C0B2FFF7ABFF6878012140308C
:10BEA000C0B2FFF7A5FF2078FFF7C4FF6068FFF777
:10BEB000C1FF0D200121FFF79BFF38BD08000020C6
:10BEC00070B5124B06461B78EBB1FCF749FE104CDF
:10BED000054618B100232371012016E0E36C226DA2
:10BEE000934208D21A1992F854200133012032707B
:10BEF000E364207109E004F15400FDF789FBE56477
:10BF00002065284601E0FCF72BFE70BD740B002075
:10BF1000380500202DE9F34104460DF10700FFF735
:10BF2000CFFF002800F0CB808B4B8C4A93F8941005
:10BF300019BB51789DF80700403188420DD1D3F8E4
:10BF40009810002940F0BB801179012231F00101E5
:10BF500083F8942040F0B380AFE00D2801D01B2877
:10BF600002D100227C4B05E0D3F898207E2A00F213
:10BF7000A6800132C3F89820A1E0117931F00101C7
:10BF800003D19DF80700FFF733FF9DF807301F2B03
:10BF90000BD9714AD2F898107E297FD8481C89188D
:10BFA00081F89C30C2F8980078E0082B08D16A4BE1
:10BFB000D3F89820002A71D0013AC3F898206DE098
:10BFC0000D2B6BD1644BD3F89830002B66D0634BAC
:10BFD0001A79112A15D1587801214030C0B2FFF7E3
:10BFE00007FF002503E0585DFFF702FF01355A4BBC
:10BFF0000121D3F898209C339542F4D30D20FFF70C
:10C00000F7FE554A00231568D2F8987019461A466B
:10C0100033E001290FD002D302292DD122E04E4E68
:10C0200006F19C00805C202826D09E1986F81C0111
:10C030000133012120E0484800F19C0C1CF802C0AB
:10C04000BCF1200F0AD1012B04D91818002180F867
:10C050001C110133424D0221ED180DE0181880F833
:10C060001CC108E03C4E06F19C00805C202803D0F7
:10C070009E1986F81C0101330132BA42C9D3364AEF
:10C080000021981880F81C110120C2F89810156042
:10C0900082F8A001C2F89C3182F894109DF8073014
:10C0A0001B2B0CD12D4A2C4B12790021012A83F82D
:10C0B0009410C3F8981002D10D20FFF799FE264B7B
:10C0C00093F8A001002878D00022164683F8A0211A
:10C0D0001546DFF8A880072707FB05872048394663
:10C0E000013503F023FE30B9BE797B7916F0010FDC
:10C0F000237049D007E018F806300736002B5ED0D1
:10C10000FF2DE6D15BE0FFF75FFE23780546042BA9
:10C110000CD1144903F00AFE0346D8B1284612494F
:10C1200003F004FE70B1284610490FE00D2B28D112
:10C130000F4903F0FBFD034660B128460D4903F0AB
:10C14000F5FD08B9012305E00B49284603F0EEFD93
:10C15000B0B90223637017E0380500200800002002
:10C1600054060020612001086520010869200108AB
:10C170006F200108752001087A200108601E01085F
:10C18000284603F0CDFD607016F0020F04D0FFF7D3
:10C190001BFE03F0C5FDA07016F0040F0CD0FFF7D6
:10C1A00013FE03F0BDFD010EC0F30722C0F30743E9
:10C1B000A17122716371E0700120BDE8FC81002350
:10C1C0002370F9E7704700BFFEE700BFFEE700BF3E
:10C1D000FEE700BFFEE700BF704700BF704700BF2B
:10C1E000704700BF704700BF704700BF704700BF77
:10C1F000704700BF704700BF704700BF704700BF67
:10C20000704700BF704700BF704700BF704700BF56
:10C21000704700BF704700BF704700BF704700BF46
:10C22000704700BF704700BF704700BF704700BF36
:10C2300008B5024B1B68984708BD00BF940B00204F
:10C2400008B5024B1B68984708BD00BF640C00206E
:10C2500008B5024B1B68984708BD00BFF40B0020CF
:10C2600008B5024B1B68984708BD00BF180C00209A
:10C27000704700BF704700BF704700BF704700BFE6
:10C28000704700BF704700BF704700BF704700BFD6
:10C29000704700BF704700BF704700BF704700BFC6
:10C2A000704700BF704700BF704700BF704700BFB6
:10C2B000704700BF704700BF704700BF704700BFA6
:10C2C000704700BF704700BF704700BF704700BF96
:10C2D000704700BF704700BF704700BF704700BF86
:10C2E000704700BF704700BF704700BF704700BF76
:10C2F000704700BF704700BF704700BF704700BF66
:10C30000704700BF436830B523F470230C680A7986
:10C3100023F48073234343EA0223436082688D68D9
:10C32000CC680A4B45EA040C02EA03034A794CEA5A
:10C33000030343EA420383600B7CC26A013B22F49D
:10C340007002DBB242EA0353C36230BDFDF7F1FF76
:10C35000002301220274C360036003714371836090
:10C36000704700BF19B1836843F0010302E083689E
:10C3700023F001038360704719B1836843F480732D
:10C3800002E0836823F4807383607047C9B212B1FE
:10C390004368194302E0436823EA010141607047A2
:10C3A000836843F008038360704700BF8068C0F370
:10C3B000C0007047836843F004038360704700BF88
:10C3C0008068C0F38000704719B1836843F4A0030C
:10C3D00002E0836823F4A003836070478068C0F3A1
:10C3E000805070474368013923F4604343EA413386
:10C3F0004360704719B1436843F4006302E0436847
:10C4000023F4006343607047092930B511D94FF018
:10C41000030C0CFB01FC0725ACF11E0C05FA0CF516
:10C4200003FA0CFCC46824EA050343EA0C03C36066
:10C430000EE04FF0030C0CFB01FC072505FA0CF590
:10C4400003FA0CFC046924EA050343EA0C030361C4
:10C45000062A0DD80523013A5A434FF01F0C0CFA57
:10C4600002FC9140436B23EA0C020A4342631CE046
:10C470000C2A0DD805235A434FF01F0C233A0CFA0F
:10C4800002FC9140036B23EA0C020A4302630CE0B6
:10C4900005235A434FF01F0C413A0CFA02FC91401D
:10C4A000C36A23EA0C020A43C26230BD19B1836831
:10C4B00043F4801302E0836823F4801383607047A1
:10C4C000C06C80B2704700BF014B1868704700BF56
:10C4D0004C24014019B1436843F4806302E043688F
:10C4E00023F480634360704719B1436843F4805379
:10C4F00002E0436823F4805343607047836823F469
:10C50000E04341EA03038360704700BF19B18368C9
:10C5100043F4004302E0836823F4004383607047E0
:10C5200019B1836843F4021302E0836823F4021311
:10C53000836070478068C0F340507047092930B568
:10C5400011D94FF0030C0CFB01FC0725ACF11E0CBC
:10C5500005FA0CF503FA0CFCC46824EA050343EA67
:10C560000C03C3600EE04FF0030C0CFB01FC07252D
:10C5700005FA0CF503FA0CFC046924EA050343EA06
:10C580000C030361836BC3F3015CCCEB0202023248
:10C590004FF0050CD2B20CFB02F20CF11A0C0CFAA3
:10C5A00002FC914023EA0C030B43836330BD00BFC0
:10C5B000836B013923F4401343EA015383637047CB
:10C5C0000A5070472830405880B27047436823F4BF
:10C5D000400323F4007341EA03034360704700BF44
:10C5E00041628262704700BF436823F01F0341EA43
:10C5F00003034360704700BF20B1054B9A6842F4C3
:10C60000000203E0024B9A6822F400029A6070472D
:10C6100000240140036819420CBF0020012070472C
:10C62000C9430160704700BF4368006810EA1120E9
:10C6300004D0C9B219420CBF00200120704700BFCE
:10C640006FEA11210160704708B5134B98420FD073
:10C6500003F5A053984213D0A3F5C053984219D1C3
:10C660004FF40070012100F0F3FF4FF400700EE072
:10C670004FF48060012100F0EBFF4FF4806006E092
:10C680004FF40040012100F0E3FF4FF4004000218F
:10C6900000F0DEFF08BD00BF002801400268002353
:10C6A00022F001020260036043608360C3602D4B8F
:10C6B000984233D011D83C3B984229D006D8283B29
:10C6C000984221D0143398424BD11FE0264B984218
:10C6D00020D01433984244D11EE0244B98422CD0F1
:10C6E00008D8A3F5677398421DD003F5627398428A
:10C6F00037D11DE01E4B984229D0143398422BD0DD
:10C70000283B98422DD11DE01A4B12E0194B15E041
:10C71000184B18E0174B1BE0164B1EE0154B5A68E0
:10C7200042F470021CE0134B5A6842F0706217E04A
:10C73000114B5A6842F00F0212E00F4B5A6842F058
:10C74000F0020DE00C4B5A6842F4706208E00A4BAC
:10C750005A6842F4704203E0074B5A6842F4702270
:10C760005A6070476C000240440002401C040240C2
:10C770004404024000000240000402408A6870B590
:10C780000C6A0B6944EA02024C691A438B69224322
:10C79000CC6905684E6A42EA030323438C6A33433B
:10C7A00025F4FE4C23432CF0F00C43EA0C03036009
:10C7B000CB6843600B6883604B68C36070BD00BF8B
:10C7C00000238362036043608360C360036143614D
:10C7D0008361C36103624362704700BF19B103689C
:10C7E00043F0010302E0036823F001030360704794
:10C7F00012B10368194302E0036823EA01010160F2
:10C80000704700BF406880B2704700BF10F0805F83
:10C8100014BF044B044B1B6803420CBF00200120D3
:10C82000704700BF000402400000024010F0805F2B
:10C8300014BF024B024B5860704700BF0004024017
:10C840000000024010F0805F14BF044B044B1B68D3
:10C8500003420CBF00200120704700BF00040240CB
:10C860000000024010F0805F14BF024B024B586082
:10C87000704700BF0004024000000240044B002249
:10C880001A605A609A60DA60024A5A61704700BFC3
:10C8900000040140FFFF0700837930B50168027989
:10C8A0004BB3184BCC431D6890F805C004EA05054E
:10C8B0001D605D682C405C60D45844EA0101D15091
:10C8C00002689868D14301EA00009860D868014086
:10C8D000BCF1100FD96007D1996811439960D968EC
:10C8E00041EA0202DA600BE05CF8031041EA02025E
:10C8F0004CF8032004E0034BD05820EA0101D1504A
:10C9000030BD00BF0004014000230C22837142713E
:10C9100003600371704700BF024B1A6940EA0202CC
:10C920001A61704700040140034B5B6918420CBF59
:10C9300000200120704700BF00040140014B5861F6
:10C94000704700BF00040140054B1A685B69034053
:10C9500001D1184603E010420CBF002001207047AF
:10C9600000040140014B5861704700BF00040140C2
:10C97000044B1A6802F038021A601A6840EA020290
:10C980001A60704700200240044B1A6822F0080227
:10C990001A601A6840EA02021A60704700200240DA
:10C9A000044B1A6822F010021A601A6840EA020268
:10C9B0001A60704700200240034B044A5A6002F19B
:10C9C00088325A60704700BF00200240230167454B
:10C9D000024B1A6942F080021A617047002002403F
:10C9E000014BD8698008704700200240014B186A4B
:10C9F000704700BF00200240024BD869C0F34000DE
:10CA0000704700BF00200240024B1868C0F340107E
:10CA1000704700BF0020024019B1054B1A6910434E
:10CA200003E0034B1A6922EA00001861704700BF57
:10CA300000200240012804D1054BD86900F0010014
:10CA400005E0034BDB6818420CBF00200120704753
:10CA500000200240014BD860704700BF0020024018
:10CA6000094BDA6812F0010F01D001200BE0DA68FF
:10CA700012F0040F01D0022005E0DB6813F0100F64
:10CA800014BF0320042070470020024013B5044661
:10CA90000AE000230193FF3301E0019B013B019376
:10CAA000019B002BF9D1013CFFF7DAFF012802D1ED
:10CAB000002CEED100E004B905201CBDF8B5124CE5
:10CAC000124B0546A36003F188330F20A3600E4686
:10CAD0001746FFF7DBFF042814D1236945F0F8055A
:10CAE00043F0100323612E43094B37430B305F8023
:10CAF000FFF7CCFF012805D0226941F6EF7302EA67
:10CB000003032361F8BD00BF0020024023016745F5
:10CB100000F8FF1F38B5054640F6FF70FFF7B6FF77
:10CB200004283CD11E4C1F4B40F6FF70A36003F15C
:10CB30008833A360236943F020032361236943F012
:10CB400040032361FFF7A2FF042820D1226941F6A8
:10CB5000DF7302EA03032361236943F010032361B7
:10CB60001DB1114B4FF0000202E00F4B4FF0A50238
:10CB70001A8040F6FF70FFF789FF01280FD0084A9E
:10CB800041F6EF73116901EA0303136107E001281D
:10CB900005D0226941F6DF7302EA0303236138BD41
:10CBA000002002402301674500F8FF1F10B504462E
:10CBB0000F20FFF76BFF04283DD11F4A1F4BE443B2
:10CBC000936003F1883393601169E3B241F010017F
:10CBD000FF2B116106D01A4A0B301381FFF756FF65
:10CBE00004281FD1C4F30723FF2B06D0144A0F20BB
:10CBF0005381FFF74BFF042814D1C4F30743FF2BE5
:10CC000006D00F4A0F209381FFF740FF042809D177
:10CC1000240EFF2C01D1042006E0094B0F20DC81FB
:10CC2000FFF734FF012806D0034A41F6EF7311697C
:10CC300001EA0303136110BD002002402301674590
:10CC400000F8FF1F70B504460F200E46FFF71EFFC9
:10CC5000042815D10B4D0C4B0B30AB6003F188331E
:10CC6000AB602B6943F010032B612680FFF70EFFAA
:10CC7000012805D02A6941F6EF7302EA03032B610C
:10CC800070BD00BF002002402301674570B5044617
:10CC90000F200E46FFF7FAFE042810D1084D0B3086
:10CCA0002B6943F001032B612680FFF7EFFE01287B
:10CCB00005D02A6941F6FE7302EA03032B6170BDB9
:10CCC0000020024070B504460F200E46FFF7DEFE3E
:10CCD000042818D10C4DB3B22A690B3042F001027E
:10CCE0002A612380FFF7D2FE042804D1360C668027
:10CCF0000B30FFF7CBFE012805D02A6941F6FE7301
:10CD000002EA03032B6170BD0020024010B540F61B
:10CD1000FF70FFF7BBFE04282CD1174C174B40F6D1
:10CD2000FF70A36003F18833A360236943F02003FD
:10CD30002361236943F040032361FFF7A7FE042822
:10CD400010D1226941F6DF7302EA030323612369EC
:10CD50004FF0A50243F010032361094B0B301A80FA
:10CD6000FFF794FE012805D0226941F6EF7302EA2D
:10CD70000303236110BD00BF00200240230167456B
:10CD800000F8FF1F10B540F6FF70FFF77FFE042884
:10CD900014D10B4C40F6FF70236943F00403236168
:10CDA000236943F040032361FFF770FE012805D09B
:10CDB000226941F6FB7302EA0303236110BD00BF41
:10CDC0000020024038B5054640F6FF70FFF75EFED2
:10CDD000042815D10B4C40F6FF70236943F0020381
:10CDE00023616561236943F040032361FFF74EFE31
:10CDF000012805D0226941F6FD7302EA030323618D
:10CE000038BD00BF00200240CB78F0B513F0100F02
:10CE100018BF8A78098803F00F0C18BF4CEA020C7F
:10CE200011F0FF0F1AD0046800220126964006EA8E
:10CE30000105B5420ED196000F27B7400CFA06F651
:10CE400024EA07043443282B01D1456102E0482B32
:10CE500008BF05610132082AE7D10460FF291CD907
:10CE60004468002202F108050126AE4006EA0105E9
:10CE7000B5420ED196000F27B7400CFA06F624EA09
:10CE800007043443282B01D1456102E0482B08BF39
:10CE900005610132082AE5D14460F0BD0423C37066
:10CEA000022383704FF0FF33038070478368194279
:10CEB0000CBF002001207047806880B2704700BF1F
:10CEC000C36819420CBF002001207047C06880B2BF
:10CED000704700BF01617047416170470AB101614D
:10CEE00000E04161704700BFC160704741F480338A
:10CEF000836181618361836983697047064A10B5E4
:10CF000014684FF6807341EA001104EA030341EA12
:10CF10000303136010BD00BF00000140014B186007
:10CF2000704700BF1C0020420304154A00F4401C57
:10CF30001B0CBCF5401F30B5546806D1556824F071
:10CF4000706425F07065556011E010F4801F06D004
:10CF5000C0F303424FF0030C0CFA02F203E0420D5F
:10CF6000120113FA02F224EA020444F0706419B1C7
:10CF7000400D000183401C43014B5C6030BD00BF8D
:10CF80000000014001F003039B000F229A4010FAB9
:10CF900003F310B58908074C023154F8210020EA48
:10CFA000020244F8212054F82120134344F8213090
:10CFB00010BD00BF000001400120014608B500F08F
:10CFC00047FB0120002100F043FB08BD08B5264BBC
:10CFD00098422BD00CD8A3F5006398421AD003F5E1
:10CFE000806398421CD0A3F5006398423AD10BE0CD
:10CFF0001E4B984226D003F58063984228D0A3F5B3
:10D00000006398422ED117E00420012100F020FB9C
:10D01000042024E00820012100F01AFB08201EE073
:10D020001020012100F014FB102018E02020012125
:10D0300000F00EFB202012E04020012100F008FB50
:10D0400040200CE08020012100F002FB802006E05F
:10D050004FF48070012100F0FBFA4FF48070002142
:10D0600000F0F6FA08BD00BF00140140001C0140AA
:10D070000B4B4FF0FF316FF07042C3F88010C3F8D4
:10D080008420C3F88011C3F88421002303F1C00178
:10D09000034A013300200F2B42F82100F6D17047DC
:10D0A00000E100E0094B4FF0206058600848002282
:10D0B0004FF0FF319A60D8601A615A619A61DA6163
:10D0C0001A625A629962D9621963704700ED00E0F2
:10D0D0000000FA0540F0BE60024B40F42020D8600A
:10D0E000704700BF00ED00E030B5C27803787AB336
:10D0F0001C4A4178D2684FF00F0CD243C2F302228F
:10D100002CFA02FCC2F104029140807803F0030281
:10D110000CEA000C4CEA010CD2004FEA0C1CFF2078
:10D1200090400CFA02FC012403F01F02944099087D
:10D130000D4AC03152F821500CEA000C25EA0000DB
:10D140004CEA00005B0942F8210042F8234008E065
:10D1500003F01F02012191405B09034A203342F88A
:10D16000231030BD00ED00E000E100E00023C370BB
:10D170000370437083707047024B5868C0F30930E6
:10D18000704700BF00ED00E0012200F01F0312FA1B
:10D1900003F34009044A403052F8200018409842F6
:10D1A00014BF00200120704700E100E0014B18602F
:10D1B000704700BF00EF00E000F01F0301229A401B
:10D1C0004009024B603043F82020704700E100E046
:10D1D000024B58688005800D704700BF00ED00E0ED
:10D1E000012200F01F0312FA03F34009044A8030C1
:10D1F00052F820001840984214BF002001207047C8
:10D2000000E100E0014B1868704700BF00ED00E04E
:10D2100021F0604121F07F01014B0143996070478B
:10D2200000ED00E0014A024BDA6070470400FA05A5
:10D2300000ED00E0014A024BDA6070470100FA0598
:10D2400000ED00E019B1054B1A69104303E0034BF0
:10D250001A6922EA00001861704700BF00ED00E083
:10D2600000F01F00012313FA00F019B1044B5A6AB1
:10D27000104303E0024B5A6A22EA000058627047EA
:10D2800000ED00E0144B70B5DC684FF0FF0CE44398
:10D29000C4F302242CFA04F5C4F1040411FA04F4D2
:10D2A000C0F30126F6000CFA06FC02EA050545EA81
:10D2B0000404240114FA06F6C0F38110063053F872
:10D2C000202022EA0C0243F8202053F820201643A5
:10D2D00043F8206070BD00BF00ED00E0C0F3832084
:10D2E00001238340044A506A03EA0000984214BFB5
:10D2F00000200120704700BF00ED00E000F01F009B
:10D3000001228240024B59680A435A60704700BFAD
:10D3100000ED00E000F01F020123013A13FA02F2CF
:10D32000024B59680A435A60704700BF00ED00E0A5
:10D33000C0F3833001238340044A506A03EA0000AB
:10D34000984214BF00200120704700BF00ED00E0AC
:10D35000C0F3814313B90A4BD86A10E0012B0CD1FA
:10D36000074AC0F30153906ADA00D040022B14BF81
:10D3700000F00F0000F0FF0001E0014B186B704758
:10D3800000ED00E010F4800F0BBF024B014B586B17
:10D39000986B704700ED00E008B5F6F7E9FE08BDB0
:10D3A00008B50001F6F7E1FE08BD00BF08B5F6F7C5
:10D3B000DAFE08BD08B5F6F7D4FE08BD08B5F6F7E5
:10D3C000CEFE08BD08B5F6F7C8FE08BD0D4B0E4AE7
:10D3D000196841F001011960596801EA02025A60B6
:10D3E0001A6822F0847222F480321A601A6822F4D9
:10D3F00080221A605A6822F4FE025A6000229A6063
:10D40000704700BF001002400000FFF80C4BB0F561
:10D41000803F1A6822F480321A601A6822F480224F
:10D420001A6003D0B0F5802F08D103E01A6842F4E7
:10D43000803202E01A6842F4A0221A60704700BFEE
:10D4400000100240034B1A6822F0F80242EAC002C0
:10D450001A60704700100240014B1860704700BF0F
:10D4600000004242044B5A6822F47C1240EA020255
:10D470000A435A60704700BF00100240014B186019
:10D48000704700BF60004242034B5A6822F003021B
:10D4900040EA02025A60704700100240024B58688E
:10D4A00000F00C00704700BF00100240034B5A68A8
:10D4B00022F0F00240EA02025A6070470010024077
:10D4C000034B5A6822F4E06240EA02025A60704755
:10D4D00000100240034B5A6822F4605242EAC00234
:10D4E0005A6070470010024019B1054B1A7810437A
:10D4F00003E0034B1A7822EA00001870704700BF5F
:10D5000009100240014B1860704700BFD80042422A
:10D51000034B5A6822F4404240EA02025A607047C4
:10D5200000100240064B002201281A701A7002D027
:10D53000042804D101E0187001E005221A70704738
:10D5400020100240014B1860704700BF8004424227
:10D55000024B1A6A40EA02021A6270470010024047
:10D56000014B1860704700BF3C0442421F4B10B58E
:10D570005A6802F00C02042A13D0082A11D15A6802
:10D580005968C2F38342023211F4803F03D05B68D2
:10D5900013F4003F01D0164B00E0164B5A430260D3
:10D5A00001E0144B0360114A134B51680468C1F346
:10D5B0000311595C34FA01F141605468C4F3022C40
:10D5C00013F80C4031FA04F484605468C4F3C22C9C
:10D5D00013F80CC021FA0CF1C1605268C2F3813219
:10D5E0009B181B7CB1FBF3F1016110BD00100240E0
:10D5F00000093D0000127A00401F010819B1054BD7
:10D600005A69104303E0034B5A6922EA000058614B
:10D61000704700BF0010024019B1054B9A691043D2
:10D6200003E0034B9A6922EA00009861704700BF4B
:10D630000010024019B1054BDA69104303E0034BB7
:10D64000DA6922EA0000D861704700BF001002408A
:10D6500019B1054BDA68104303E0034BDA6822EA9C
:10D660000000D860704700BF0010024019B1054BA0
:10D670001A69104303E0034B1A6922EA000018619B
:10D68000704700BF00100240014B1860704700BF98
:10D6900040044242014B1860704700BF4C004242B8
:10D6A000014B1870704700BF071002404309012B5F
:10D6B00002D1084B1B6805E0022B0BBF054B054B45
:10D6C0001B6A5B6A00F01F0033FA00F000F00100F3
:10D6D000704700BF0010024008B53120FFF7E6FF99
:10D6E000094B18705A6801325A601A7822B95A6880
:10D6F00040F2FF139A42F0D13120FFF7D7FF0038F4
:10D7000018BF012008BD00BFDC060020024B5A6A8A
:10D7100042F080725A62704700100240034B9B68CF
:10D7200018420CBF00200120704700BF00100240CB
:10D73000014B1870704700BF0A1002400B884A88DE
:10D74000B1F804C01A43CB8842EA0C02B1F808C011
:10D750001A434B8930B542EA0C028D89B0F800C0FB
:10D76000CC891A432A4322430CF4415313439BB2FE
:10D770000380838B23F400631B041B0C83830B8ABD
:10D78000038230BD00234FF00702C3810282038071
:10D7900043808380C380038143818381704700BFBE
:10D7A00000234381038043808380C3804FF00203C2
:10D7B0000381704721B103889BB243F0400304E02A
:10D7C000038823F040031B041B0C0380704700BF39
:10D7D00021B1838B9BB243F4806304E0838B23F4F9
:10D7E00080631B041B0C8383704700BF090901235E
:10D7F00013FA01F189B21AB183889BB2194303E08D
:10D8000083889BB223EA0101818070471AB1838823
:10D810009BB2194303E083889BB223EA0101818014
:10D82000704700BF81817047808980B2704700BF18
:10D830004FF6FF63994205D003889BB243F480738F
:10D84000038002E0038819400180704721B183887A
:10D850009BB243F0040304E0838823F004031B0419
:10D860001B0C8380704700BF038823F400631B04F4
:10D870001B0C038003889BB241EA030303807047BB
:10D8800003889BB243F480530380704721B103881F
:10D890009BB243F4005304E0038823F400531B04B9
:10D8A0001B0C0380704700BF012914BF008B808AC6
:10D8B00080B27047008A80B2704700BFB1F5804FD8
:10D8C00004D103889BB243F4804304E0038823F42B
:10D8D00080431B041B0C0380704700BF038919425F
:10D8E0000CBF002001207047202906D1038903883E
:10D8F0009BB243F04003038008E0402901D008298F
:10D9000001D1038902E0C94389B20181704700BF98
:10D91000012301F00F0213FA02F2B0F804C00089EB
:10D920001FFA8CFC80B2104006D009098B401CEA1B
:10D93000030F0CBF00200120704700BF552906D1FE
:10D94000038903889BB243F0400303800DE056290E
:10D9500001D0532901D1038907E001F00F01012310
:10D9600013FA01F1C94389B201817047838BF0B585
:10D9700023F47A6323F01F031B041B0C83834FF0F3
:10D98000020303840B89868B022B87B004460D4665
:10D99000B6B201D1002225E001A88F88FFF7E6FD8D
:10D9A000EB88002F0CBF01270227B3F5007F2989E0
:10D9B000019A06D1A3F5FB7353430902B3FBF1F3BC
:10D9C00005E00A2349015A434F43B2FBF7F30533FD
:10D9D0000A229BB2B3FBF2F303F001021202C3F37B
:10D9E0004F0392B2991E89B2FE2928BF002228BF98
:10D9F0000223E98842EA03030B439BB223842B886A
:10DA00006A8846EA0303A98843F4006313436A89DA
:10DA10000B4313439BB2A38307B0F0BD08B5154B6E
:10DA200098421BD003F57443984204D0A3F5784381
:10DA300098421DD10AE001214FF48050FFF708FE03
:10DA40004FF480500021FFF703FE11E04FF48040B7
:10DA50000121FFF70BFE4FF4804006E04FF4004039
:10DA60000121FFF703FE4FF400400021FFF7FEFD08
:10DA700008BD00BF003C0040042804D1054B1A68D3
:10DA800042F0040203E0034B1A6822F004021A6019
:10DA9000704700BF10E000E0014B5860704700BFC6
:10DAA00010E000E0012804D1084B1A6842F001029E
:10DAB00006E010F1020F05D1044B1A6822F00102B2
:10DAC0001A6002E0014B00229A60704710E000E00B
:10DAD00020B1054B1A6842F0020203E0024B1A68BB
:10DAE00022F002021A60704710E000E0014B9868D3
:10DAF000704700BF10E000E0C308022B0BBF044BCF
:10DB0000034B1B68DB6833FA00F000F0010070473C
:10DB100010E000E0038803F08F0303800388B1F86E
:10DB200006C04A889BB243EA0C0313439BB20380AE
:10DB30008B8883850B880385064B984203D003F5B9
:10DB40000063984201D10B7A03864FF00103838270
:10DB5000704700BF002C0140038C2DE9F04123F0F9
:10DB600001031B041B0C0384038C0A894C8823F0DB
:10DB700002031C4E14431B048288B1F806C0058BB7
:10DB80001B0CA4B2B04244EA030392B20C88ADB2BB
:10DB9000A0F834C003D006F50066B04218D18E89D3
:10DBA0004F89B1F80E804FF6F77C03EA0C0C4CEA73
:10DBB000070748EA06064FF6FB73898847F6FF4CCD
:10DBC00002EA0C0C07EA0303B2B20B4342EA0C026E
:10DBD0004FF68F7105EA010121438280018303849E
:10DBE000BDE8F081002C0140038C2DE9F04123F0C9
:10DBF00010031B041B0C0384028CB1F808C022F034
:10DC0000200212048488120C4B8842EA0C1242EA69
:10DC10000313A2B21B4C068BB1F806C0A0420D88BC
:10DC2000B6B29BB2A0F838C003D004F50064A0429D
:10DC30001BD1B1F80A804FF67F748F8903EA040480
:10DC400047F2FF3C02EA0C0C44EA0814CA894FF67A
:10DC5000BF73898804EA03034CEA870C43EA011383
:10DC60004CEA82023C469BB292B248F6FF7106EA49
:10DC7000010141EA052189B2828001830384BDE864
:10DC8000F08100BF002C0140038C2DE9F04123F40A
:10DC900080731B041B0C0384028CB1F808C022F4AF
:10DCA000007212048488120C4B8842EA0C2242EA69
:10DCB0000323A2B21A4C868BB1F806C0A0420D888D
:10DCC000B6B29BB2A0F83CC003D004F50064A042F9
:10DCD0001BD1B1F80A804FF2FF748F8903EA040464
:10DCE00044F6FF7C02EA0C0C44EA0824CA894FF689
:10DCF000FF33898804EA03034CEA071C43EA012343
:10DD00004CEA02123C469BB292B24FF68F7106EA81
:10DD100001012943828081830384BDE8F08100BF33
:10DD2000002C0140038CF0B523F480531B041B0C22
:10DD30000384B1F806C0078C0C8882880D89868B15
:10DD40004B88A0F840C0DFF848C0BFB2604592B22F
:10DD5000B6B203D00CF5006C604505D192048989F8
:10DD6000920C42EA811292B24DF6FF7C07EA0C0C4B
:10DD700048F6FF7106EA01014CEA053C41EA04213C
:10DD80004CEA033389B29BB2828081830384F0BD65
:10DD9000002C0140B1F802C00B888A884CEA0303CA
:10DDA000B1F806C013430A8943EA0C03B1F80AC06C
:10DDB00013438A8943EA0C0313439BB2A0F844300F
:10DDC000704700BF00234FF0FF3203724380828010
:10DDD0000380C380704700BF0023C381038043805A
:10DDE0008380C380038143818381704700234FF088
:10DDF00001020381038043808280C380704700BF9B
:10DE000000238381038043808380C3800381438117
:10DE1000704700BF21B103889BB243F0010304E0C7
:10DE2000038823F001039B059B0D0380704700BF0F
:10DE300039B1B0F844306FEA43436FEA53439BB2C1
:10DE400003E0B0F844305B045B0CA0F8443070474A
:10DE50001AB183899BB2194303E083899BB223EAF9
:10DE600001018181704700BF818270470A43A0F899
:10DE7000482070471AB183899BB2194303E0838914
:10DE80009BB223EA01018181704700BF038923F01F
:10DE900007031B041B0C0381704700BFB0F808C0C8
:10DEA0005FFA8CFC41EA0C0C42EA0C0C4CEA032CA5
:10DEB0001FFA8CFCA0F808C0704700BF10B50446DC
:10DEC000FFF7ECFF23899BB243F48043238110BD0D
:10DED00010B50446FFF7E2FF238923F077031B0404
:10DEE0001B0C43F07703238110BD00BF01858282A4
:10DEF000704700BF038823F070039B059B0D41EA28
:10DF000003030380704700BF038923F070031B04E1
:10DF10001B0C41EA03030381704700BF10B50446A0
:10DF2000FFF7F2FF23899BB243F00703238110BD63
:10DF300030B50489B0F818C0058C2CF4407CADB223
:10DF40002CF0030C24F007044FEA0C4C25F02205BA
:10DF500042EA050524044FEA1C4C45EA0315240C4B
:10DF60004CF4807C21434CF0010CADB20181A0F84F
:10DF700018C0058430BD00BF038B23F070031B0461
:10DF80001B0C41EA03030383704700BF038B23F498
:10DF9000E0431B041B0C43EA01239BB2038370473D
:10DFA000838B23F070031B041B0C41EA0303838360
:10DFB000704700BF838B23F4E0431B041B0C43EA30
:10DFC00001239BB28383704721B103889BB243F046
:10DFD000800304E0038823F080039B059B0D0380EE
:10DFE000704700BF21B183889BB243F0040304E073
:10DFF000838823F004031B041B0C8380704700BF3D
:10E0000021B183889BB243F0080304E0838823F0A6
:10E0100008031B041B0C8380704700BF21B1838859
:10E020009BB243F0010304E0838823F001031B0447
:10E030001B0C8380704700BF038B23F008031B0475
:10E040001B0C41EA03030383704700BF038B23F4D7
:10E0500000631B041B0C43EA01239BB2038370473C
:10E06000838B23F008031B041B0C41EA0303838307
:10E07000704700BF838B23F400631B041B0C43EA2F
:10E0800001239BB283837047038B23F004031B049B
:10E090001B0C41EA03030383704700BF038B23F487
:10E0A00080631B041B0C43EA01239BB2038370476C
:10E0B000838B23F004031B041B0C41EA03038383BB
:10E0C000704700BF838B23F480631B041B0C43EA5F
:10E0D00001239BB283837047038B23F080031B04CF
:10E0E0001B0C41EA03030383704700BF038B5B04EF
:10E0F0005B0C43EA01239BB203837047838B23F0BD
:10E1000080031B041B0C41EA03038383704700BF99
:10E11000838B5B045B0C43EA01239BB283837047D0
:10E12000038C23F002031B041B0C41EA030303844A
:10E13000704700BF038C23F008031B041B0C41EA4B
:10E1400003030384704700BF038C23F020031B04E8
:10E150001B0C43EA01139BB203847047038C23F02A
:10E1600080031B041B0C43EA01139BB2038470471A
:10E17000038C23F400731B041B0C43EA01239BB2A2
:10E1800003847047038C23F400631B041B0C43EAD5
:10E1900001239BB203847047038C23F400531B04B8
:10E1A0001B0C43EA01339BB20384704701238B406D
:10E1B0008A40018C89B221EA03030384018C0A435B
:10E1C00092B20284704700BF04238B408A40018CC6
:10E1D00089B221EA03030384018C0A4392B20284C8
:10E1E000704700BF01238B40B0F820C010B51FFA64
:10E1F0008CFC2CEA0303038409B1082909D11830E7
:10E20000490844584FF68F7304EA030343504358B8
:10E210000CE004391830C1F34E01445848F6FF733E
:10E2200004EA030343501202435892B243EA020243
:10E23000425010BD21B103889BB243F0020304E0B9
:10E24000038823F002039B059B0D0380704700BFEA
:10E2500021B103889BB243F0040304E0038823F058
:10E2600004039B059B0D0380704700BF21B1838889
:10E270009BB243F0800304E0838823F080031B04F7
:10E280001B0C8380704700BF038823F008039B05A5
:10E290009B0D038003889BB241EA03030380704710
:10E2A000838823F070031B041B0C838083889BB23C
:10E2B00041EA030383807047038923F007031B04AB
:10E2C0001B0C038103899BB241EA0303038170475E
:10E2D000038923F080031B041B0C038103899BB279
:10E2E00041EA030303817047818470478185704749
:10E2F000818670470187704781877047A0F840107A
:10E30000704700BF038B23F00C031B041B0C03831B
:10E31000038B9BB241EA030303837047038B23F40F
:10E3200040631B041B0C0383038B9BB243EA012352
:10E330009BB20383704700BF838B23F00C031B0445
:10E340001B0C8383838B9BB241EA03038383704757
:10E35000838B23F440631B041B0C8383838B9BB24E
:10E3600043EA01239BB28383704700BF0388DBB27B
:10E37000038003889BB241EA03030380704700BF18
:10E38000808E80B2704700BF008F80B2704700BFA0
:10E39000808F80B2704700BFB0F8400080B27047F5
:10E3A000808C80B2704700BF008D80B2704700BF84
:10E3B000038A19420CBF002001207047C94389B26B
:10E3C00001827047038A828911EA030092B203D066
:10E3D00011420CBF00200120704700BFC94389B221
:10E3E00001827047B0F820C010B52CF0010C4FEA44
:10E3F0000C4C4FEA1C4CA0F820C0048BB0F820C095
:10E40000A4B21FFA8CFC24F0F30442EA04042CF0BA
:10E41000020C44EA03144CF0010C4CEA010CA4B2C7
:10E420000483A0F820C010BDB0F820C010B52CF0B7
:10E43000100C4FEA0C4C4FEA1C4CA0F820C0B0F86E
:10E4400018C0048C2CF4407CA4B24FEA0C5C4FEA58
:10E450001C5C24F020044CEA022C44F010044CEA2A
:10E46000033C44EA01141FFA8CFCA4B2A0F818C0C3
:10E47000048410BD38B50D46602D1146044603D105
:10E480000122FFF7D1FF02E00122FFF7ABFF29468F
:10E490002046FFF739FD23899BB243F00703238110
:10E4A00038BD00BFF8B50C46A2884988B4F800C052
:10E4B000054600290CBF02270027012A0CBF0226AF
:10E4C00001262389BCF1000F10D1FFF78BFF2846EE
:10E4D000E188FFF717FF2846394632462389FFF7C0
:10E4E000A3FF2846E188FFF719FF0FE0FFF79CFF25
:10E4F0002846E188FFF712FF28463946324623892D
:10E50000FFF770FF2846E188FFF7FCFEF8BD00BF6B
:10E5100038B50B880C4605464BB94988A288238933
:10E52000FFF760FF2846E188FFF7ECFE53E0042B7D
:10E5300009D14988A2882389FFF776FF2846E18818
:10E54000FFF7ECFE47E0082BB1F802C0B1F804E099
:10E55000098920D1028C22F480721204120C0284E8
:10E56000838B028C9BB292B223F0F30322F40072ED
:10E5700043EA011142EA0C2C89B21FFA8CFC41EAF1
:10E580000E0E4CF4807CA0F81CE0A0F820C0E188BE
:10E59000FFF7D2FE1FE0028C22F480521204120C0C
:10E5A0000284838B028C23F4407392B21B051B0DF3
:10E5B00022F4005243EA0E2342EA0C3C43EA0133C0
:10E5C0001FFA8CFC9BB24CF4805C8383A0F820C0C3
:10E5D000E188FFF7BDFE38BD08B52D4B984237D016
:10E5E0000BD8A3F50063984226D003F580639842C8
:10E5F00028D0B0F1804F4AD118E0264B984233D052
:10E6000004D8A3F58063984241D127E0224B984279
:10E6100004D003F50063984239D12EE04FF4006036
:10E620000121FFF715F84FF400602DE001200146AD
:10E63000FFF71CF801201CE002200121FFF716F86B
:10E64000022016E004200121FFF710F8042010E05A
:10E6500008200121FFF70AF808200AE01020012114
:10E66000FFF704F8102004E020200121FEF7FEFF50
:10E6700020200021FEF7FAFF09E04FF400500121AD
:10E68000FEF7E6FF4FF400500021FEF7E1FF08BD62
:10E69000000C004000140040002C01400023838146
:10E6A0004FF416528380C38003814FF00C03026045
:10E6B000438170470A8810B54C88B1F804C0038ABA
:10E6C000C98844EA020242EA0C0223F470630A4356
:10E6D0001B041B0C92B242EA0303038210BD00BF6D
:10E6E0000023C380038043808380704721B18389E6
:10E6F0009BB243F4005304E0838923F400531B04CA
:10E700001B0C8381704700BF01F01F034FF0010C09
:10E71000C1F3421161450CFA03F301D10C3004E05E
:10E72000022901D1103000E014301AB1026842EA27
:10E73000030302E0026822EA03030360704700BF9C
:10E740001AB1838A9BB2194303E0838A9BB223EAFE
:10E7500001018182704700BF038A23F00F031B046D
:10E760001B0C0382038A9BB241EA030303827047B6
:10E77000838923F400631B041B0C838183899BB270
:10E7800041EA03038381704721B183899BB243F03F
:10E79000020304E0838923F002031B041B0C838122
:10E7A000704700BF038A23F020031B041B0C038265
:10E7B000038A9BB241EA03030382704721B1038AB3
:10E7C0009BB243F4804304E0038A23F480431B0498
:10E7D0001B0C0382704700BFC905C90D81807047BB
:10E7E0008088C005C00D704783899BB243F0010348
:10E7F00083817047038BDBB20383038B9BB243EAB5
:10E8000001230383704700BF038B03F47F4303831B
:10E81000038B9BB241EA03030383704721B1838AD0
:10E820009BB243F0200304E0838A23F020031B04FF
:10E830001B0C8382704700BF21B1838A9BB243F0D7
:10E84000100304E0838A23F010031B041B0C838253
:10E85000704700BF21B1838A9BB243F0080304E0F4
:10E86000838A23F008031B041B0C8382704700BFBC
:10E87000838A23F004031B041B0C8382838A9BB2CC
:10E8800041EA03038382704721B1838A9BB243F03C
:10E89000020304E0838A23F002031B041B0C83821F
:10E8A000704700BF038819420CBF00200120704749
:10E8B000C94389B2018070474FF0010CC1F3421285
:10E8C00001F01F0362450CFA03F301D1828903E0D2
:10E8D000022A0CBF028A828A92B21340028892B244
:10E8E0000BB9184607E0090A012313FA01F1114296
:10E8F0000CBF002001207047090A01238B40DB4335
:10E900009BB20380704700BF038ACA8823F4405338
:10E910001B041B0C1343038283898A8830B5044689
:10E9200008890D4623F4B053498940EA020223F0D6
:10E930000C030A431B041B0C92B242EA0303A3819B
:10E94000A38AAA8923F440731B041B0C134387B0CA
:10E95000A38201A8FEF70AFE0E4B2A689C420CBF58
:10E96000049B039B1921594392006423B1FBF2F1EC
:10E97000B1FBF3F21201100903FB1011090132314E
:10E98000B1FBF3F303F00F0343EA020292B22281D8
:10E9900007B030BD0038014008B5214B98422BD05C
:10E9A00008D8A3F50063984216D003F58063984217
:10E9B00034D119E01B4B984226D003F568439842A6
:10E9C0002CD101214FF48040FEF742FE4FF48040ED
:10E9D0000021FEF73DFE21E04FF400300121FEF75B
:10E9E00045FE4FF4003016E04FF480200121FEF781
:10E9F0003DFE4FF480200EE04FF400200121FEF791
:10EA000035FE4FF4002006E04FF480100121FEF7A0
:10EA10002DFE4FF480100021FEF728FE08BD00BF38
:10EA2000004C004000500040684620F007018D4631
:10EA300001B5002303E00B495958995004330A4AA1
:10EA40000A4998188842F6D3094B02E0002243F89D
:10EA5000042B084A9342F9D3F5F792FBBDE8014035
:10EA600085467047982001080000002030020020F1
:10EA700030020020880D002010B5074C20B9226814
:10EA80004FF00103138205E0044B1B681B68984795
:10EA900020680A3010BD00BF200D0020DC0C0020D3
:10EAA00010B50A4B0A4A1B685178DA7891420AD3AA
:10EAB000997841B99C8834B99A72064B1B685B6897
:10EAC0009847204600E0022010BD00BF200D002026
:10EAD00004010020DC0C002010B5074C20B922688E
:10EAE0004FF00103138205E0044B1B689B689847B5
:10EAF00020680C3010BD00BF200D0020DC0C002071
:10EB000038B50E4C0E4B22681B68D1789B69507942
:10EB1000984723689A7A7AB170B91A7962B99D7860
:10EB200055B9084B1B68DB68984723682846597914
:10EB3000DA78D9721A7300E0022038BD200D002067
:10EB4000B80C0020DC0C002008B50246244B20B98C
:10EB50001B684FF00201198240E0224A4FF0000189
:10EB60001B681180197811F07F0113D15B7A13F0C3
:10EB7000200F03D0117841F00201117013F0400F03
:10EB8000184B15BF1A781A7822F0010242F00102E0
:10EB90001A701EE0012921D0022901D000221DE0B7
:10EBA000597911F0800F01F00F0306D00E4951F88A
:10EBB000233003F03003102B06E00B4951F82330CB
:10EBC00003F44053B3F5805F03D1137843F001039E
:10EBD0001370064B1B681B699847024A104608BD14
:10EBE000200D0020800D0020005C0040DC0C002087
:10EBF00010B51E4B19684A7912F0800F22F080037D
:10EC000005D01B4850F8230000F0300004E01848FD
:10EC100050F8230000F44050164C94F800C06345AF
:10EC200022D24C8804BBF8B1897AE9B112F0800F86
:10EC300009D00F4948F6BF7251F8230000EA0202DA
:10EC400082F0100208E00A494BF68F7251F8230057
:10EC500000EA020282F4805241F82320064B1B682E
:10EC60009B699847002000E0022010BD200D002085
:10EC7000005C004004010020DC0C002008B5064BBD
:10EC80001B685A7A42F020025A72044B1B68DB69F7
:10EC90009847002008BD00BF200D0020DC0C00209C
:10ECA000054B1A68538A18B98988CB1A138201E078
:10ECB00008681818704700BF200D002030B50E4BB3
:10ECC0001C78002310E05FFA83FC4FEA8C0202F10B
:10ECD000804202F5B842156848F68F7105EA0101D5
:10ECE00041EA0C0111600133A342ECD3034B40F025
:10ECF0008000186030BD00BF040100204C5C004063
:10ED0000704700BF08B50C4B002093F82C1000F0A2
:10ED10004FFE0A4B1B68187A082807D1084B4FF49E
:10ED200080521A80074B4FF010021A80092814BF36
:10ED30000020012008BD00BF80000020200D002021
:10ED4000820D0020840D002070B52D4B1C68237AA5
:10ED5000032B01D0052B46D1A369228AABB1A2B106
:10ED6000A58A954228BF154628469847228A638A75
:10ED7000521BEB18064622826382002000F0E8FD59
:10ED80002A460146304600F0FBFB238A5BB11D4B4F
:10ED90004FF4405200201A80014600F0E7FD1A4B64
:10EDA0004FF030021A80A28A238A9A4203D8144B69
:10EDB00003221B6803E0124A1BB1136805221A7272
:10EDC0000DE0126806211172104A1168104A89B2CA
:10EDD0008A18520013600C4B4FF030021A80084B17
:10EDE0001B681B7A06E0072B03D10A4B1B68DB6804
:10EDF00098470823024A12681372FFF783FF70BD19
:10EE0000200D0020820D0020840D0020505C004069
:10EE100002300020B80C0020F8B5244B1C68238A6F
:10EE2000267ABBB9042E15D1214822490278012A3D
:10EE30000BD1214C214A24680370A0B282185200E1
:10EE400013604FF030020A802BE04FF010030B806C
:10EE5000072626E0A68AA2699E4234BF35461D4693
:10EE60002846B34294BF0426022690470746002056
:10EE700000F060FD2A460146384600F069FB29464D
:10EE8000002000F073FD638A228AEB186382094B2D
:10EE9000551B4FF0300225821A80094B4FF4405227
:10EEA0001A80024B1B681E72F8BD00BF200D0020A7
:10EEB000E4060020840D0020505C00400230002059
:10EEC000820D002008B5144B1B681A7A022A01D063
:10EED000042A05D1FFF7A0FF0F4B1B681B7A14E033
:10EEE000062A11D15A78052A0AD11A7812F07F0F12
:10EEF00006D1D878FFF7E2FE084B1B681B6A9847DB
:10EF0000074B1B689B6898470823034A12681372D3
:10EF1000FFF7F8FE08BD00BF200D0020DC0C00202C
:10EF2000B80C002038B5324B1B68187810F07F0001
:10EF300004D15A7A22F020025A7258E0022855D1A0
:10EF40005A88002A52D11A79002A4FD15A7912F0E0
:10EF5000800F22F0800405D0264951F8241001F0DA
:10EF6000300104E0234951F8241001F440512248B3
:10EF7000007884423AD2002938D09B7A002B35D0D1
:10EF800012F0800F0FD01B4B53F8243003F03003E6
:10EF9000102B25D1E4B2204600F082FC204630211F
:10EFA00000F05EFB1CE0134D55F8243003F4405391
:10EFB000B3F5805F14D134B9104B204693F82C1070
:10EFC00000F0F6FC02E0204600F056FC55F8242044
:10EFD0004BF68F7302EA030383F4405345F8243061
:10EFE000074B1B685B699847002000E0022038BD92
:10EFF000200D0020005C0040040100208000002063
:10F00000DC0C0020F7B58D4B8D4E1A6835688D4BA2
:10F0100092B2D3182A7A5B00092A1B681BD09BB2D4
:10F0200003F1005303F540535B001C4614F8012B19
:10F0300003F10A072A705B786B70B4F8030000F0E4
:10F0400063FE6880B4F80700346800F05DFEA080BD
:10F0500033687F88DF807A4C01212368DA8819724F
:10F060005D78002A62D11A7812F07F022ED1092D24
:10F0700002D1FFF715FD3BE0052D0DD193F90320DB
:10F08000002A4EDB9A78002A4BD19A88002A48D170
:10F090009B7A002B37D044E0032D0BD1DA78012A7C
:10F0A00027D19A882ABB5B7A13F0200F21D0FFF773
:10F0B000E5FD1DE0012D1CD1DA78012A19D19A88CD
:10F0C000BAB95B7A13F0200F13D00AE0012A04D1F9
:10F0D0000B2D0ED1FFF714FD0AE0022A09D1012DF4
:10F0E00002D1FFF71FFF03E0032D02D1FFF780FDE0
:10F0F00048B1554B28461B685B699847032801D1E6
:10F1000009230FE068B94D4A504B12684FF03001A7
:10F1100092B2D3185B0000221A604D4B198006236F
:10F1200000E00823464A12681372E3E0062D18D166
:10F130001A7812F07F0F40F097809B78012B03D153
:10F14000414B1B68DB696EE0022B03D13E4B1B6811
:10F150001B6A68E0032B40F087803B4B1B685B6AAF
:10F1600061E0002D3CD1598800297DD15A6822F4F4
:10F170007F42B2F5003F77D11A7812F07F0203D1B7
:10F180009B88002B70D129E0012A0BD158792E4B96
:10F190001B689B699847002866D123689B7A002BDF
:10F1A00062D01BE0022A5FD15B7913F0800F03F07D
:10F1B0000F0205D0274951F8221001F0300104E078
:10F1C000244951F8221001F440512348007882422A
:10F1D0004AD213F0700F47D1002945D01F4B23E0CE
:10F1E000082D05D11B7813F07F0F3DD11C4B1BE080
:10F1F0000A2D39D11A7802F07F02012A34D19A7A85
:10F20000002A31D0598800292ED15A6822F47F4231
:10F21000B2F5803F28D158790B4B1B689B69984702
:10F2200010BB104B00E0FBB1054A4FF00001126823
:10F230000020936151829847002020E0505C0040FC
:10F24000200D002004300020B80C002002300020E7
:10F25000840D0020005C00400401002049EB000800
:10F2600079EA0008D9EA0008244C254B22681B687B
:10F2700050781B699847032801D1236806E01F4B8B
:10F280004FF6FF711B681A8A8A4201D1092203E0F6
:10F29000022800D012B908221A722BE093F900104C
:10F2A000002921DAD98801910198824202D9019A74
:10F2B0001A8211E08A420FD21149096891F82C1084
:10F2C0008A4201D2002105E092FBF1F001FB1022FD
:10F2D00012B901210B4A1170094A126892F82C20C8
:10F2E0009A82FFF799FD05E003221A72064B4FF44C
:10F2F00040521A80FFF706FDFEBD00BF200D002022
:10F30000B80C0020E4060020820D0020074A0221EC
:10F3100008B5074811720749074B086007490A609A
:10F32000074A13601B68984708BD00BFC00C002047
:10F3300008010020DC0C002080000020200D0020AF
:10F34000B80C002008B529E047F6FF70086019885E
:10F3500001F00F018B0003F18043117003F5B843F6
:10F36000196889B211F4004F09D0186840F68F71FE
:10F3700000EA0101196012780E4B013A0BE011F01E
:10F38000800F0BD0186848F60F7100EA0101196070
:10F390001278094B013A53F8223098470749084B35
:10F3A0000868084A80B21880188800B20028CBDBB1
:10F3B00008BD00BFE8000020CC000020445C0040F5
:10F3C000B60C0020BC0C0020F8B59AE047F6FF769A
:10F3D0001E601688564F06F00F06B30003F18043F7
:10F3E00003F5B8433E70002E64D127682668236871
:10F3F00007F4405C03EA000080F4005020602368BA
:10F4000006F0300003EA010181F020012160138839
:10F41000484A13F0100F1080A5F800C004D02368EC
:10F420009BB213F0800F08D0226848F60F7302EAEF
:10F4300003032360FFF746FD16E013F4006F08D0C6
:10F44000226840F68F7302EA03032360FFF7DAFDB8
:10F450000AE013F4004F54D0226840F68F7302EA9A
:10F4600003032360FFF770FC21682A884BF68F7333
:10F4700001EA030312F4805F18BF83F4805312F48F
:10F48000005F2D4A18BF83F400531360294B1168A5
:10F490001A8848F6BF7301EA030312F0100F18BF71
:10F4A00083F0100312F0200F234A18BF83F02003CB
:10F4B00013603BE01C68A4B214F4004F0BD0196831
:10F4C00040F68F7201EA02021A603A781B4B013A49
:10F4D00053F82230984714F0800F12D0144948F6A0
:10F4E0000F720B789B0003F1804303F5B843186853
:10F4F00000EA02021A600A78114B013A53F82230EE
:10F500009847104B104A1D680B4C1FFA85FCA2F857
:10F5100000C0B2F800C04BF68F700FFA8CFCBCF143
:10F52000000F48F6BF71094DFFF650AFF8BD00BFA0
:10F53000BC0C0020840D0020005C0040E80000208E
:10F54000CC000020445C0040B60C0020820D00205E
:10F5500001F10051013201F5405110B54900520846
:10F56000002308E010F803C06478013A4CEA042C48
:10F5700021F813C00233C418002AF3D110BD00BF14
:10F5800001F10051013201F5405110B54900520816
:10F59000002304E031F81340013AC4520233002A38
:10F5A000F8D110BD014B1860704700BF405C0040AF
:10F5B000014B186880B27047405C0040014B1860F6
:10F5C000704700BF445C0040014B186880B2704730
:10F5D000445C0040014B186880B27047485C0040B2
:10F5E000014B1860704700BF4C5C0040014B18682D
:10F5F00080B270474C5C00404FF6F873024A00EA54
:10F6000003031360704700BF505C0040014B186853
:10F6100080B27047505C0040014B43F820107047A7
:10F62000005C0040024B53F8200080B2704700BFDE
:10F63000005C0040054B10B553F8204048F68F128F
:10F6400004EA02020A4343F8202010BD005C004097
:10F65000024B53F8200000F4C0607047005C00408B
:10F660000A4B10B553F8202048F6BF7402EA040490
:10F6700011F0100F18BF84F0100411F0200F18BF04
:10F6800084F0200443F8204010BD00BF005C00401F
:10F690000A4B10B553F820204BF68F7402EA04048D
:10F6A00011F4805F18BF84F4805411F4005F18BF18
:10F6B00084F4005443F8204010BD00BF005C0040BB
:10F6C00038B50D460446FFF7ADFF012D02D120F4F9
:10F6D000805003E0022D04D120F01000014B43F8CC
:10F6E000240038BD005C0040024B53F8200000F0BD
:10F6F00030007047005C0040024B53F8200000F4DB
:10F7000040507047005C0040054B48F6BF7253F80C
:10F71000201001EA020282F0300243F820207047F4
:10F72000005C0040054B4BF68F7253F8201001EA45
:10F73000020282F4405243F820207047005C0040EF
:10F74000054B48F68F6253F8201001EA020242F49A
:10F75000807243F820207047005C0040044B48F65C
:10F760008F6253F8201001EA020243F8202070470C
:10F77000005C0040044B48F68F6253F8201001EA09
:10F78000020243F820207047005C0040054B48F619
:10F790008F6253F8201001EA020242F4807243F8AB
:10F7A00020207047005C0040054B48F68F6253F8FC
:10F7B000201001EA020242F4807243F820207047D0
:10F7C000005C0040044B48F68F6253F8201001EAB9
:10F7D000020243F820207047005C0040044B53F8BD
:10F7E000200000F03000102814BF002001207047D6
:10F7F000005C0040054B53F8200000F44050B0F589
:10F80000805F14BF00200120704700BF005C0040F3
:10F81000044B40F68F7253F8201001EA020243F8BD
:10F8200020207047005C0040044B48F60F7253F8EC
:10F83000201001EA020243F820207047005C0040DB
:10F84000054B48F68F7253F8201001EA020242F489
:10F85000804243F820207047005C0040054B48F68A
:10F860008F7253F8201001EA020242F0400243F87E
:10F8700020207047005C0040084B53F8202012F411
:10F88000804F09D053F8201048F68F7201EA020227
:10F8900042F4804243F82020704700BF005C0040E3
:10F8A000084B53F8202012F0400F09D053F82010D5
:10F8B00048F68F7201EA020242F0400243F820202B
:10F8C000704700BF005C0040054B10B553F8204066
:10F8D00048F68F7204EA02020A4343F8202010BD62
:10F8E000005C0040024B53F8200000F00F0070470E
:10F8F000005C0040064B49081B6849009BB203EBC3
:10F90000C00303F1005303F540535B0019607047D7
:10F91000505C0040054A064B1268490892B202EB5F
:10F92000C002D3185B00490019607047505C00406A
:10F9300004300020054B1B689BB203EBC00303F1AE
:10F94000005303F540535B0018887047505C00403B
:10F95000044A054B126892B202EBC002D3185B0056
:10F9600018887047505C004004300020044A054B62
:10F97000126892B202EBC002D3185B0019607047A4
:10F98000505C0040023000203E2909D94B0911F09B
:10F990001F0F01D1013B9BB29B0243F4004305E0E2
:10F9A0004B0811F0010F18BF01339B020360704731
:10F9B0000D4A0E4B126892B2D31803EBC0035B00E2
:10F9C0003E2909D94A0911F01F0F01D1013A92B21B
:10F9D000920242F4004205E04A0811F0010F18BFFC
:10F9E000013292021A607047505C004006300020DD
:10F9F000054A064B126892B202EBC002D3185B00B4
:10FA000018688005800D7047505C0040023000206F
:10FA1000054A064B126892B202EBC002D3185B0093
:10FA200018688005800D7047505C0040063000204B
:10FA30000C4B30B51D681C68C0001FFA85FC84445F
:10FA4000A4B2094B00190CF1005CC3180CF5405C22
:10FA5000490852084FEA4C0049005B00520001601F
:10FA60001A6030BD505C004004300020064B49084D
:10FA70001B6849009BB203EBC00303F1005303F57D
:10FA800040535B0019607047505C0040054A064BCC
:10FA90001268490892B202EBC002D3185B00490019
:10FAA00019607047505C004004300020054B1B6813
:10FAB0009BB203EBC00303F1005303F540535B001B
:10FAC00018887047505C0040044A054B126892B297
:10FAD00002EBC002D3185B0018887047505C0040EE
:10FAE00004300020012910B524D1254B25491B687D
:10FAF000C0009BB2591809184B003E2A09D9510978
:10FB000012F01F0F01D1013989B2890241F400417D
:10FB100005E0510812F0010F18BF01318902196088
:10FB20001749194B096889B2CB18181840003E2AAA
:10FB30001ED913E0022922D1114BC0001C681B689A
:10FB4000A4B21FFA83FC0F490F4B844400194118DB
:10FB5000634449005B000A601A6010E0530912F028
:10FB60001F0F01D1013B9BB29B0243F4004305E010
:10FB7000530812F0010F18BF01339B02036010BD40
:10FB8000505C0040023000200630002001291BD1CB
:10FB90001349144B096889B2CB1803EBC00040002D
:10FBA0003E2A09D9530912F01F0F01D1013B9BB224
:10FBB0009B0243F4004305E0530812F0010F18BF05
:10FBC00001339B0203600AE0022908D10449054B76
:10FBD000096889B201EBC000C3185B001A60704766
:10FBE000505C00400230002001291BD11349144B06
:10FBF000096889B2CB1803EBC00040003E2A09D93E
:10FC0000530912F01F0F01D1013B9BB29B0243F439
:10FC1000004305E0530812F0010F18BF01339B02A7
:10FC200003600AE0022908D10449054B096889B23A
:10FC300001EBC000C3185B001A607047505C0040C5
:10FC400006300020054A064B126892B202EBC00251
:10FC5000D3185B0018688005800D7047505C004029
:10FC600002300020054A064B126892B202EBC00235
:10FC7000D3185B0018688005800D7047505C004009
:10FC8000063000200D4BC00019680D4A89B241189A
:10FC90008A185200128812F47C4F01D001200CE027
:10FCA0001A68084B92B28018C3185B001888800548
:10FCB000800D002814BF022000207047505C0040D7
:10FCC0000630002002300020012909D10B4A48F6F5
:10FCD0008F7352F8201001EA030343F040030AE057
:10FCE00002290AD1054A48F68F7352F8201001EA1A
:10FCF000030343F4804342F820307047005C004027
:10FD000041EA0020704700BF030AC0B243EA002066
:10FD1000704700BF08B500220A2300F045F808BD6F
:10FD200008B500210A2200F0DFF808BDF0B403781E
:10FD3000002B2DD040F23412C2F20002156802E00E
:10FD400010F8013FEBB15A1903F12004527812F078
:10FD500001070A7808BF1C4601F10101561C9446B0
:10FD6000AE5D16F0010F18BF02F1200C6445E7D01C
:10FD700007B1203316F0010F18BF2032981AF0BCDB
:10FD800070470A786F78561C07F00107AE5DEFE701
:10FD900040F234100A78C2F20000561C05686F78F1
:10FDA000AE5D07F00107E3E72DE9F04F40F23415AF
:10FDB000C2F2000583B00C461F46D5F800800E46FF
:10FDC0000190009216F8015B08EB050393F801B06F
:10FDD0001BF0080BF6D12D2D65D02B2D08BF16F882
:10FDE000015BD7F1010338BF0023102F14BF1A465F
:10FDF00043F0010232B1302D66D01BB1302D0CBF63
:10FE000008270A27BBF1000F394614BF4FF00049FD
:10FE10006FF00049484600F059FC48468A4639468A
:10FE200000F026FB00218C4608EB0502A5F130030B
:10FE3000527812F0040F08D112F0030F20D012F004
:10FE4000010F14BF37235723EB1A9F4218DD844557
:10FE500094BF0022012252EAD1714FF0FF310CD140
:10FE6000844514BF002201225345D4BF002202F072
:10FE7000010212B907FB0C3C012116F8015BD3E724
:10FE8000B1F1FF3F14D0BBF1000F09D16046009BD8
:10FE90001BB101B1741E009A146003B0BDE8F08F6D
:10FEA000CCF10000F3E716F8015B4FF0010B98E787
:10FEB000019ABBF1000F4FF0220314BF4FF0004036
:10FEC0006FF000401360E2E73278782A14BF002117
:10FED0000121582A14BF0A4641F00102002A8CD0A1
:10FEE0007578102702368DE710B540F23814C2F24B
:10FEF00000048C461346014662462068FFF754FF13
:10FF000010BD00BF2DE9F0438BB006460F4600F050
:10FF10007BF840F22C24C2F2000494F90030B3F1D3
:10FF2000FF3F8046894638D03046394600F084FA93
:10FF30000546002831D1304639460022002301F021
:10FF40001DF8002829D1247842F28803C0F6010365
:10FF500008950193CDE90267CDE90467002C21D013
:10FF600040F200030022CFF6F0733046CDE90623BD
:10FF700039460022002300F0D9FF002822D00223B6
:10FF800000939C4234D0684600F064FA00282FD0D9
:10FF9000089B002B27D1DDE90689404649460BB076
:10FFA000BDE8F0834FF6FF734FF06042CCF2EF7381
:10FFB0003046CDE9062339460022002300F0B6FF83
:10FFC0000028DCD10123022C009316D0684600F0F3
:10FFD00041FA90B142F28C00C0F6010000F03CFA08
:10FFE000CDE90601D4E700F03DFA089B0360D2E7B3
:10FFF00000F038FA22230360CAE700F033FA212325
:020000040801F1
:100000000360E7E700000000B1F5801F0B462DE913
:10001000F04F804687B0894604460D463EDB4FF6DA
:10002000FF720026C7F6EF72934251DC23F07F4443
:1000300045F6647C24F47004C0F2090CA44440F238
:100040000002A6F57E760CF4801C073EC3F6F07223
:100050008CEA020206EB235640F20003404642EAD5
:100060000401C3F6F073002206EB1C5600F042FBBD
:10007000A31C23F07F4323F47003022B80468946A0
:100080002FDC0022002300F051FF002800F0CA807E
:10009000002E40F07C81002000211FE021F0004371
:1000A000034300F0B5800029C0F2468140F200030E
:1000B0000022C4F250336FF0350600F0CFFC4FF64B
:1000C000FF72C7F6EF720B46804693428946ADDD5C
:1000D0004046494642464B4600F00EFB07B0BDE89D
:1000E000F08F00224FF0804300F006FB4EF686357D
:1000F000CFF6F975651902460B464046494600F0B1
:10010000D7FDCDE90201304600F042FCCDE9040103
:10011000DDE9020102460B4600F0A0FC02460B4658
:10012000CDE9000100F09AFCA7A3D3E900238246A1
:100130008B4600F093FCA6A3D3E9002300F0DCFA81
:1001400052465B4600F08AFCA3A3D3E9002300F0EB
:10015000D3FA52465B4600F081FCA1A3D3E9002309
:1001600000F0CAFADDE9002300F078FC9EA3D3E991
:100170000023CDE900015046594600F06FFC9CA3D6
:10018000D3E9002300F0B8FA52465B4600F066FC63
:1001900099A3D3E9002300F0AFFA52465B4600F082
:1001A0005DFC0B460246DDE9000100F0A5FA4BF6C6
:1001B0005103C0F206031B1B43EA0505002D8246CE
:1001C0008B4656DD40F200030022C3F6E073404642
:1001D000494600F043FC42464B4600F03FFC0446D3
:1001E0000D46002E75D152465B4600F085FADDE9DA
:1001F000022300F033FC02460B462046294600F05D
:1002000079FA02460B464046494600F073FA65E724
:1002100040F20001002000220023CCF2503100F017
:1002200047FD5BE742464B464046494600F016FC18
:1002300073A3D3E9002304460D464046494600F027
:100240000DFC40F200030022C3F6E07300F054FA04
:1002500002460B462046294600F000FC04460D46A7
:10026000002E72D14046494622462B4600F042FA03
:1002700034E7002E00F0D48063A3D3E90023DDE946
:10028000040100F0EBFB52465B4606460F46404633
:10029000494600F02FFADDE9022300F0DFFB5CA302
:1002A000D3E9002304460D46DDE9040100F0D6FB46
:1002B00002460B462046294600F01EFA42464B46AF
:1002C00000F018FA02460B463046394600F012FAA2
:1002D00004E74DA3D3E90023DDE9040100F0BEFBF0
:1002E00052465B46CDE900012046294600F004FA5B
:1002F000DDE9022300F0B2FB47A3D3E90023064661
:100300000F46DDE9040100F0A9FB02460B4630462A
:10031000394600F0F1F902460B462046294600F026
:10032000E9F942464B4600F0E5F902460B46DDE9A5
:10033000000100F0DFF9D1E602460B4600F0DAF9E1
:100340000022002300F0B4FCC8E6304600F020FB99
:100350002DA3D3E9002306460F4600F07FFB2CA314
:10036000D3E9002382468B463046394600F076FBBF
:1003700022462B4600F0C0F942464B4600F0BAF93F
:1003800002460B465046594600F0B4F9A6E6304600
:1003900000F0FEFA1CA3D3E9002306460F4600F046
:1003A0005DFB1DA3D3E9002304460D4630463946C4
:1003B00000F054FB02460B462046294600F09CF90B
:1003C0008CE600BFAFF3008044523EDF12F1C23F23
:1003D000DE03CB966446C73F599322942449D23F0B
:1003E000935555555555E53F9FC678D0099AC33F5B
:1003F000AF788E1DC571CC3F04FA97999999D93F72
:10040000555555555555D5BF0000E0FE422EE63FE7
:10041000763C7935EF39EABD763C7935EF39EA3DFE
:1004200002460B464046494600F064F9DDE90223E6
:1004300000F014FBE5E600BF02464042104321F005
:10044000004141EAD070C0F1FE4000F57000C00FDD
:10045000704700BF0020704740F200010020C7F63F
:10046000F871704740F23813C2F200031868704701
:100470004A1E08BF7047C0F02481884240F21681AE
:10048000114200F01781B0FA80F3B1FA81F2A2EBC9
:100490000303C3F11F0304A202EB03134FF0000296
:1004A0009F4600BFAFF30080B0EBC17F00BF42EBBF
:1004B000020228BFA0EBC170B0EB817F00BF42EB0E
:1004C000020228BFA0EB8170B0EB417F00BF42EB7E
:1004D000020228BFA0EB4170B0EB017F00BF42EBEE
:1004E000020228BFA0EB0170B0EBC16F00BF42EB6E
:1004F000020228BFA0EBC160B0EB816F00BF42EBEE
:10050000020228BFA0EB8160B0EB416F00BF42EB5D
:10051000020228BFA0EB4160B0EB016F00BF42EBCD
:10052000020228BFA0EB0160B0EBC15F00BF42EB4D
:10053000020228BFA0EBC150B0EB815F00BF42EBCD
:10054000020228BFA0EB8150B0EB415F00BF42EB3D
:10055000020228BFA0EB4150B0EB015F00BF42EBAD
:10056000020228BFA0EB0150B0EBC14F00BF42EB2D
:10057000020228BFA0EBC140B0EB814F00BF42EBAD
:10058000020228BFA0EB8140B0EB414F00BF42EB1D
:10059000020228BFA0EB4140B0EB014F00BF42EB8D
:1005A000020228BFA0EB0140B0EBC13F00BF42EB0D
:1005B000020228BFA0EBC130B0EB813F00BF42EB8D
:1005C000020228BFA0EB8130B0EB413F00BF42EBFD
:1005D000020228BFA0EB4130B0EB013F00BF42EB6D
:1005E000020228BFA0EB0130B0EBC12F00BF42EBED
:1005F000020228BFA0EBC120B0EB812F00BF42EB6D
:10060000020228BFA0EB8120B0EB412F00BF42EBDC
:10061000020228BFA0EB4120B0EB012F00BF42EB4C
:10062000020228BFA0EB0120B0EBC11F00BF42EBCC
:10063000020228BFA0EBC110B0EB811F00BF42EB4C
:10064000020228BFA0EB8110B0EB411F00BF42EBBC
:10065000020228BFA0EB4110B0EB011F00BF42EB2C
:10066000020228BFA0EB0110B0EBC10F00BF42EBAC
:10067000020228BFA0EBC100B0EB810F00BF42EB2C
:10068000020228BFA0EB8100B0EB410F00BF42EB9C
:10069000020228BFA0EB4100B0EB010F00BF42EB0C
:1006A000020228BFA0EB0100104670470CBF0120DA
:1006B00000207047B1FA81F2C2F11F0220FA02F065
:1006C000704708B14FF0FF3000F00EB80029F8D0A5
:1006D0002DE90340FFF7CCFEBDE8064002FB00F326
:1006E000A1EB0301704700BF704700BF81F00041DC
:1006F00002E000BF83F0004330B54FEA41044FEA07
:10070000430594EA050F08BF90EA020F1FBF54EAA1
:10071000000C55EA020C7FEA645C7FEA655C00F03D
:10072000E2804FEA5454D4EB5555B8BF6D420CDD0E
:100730002C4480EA020281EA030382EA000083EA91
:10074000010180EA020281EA0303362D88BF30BD31
:1007500011F0004F4FEA01314FF4801C4CEA113187
:1007600002D0404261EB410113F0004F4FEA0333E6
:100770004CEA133302D0524263EB430394EA050F71
:1007800000F0A780A4F10104D5F1200E0DDB02FAE0
:100790000EFC22FA05F2801841F1000103FA0EF274
:1007A000801843FA05F359410EE0A5F120050EF13A
:1007B000200E012A03FA0EFC28BF4CF0020C43FA6B
:1007C00005F3C01851EBE37101F0004507D54FF078
:1007D000000EDCF1000C7EEB00006EEB0101B1F5C8
:1007E000801F1BD3B1F5001F0CD349085FEA30000E
:1007F0004FEA3C0C04F101044FEA445212F5800F19
:1008000080F09A80BCF1004F08BF5FEA500C50F1B5
:10081000000041EB045141EA050130BD5FEA4C0C98
:10082000404141EB010111F4801FA4F10104E9D121
:1008300091F0000F04BF01460020B1FA81F308BF18
:100840002033A3F10B03B3F120020CDA0C3208DDE4
:1008500002F1140CC2F10C0201FA0CF021FA02F1BF
:100860000CE002F11402D8BFC2F1200C01FA02F12F
:1008700020FA0CFCDCBF41EA0C019040E41AA2BF54
:1008800001EB0451294330BD6FEA04041F3C1CDA1C
:100890000C340EDC04F11404C4F1200220FA04F03C
:1008A00001FA02F340EA030021FA04F345EA0301E6
:1008B00030BDC4F10C04C4F1200220FA02F001FAA8
:1008C00004F340EA0300294630BD21FA04F029462A
:1008D00030BD94F0000F83F4801306BF81F48011C3
:1008E0000134013D4EE77FEA645C18BF7FEA655C36
:1008F00029D094EA050F08BF90EA020F05D054EA08
:10090000000C04BF1946104630BD91EA030F1EBF0C
:100910000021002030BD5FEA545C05D14000494110
:1009200028BF41F0004130BD14F580043CBF01F503
:10093000801130BD01F0004545F0FE4141F47001E9
:100940004FF0000030BD7FEA645C1ABF19461046C4
:100950007FEA655C1CBF0B46024650EA013406BFC5
:1009600052EA033591EA030F41F4002130BD00BF84
:1009700090F0000F04BF0021704730B54FF4806441
:1009800004F132044FF000054FF0000150E700BFC2
:1009900090F0000F04BF0021704730B54FF4806421
:1009A00004F1320410F0004548BF40424FF000010E
:1009B0003EE700BF42004FEAE2014FEA31014FEA51
:1009C00002701FBF12F07F4393F07F4F81F06051A0
:1009D000704792F0000F14BF93F07F4F704730B50F
:1009E0004FF4607401F0004521F0004120E700BFA2
:1009F00050EA010208BF704730B54FF000050AE029
:100A000050EA010208BF704730B511F0004502D529
:100A1000404261EB41014FF4806404F132045FEA2B
:100A2000915C3FF4DCAE4FF003025FEADC0C18BFD0
:100A300003325FEADC0C18BF033202EBDC02C2F1C6
:100A4000200300FA03FC20FA02F001FA03FE40EA58
:100A50000E0021FA02F11444C1E600BF70B54FF058
:100A6000FF0C4CF4E06C1CEA11541DBF1CEA13553A
:100A700094EA0C0F95EA0C0F00F0DEF82C4481EAA2
:100A8000030621EA4C5123EA4C5350EA013518BFC2
:100A900052EA033541F4801143F4801338D0A0FBAF
:100AA00002CE4FF00005E1FB02E506F00042E0FB5C
:100AB00003E54FF00006E1FB03569CF0000F18BF62
:100AC0004EF0010EA4F1FF04B6F5007F64F540740A
:100AD00004D25FEA4E0E6D4146EB060642EAC6219D
:100AE00041EA55514FEAC52040EA5E504FEACE2E0A
:100AF000B4F1FD0C88BFBCF5E06F1ED8BEF1004F0D
:100B000008BF5FEA500E50F1000041EB045170BD88
:100B100006F0004646EA010140EA020081EA0301CC
:100B2000B4EB5C04C2BFD4EB0C0541EA045170BDC8
:100B300041F480114FF0000E013C00F3AB8014F142
:100B4000360FDEBF002001F0004170BDC4F100048B
:100B5000203C35DA0C341BDC04F11404C4F120050C
:100B600000FA05F320FA04F001FA05F240EA020067
:100B700001F0004221F0004110EBD37021FA04F69D
:100B800042EB06015EEA430E08BF20EAD37070BD57
:100B9000C4F10C04C4F1200500FA04F320FA05F0B6
:100BA00001FA04F240EA020001F0004110EBD370B8
:100BB00041F100015EEA430E08BF20EAD37070BD28
:100BC000C4F1200500FA05F24EEA020E20FA04F301
:100BD00001FA05F243EA020321FA04F001F00041B0
:100BE00021FA04F220EA020000EBD3705EEA430E21
:100BF00008BF20EAD37070BD94F0000F0FD101F050
:100C00000046400041EB010111F4801F08BF013C88
:100C1000F7D041EA060195F0000F18BF704703F0C6
:100C20000046520043EB030313F4801F08BF013D4D
:100C3000F7D043EA0603704794EA0C0F0CEA135509
:100C400018BF95EA0C0F0CD050EA410618BF52EAC3
:100C50004306D1D181EA030101F000414FF00000C9
:100C600070BD50EA410606BF1046194652EA4306D7
:100C700019D094EA0C0F02D150EA013613D195EA4B
:100C80000C0F05D152EA03361CBF104619460AD193
:100C900081EA030101F0004141F0FE4141F470019D
:100CA0004FF0000070BD41F0FE4141F4780170BD8D
:100CB00070B54FF0FF0C4CF4E06C1CEA11541DBFF2
:100CC0001CEA135594EA0C0F95EA0C0F00F0A7F8F4
:100CD000A4EB050481EA030E52EA03354FEA013121
:100CE00000F088804FEA03334FF0805545EA131334
:100CF00043EA12634FEA022245EA111545EA1065FC
:100D00004FEA00260EF000419D4208BF964244F192
:100D1000FD0404F5407402D25B084FEA3202B61AB1
:100D200065EB03055B084FEA32024FF480104FF485
:100D3000002CB6EB020E75EB030E22BFB61A7546F9
:100D400040EA0C005B084FEA3202B6EB020E75EB8C
:100D5000030E22BFB61A754640EA5C005B084FEAF4
:100D60003202B6EB020E75EB030E22BFB61A7546C1
:100D700040EA9C005B084FEA3202B6EB020E75EBCC
:100D8000030E22BFB61A754640EADC0055EA060E8D
:100D900018D04FEA051545EA16754FEA06164FEAD0
:100DA000C30343EA52734FEAC2025FEA1C1CC0D17C
:100DB00011F4801F0BD141EA00014FF000004FF009
:100DC000004CB6E711F4801F04BF01430020B4F1CA
:100DD000FD0C88BFBCF5E06F3FF6AFAEB5EB030C82
:100DE00004BFB6EB020C5FEA500C50F1000041EB7F
:100DF000045170BD0EF0004E4EEA113114EB5C044C
:100E0000C2BFD4EB0C0541EA045170BD41F480111E
:100E10004FF0000E013C90E645EA060E8DE60CEA26
:100E2000135594EA0C0F08BF95EA0C0F3FF43BAF43
:100E300094EA0C0F0AD150EA01347FF434AF95EAFA
:100E40000C0F7FF425AF104619462CE795EA0C0FDE
:100E500006D152EA03353FF4FDAE1046194622E7AB
:100E600050EA410618BF52EA43067FF4C5AE50EA85
:100E700041047FF40DAF52EA43057FF4EBAE12E775
:100E80004FF0FF3C06E000BF4FF0010C02E000BF56
:100E90004FF0010C4DF804CD4FEA410C7FEA6C5C39
:100EA0004FEA430C18BF7FEA6C5C1BD001B050EADC
:100EB000410C0CBF52EA430C91EA030F02BF90EAC7
:100EC000020F0020704710F1000F91EA030F58BF86
:100ED000994208BF90422CBFD8176FEAE37040F0E8
:100EE000010070474FEA410C7FEA6C5C02D150EA86
:100EF000013C07D14FEA430C7FEA6C5CD6D152EA41
:100F0000033CD3D05DF8040B704700BF8446104605
:100F100062468C461946634600E000BF01B5FFF704
:100F2000B7FF002848BF10F1000F01BD4DF808EDD4
:100F3000FFF7F4FF0CBF012000205DF808FB00BFA5
:100F40004DF808EDFFF7EAFF34BF012000205DF8FF
:100F500008FB00BF4DF808EDFFF7E0FF94BF01204C
:100F600000205DF808FB00BF4DF808EDFFF7CEFF4D
:100F700094BF012000205DF808FB00BF4DF808ED8C
:100F8000FFF7C4FF34BF012000205DF808FB00BF5D
:100F90004FEA410212F5001215D211D56FF47873A1
:100FA000B3EB625212D94FEAC12343F0004343EA44
:100FB000505311F0004F23FA02F018BF404270471F
:100FC0004FF00000704750EA013005D111F00040A9
:100FD00008BF6FF0004070474FF00000704700BF3F
:100FE0004FEA4102B2F1E04324BFB3F5001CDCF14B
:100FF000FE5C0DD901F0004C4FEAC0024CEA507083
:10100000B2F1004F40EB830008BF20F001007047B1
:1010100011F0804F21D113F13872BCBF01F00040B4
:10102000704741F480114FEA5252C2F11802C2F1E6
:10103000200C10FA0CF320FA02F018BF40F0010067
:101040004FEAC1234FEAD32303FA0CFC40EA0C0019
:1010500023FA02F34FEA4303CCE77FEA625307D156
:1010600050EA01331EBF4FF0FE4040F4400070478D
:1010700001F0004040F0FE4040F40000704700BF27
:1010800080F0004002E000BF81F0004142001FBF3D
:101090005FEA410392EA030F7FEA226C7FEA236C46
:1010A0006AD04FEA1262D2EB1363C1BFD21841403B
:1010B00048404140B8BF5B42192B88BF704710F0D1
:1010C000004F40F4000020F07F4018BF404211F074
:1010D000004F41F4000121F07F4118BF494292EADC
:1010E000030F3FD0A2F1010241FA03FC10EB0C0008
:1010F000C3F1200301FA03F100F0004302D5494295
:1011000060EB4000B0F5000F13D3B0F1807F06D341
:1011100040084FEA310102F10102FE2A51D2B1F139
:10112000004F40EBC25008BF20F0010040EA03002E
:101130007047490040EB000010F4000FA2F10102DB
:10114000EDD1B0FA80FCACF1080CB2EB0C0200FA65
:101150000CF0AABF00EBC25052421843BCBFD040B3
:101160001843704792F0000F81F4000106BF80F42D
:1011700000000132013BB5E74FEA41037FEA226CF0
:1011800018BF7FEA236C21D092EA030F04D092F0BB
:10119000000F08BF0846704790EA010F1CBF0020EF
:1011A000704712F07F4F04D1400028BF40F000404C
:1011B000704712F100723CBF00F50000704700F06C
:1011C000004343F0FE4040F4000070477FEA226293
:1011D00016BF08467FEA23630146420206BF5FEA64
:1011E000412390EA010F40F4800070474FF0000364
:1011F00004E000BF10F0004348BF40425FEA000C2B
:1012000008BF704743F0964301464FF000001CE0D2
:1012100050EA010208BF70474FF000030AE000BF28
:1012200050EA010208BF704711F0004302D5404266
:1012300061EB41015FEA010C02BF844601460020D8
:1012400043F0B64308BFA3F18053A3F50003BCFAF3
:101250008CF2083AA3EBC25310DB01FA02FC6344A0
:1012600000FA02FCC2F12002BCF1004F20FA02F2A7
:1012700043EB020008BF20F00100704702F120029A
:1012800001FA02FCC2F1200250EA4C0021FA02F2FB
:1012900043EB020008BF20EADC7070474FF0FF0C00
:1012A0001CEAD0521EBF1CEAD15392EA0C0F93EAFB
:1012B0000C0F6FD01A4480EA010C400218BF5FEA9D
:1012C00041211ED04FF0006343EA501043EA511110
:1012D000A0FB01310CF00040B1F5000F3EBF49000A
:1012E00041EAD3715B0040EA010062F17F02FD2A0E
:1012F0001DD8B3F1004F40EBC25008BF20F00100F1
:10130000704790F0000F0CF0004C08BF49024CEA07
:10131000502040EA51207F3AC2BFD2F1FF0340EA99
:10132000C250704740F400004FF00003013A5DDC0A
:1013300012F1190FDCBF00F000407047C2F100024B
:10134000410021FA02F1C2F1200200FA02FC5FEA38
:10135000310040F1000053EA4C0308BF20EADC7082
:10136000704792F0000F00F0004C02BF400010F4F4
:10137000000F013AF9D040EA0C0093F0000F01F0A1
:10138000004C02BF490011F4000F013BF9D041EAC3
:101390000C018FE70CEAD15392EA0C0F18BF93EAC5
:1013A0000C0F0AD030F0004C18BF31F0004CD8D1EF
:1013B00080EA010000F00040704790F0000F17BF76
:1013C00090F0004F084691F0000F91F0004F14D0BC
:1013D00092EA0C0F01D142020FD193EA0C0F03D114
:1013E0004B0218BF084608D180EA010000F0004017
:1013F00040F0FE4040F40000704740F0FE4040F4F2
:10140000400070474FF0FF0C1CEAD0521EBF1CEA90
:10141000D15392EA0C0F93EA0C0F69D0A2EB0302AE
:1014200080EA010C49024FEA402037D04FF0805348
:1014300043EA111143EA10130CF000408B4238BF0D
:101440005B0042F17D024FF4000C8B4224BF5B1A1B
:1014500040EA0C00B3EB510F24BFA3EB510340EA69
:101460005C00B3EB910F24BFA3EB910340EA9C0017
:10147000B3EBD10F24BFA3EBD10340EADC001B0187
:1014800018BF5FEA1C1CE0D1FD2A3FF650AF8B422B
:1014900040EBC25008BF20F0010070470CF0004C38
:1014A0004CEA50207F32C2BFD2F1FF0340EAC25063
:1014B000704740F400004FF00003013A37E792F024
:1014C000000F00F0004C02BF400010F4000F013A82
:1014D000F9D040EA0C0093F0000F01F0004C02BF7D
:1014E000490011F4000F013BF9D041EA0C0195E7E6
:1014F0000CEAD15392EA0C0F08D142027FF47DAF7F
:1015000093EA0C0F7FF470AF084676E793EA0C0F6E
:1015100004D14B023FF44CAF08466EE730F0004C6C
:1015200018BF31F0004CCAD130F000427FF45CAFFC
:1015300031F000437FF43CAF5FE700BF4FF0FF3C6A
:1015400006E000BF4FF0010C02E000BF4FF0010CBD
:101550004DF804CD4FEA40024FEA41037FEA226C86
:1015600018BF7FEA236C11D001B052EA530C18BFA8
:1015700090EA010F58BFB2EB030088BFC81738BF0D
:101580006FEAE17018BF40F0010070477FEA226CFB
:1015900002D15FEA402C05D17FEA236CE4D15FEAF7
:1015A000412CE1D05DF8040B704700BF844608462B
:1015B0006146FFE70FB5FFF7C9FF002848BF10F1EC
:1015C000000F0FBD4DF808EDFFF7F4FF0CBF012031
:1015D00000205DF808FB00BF4DF808EDFFF7EAFFBB
:1015E00034BF012000205DF808FB00BF4DF808ED76
:1015F000FFF7E0FF94BF012000205DF808FB00BF6B
:101600004DF808EDFFF7D2FF94BF012000205DF8F0
:1016100008FB00BF4DF808EDFFF7C8FF34BF0120FD
:1016200000205DF808FB00BF42000ED2B2F1FE4F71
:101630000BD34FF09E03B3EB126209D44FEA0023A1
:1016400043F0004323FA02F070474FF00000704768
:1016500012F1610F01D1420202D14FF0FF30704709
:101660004FF00000704700BF73B96AB9002908BF86
:101670000028BCBF00204FF00041C4BF6FF0004104
:101680004FF0FF30FFF730B882B0EC462DE9005044
:1016900000F01CF8DDF804E002B00CBC704700BF9D
:1016A000F8B514461D4606460F4600F0D3F900FB78
:1016B00005F5A0FB042304FB0154E318B61A67EBFD
:1016C0000307069BC3E90067F8BD00BFF8B51446E1
:1016D0001D4606460F4600F00FF800FB05F5A0FB7F
:1016E000042304FB0154E318B61A67EB0307069BB7
:1016F000C3E90067F8BD00BF00292DE9F04F85B0B0
:10170000C0F2C9800026002BC0F2C0808946144672
:1017100005469B46002B4BD18A4258D9B2FA82F338
:1017200053B1C3F1200001FA03F925FA00F812FAC7
:1017300003F49D4048EA0909270C484639461FFA38
:1017400084FBFEF795FE394682464846FEF7BEFF0B
:101750004FEA15420BFB0AF342EA01494B4509D90E
:1017600019EB04090AF1FF3A04D24B4584BF0AF190
:10177000FF3AA144C3EB090939464846ADB2FEF72A
:1017800077FE394680464846FEF7A0FF0BFB08FB74
:1017900045EA0145AB4507D92D1908F1FF3803D2B9
:1017A000AB4588BF08F1FF3848EA0A48002703E044
:1017B0008B4257D90027B84642463B4616B15242A3
:1017C00063EB43031946104605B0BDE8F08F22B91C
:1017D00011460120FEF74CFE0446B4FA84F8B8F135
:1017E000000F5ED1C4EB0908270C1FFA84F9012110
:1017F000029139464046FEF73BFE39468246404656
:10180000FEF764FF4FEA154809FB0AF348EA014B6B
:101810005B4509D91BEB040B0AF1FF3A04D25B4587
:1018200084BF0AF1FF3AA344C3EB0B0B3946584679
:10183000ADB2FEF71DFE394680465846FEF746FF1C
:1018400009FB08F945EA0145A94507D92D1908F111
:10185000FF3803D2A94588BF08F1FF3848EA0A4893
:10186000029FA9E7B3FA83F7002F67D18B422CBF01
:101870004FF000094FF0010982428CBF4C4649F0FD
:101880000104002C96D04FF0010895E7524263EB1B
:101890004303F6433AE7404261EB41014FF0FF3624
:1018A00031E704FA08F4C8F1200735FA07F329FAFA
:1018B00007FA270C09FA08FB3946504643EA0B029F
:1018C0000292FEF7D5FD39461FFA84F98346504649
:1018D000FEF7FCFE029809FB0BF2030C43EA0143FE
:1018E0009A4204D91B190BF1FF3BC0F0AD809B1A43
:1018F000394618460193FEF7BBFD0199824608461A
:101900003946FEF7E3FE029809FB0AF31FFA80FC52
:101910004CEA0142934208D912190AF1FF3A04D263
:10192000934284BF0AF1FF3A121905FA08F54AEA10
:101930000B4EC3EB0208CDF808E05AE7C7F12000D0
:1019400003FA07FAC24035FA00F342EA0A0B21FA19
:1019500000F801FA07F940464FEA1B4A43EA090139
:10196000029151461FFA8BF20392FEF781FD514618
:1019700081464046FEF7AAFE0398029B00FB09F24F
:10198000180C14FA07F340EA0144A24204D914EBFC
:101990000B0409F1FF3951D3A41A51462046019393
:1019A000FEF766FD514680462046FEF78FFE039CFB
:1019B000019B04FB08F2029C1FFA84FC4CEA0140E4
:1019C000824204D910EB0B0008F1FF3830D348EA0B
:1019D00009481FFA83FC1B0C801A1FFA88FE4FEA85
:1019E000184A0CFB0EF90CFB0AF203FB0E2103FB59
:1019F0000AF301EB19418A4288BF03F5803303EBF8
:101A0000114E704510D31FFA89F905FA07F709EB53
:101A1000014014BF0022012287422CBF002702F0A0
:101A20000107002F3FF4C8AE08F1FF380027C3E6D6
:101A3000824284BF584408F1FF38C8E7A24284BFFD
:101A400009F1FF395C44A7E79A4284BF0BF1FF3BE1
:101A50001B194CE72DE9F04F0C4683B08046164623
:101A600089461F4615468A46002B4BD18A425CD9CF
:101A7000B2FA82F35BB1C3F1200001FA03FA28FA4B
:101A800000F216FA03F508FA03F842EA0A0A2E0CE5
:101A900050463146AFB2FEF7EBFC31464FEA1844F0
:101AA00081465046FEF712FE07FB09F344EA014A5D
:101AB000534509D91AEB050A09F1FF3904D25345F8
:101AC00084BF09F1FF39AA44C3EB0A0A31465046E4
:101AD0001FFA88F8FEF7CCFC314604465046FEF764
:101AE000F5FD07FB04F748EA0148474506D9013CE4
:101AF00018EB050802D2474588BF013C44EA094477
:101B000000265CE08B4258D8B3FA83F6002E5BD1F6
:101B10008B422CBF0022012285428CBF154642F029
:101B20000105002D49D0012449E022B911460120C8
:101B3000FEF79EFC0546B5FA85F6002E40F0BB8008
:101B4000641B2F0C1FFA85FA012639462046FEF742
:101B50008FFC39464FEA184B81462046FEF7B6FD0A
:101B60000AFB09F34BEA014B5B4509D91BEB050B5B
:101B700009F1FF3904D25B4584BF09F1FF39AB4459
:101B8000C3EB0B0B394658461FFA88F8FEF770FC7A
:101B9000394604465846FEF799FD0AFB04FA48EA1E
:101BA0000148C24506D9013C18EB050802D2C245DE
:101BB00088BF013C44EA094401E00026344631462E
:101BC000204603B0BDE8F08FC6F12000B34032FAE2
:101BD00000F721FA00FB1F4314FA06F228FA00F17D
:101BE00058464FEA174A114300915146BBB2019340
:101BF000FEF73EFC5146B54081465846FEF766FD6D
:101C0000019C009804FB09F34FEA104C4CEA014B8D
:101C10005B4505D91BEB070B09F1FF39C0F08F803D
:101C2000C3EB0B0B51465846FEF722FC51460446C7
:101C30005846FEF74BFD0198009A00FB04F31FFA8B
:101C400082FC4CEA0142934206D9013CD21903D2EC
:101C5000934201D9D219013C44EA0944A8B2D21AEC
:101C60002D0C1FFA84FC4FEA144300FB0CF700FB19
:101C700003FE05FB0CE105FB03F501EB17418E4567
:101C800088BF05F5803505EB1145AA4210D3BFB2D8
:101C900008FA06F607EB014214BF4FF0000E4FF0B2
:101CA000010E96422CBF00260EF00106002E86D0B3
:101CB000013C002683E7B540C6F1200124FA01F972
:101CC00028FA01F22F0CB4403946484622430092CC
:101CD000FEF7CEFB39461FFA85FA83464846FEF7E3
:101CE000F5FC009B1A0C0AFB0BF342EA0144A342E9
:101CF00003D964190BF1FF3B27D3E41A3946204678
:101D0000FEF7B6FB394681462046FEF7DFFC009819
:101D10000AFB09F31FFA80FC4CEA0144A34208D9EC
:101D2000641909F1FF3904D2A34284BF09F1FF39D4
:101D3000641908FA06F8E41A49EA0B4605E75B4518
:101D400084BF09F1FF39BB446AE7A34284BF0BF1AA
:101D5000FF3B6419D1E700BF000000000000000055
:101D6000010003E80000000000000003E80000009C
:101D700000000200FA060003000000000037060021
:101D80000000000000000000F401000064000000FA
:101D9000018008080000000000640000000000004E
:101DA00000000000C8000000120110010200004005
:101DB000D016A105011D0102030100000902430024
:101DC000020100C0320904000001020201000524E2
:101DD000001001052401000104240202052406006C
:101DE00001070582030800FF09040100020A000040
:101DF00000070503024000000705810240000000C3
:101E00000403090426035400720069006E00610097
:101E10006D00690063004D006F00740069006F0081
:101E20006E002000430074006C0000003203540078
:101E30004D0043004D002D003100310036003100CF
:101E400020002800760069007200740075006100AF
:101E50006C00200043004F004D00290020000000CE
:101E6000524F5200000106524F4C000002064D53E3
:101E700054000003024D5650000004075341500027
:101E80000005074741500000060353544150000726
:101E900003525341500008035347500000090747BD
:101EA000475000000A0353544750000B0352534756
:101EB00050000C0352465300000D0353494F0000DD
:101EC0000E0747494F00000F0353414300001D0711
:101ED00053434F00001E0747434F00001F03434377
:101EE0004F0000200341434F0000270355463000B8
:101EF0000040075546310000410755463200004278
:101F00000755463300004307554634000044075543
:101F1000463500004507554636000046075546370A
:101F20000000470752554E0000810553544F5000A2
:101F3000800042494E00008B0000000000000000BD
:101F4000000000000102030401020304060708095F
:101F500002040608002020202020202020202828FD
:101F60002828282020202020202020202020202059
:101F70002020202020881010101010101010101099
:101F800010101010100404040404040404040410C9
:101F90001010101010104141414141410101010157
:101FA0000101010101010101010101010101010121
:101FB000101010101010424242424242020202022D
:101FC00002020202020202020202020202020202F1
:101FD00010101010200000000000000000000000A1
:101FE00000000000000000000000000000000000F1
:101FF00000000000000000000000000000000000E1
:1020000000000000000000000000000000000000D0
:1020100000000000000000000000000000000000C0
:1020200000000000000000000000000000000000B0
:1020300000000000000000000000000000000000A0
:102040000000000000000000000000000000000090
:1020500000000000000000003131363156313239C5
:10206000004142530052454C00434F4F52440053ED
:10207000544152540053544F5000535441545553FB
:1020800000000000430000006C6F670000000000CB
:0820900068F6FF7F010000006B
:1020980058200108000100000001020000080000AB
:1020A8000100000002000000000000000000000025
:1020B8000000000000000000000000000000000018
:1020C8000000000000000000000000000000000008
:1020D800000000000000000000C20100000008002D
:1020E800001E010804000000041E0108260000006C
:1020F8002C1E010832000000B00000201A00000069
:10210800BC1D010843000000A81D010812000000C2
:10211800119900081D9700082D95000841950008A1
:1021280045950008A5950008C99500080D97000871
:10213800FD960008D9960008000000004000000045
:102148001A0354004D0043003100310036003100BD
:102158000000000000000000000000002D940008AE
:1021680001ED000801ED000801ED000801ED00088F
:1021780001ED000801ED000801ED000801ED00087F
:102188006D98000801ED000801ED000801ED000858
:1021980001ED00080401000001ED000809950008A0
:1021A80001ED000801ED000801ED000801ED00084F
:1021B80001ED000801ED000821950008010000006C
:1021C800551F0108541F01083C01002000000000B1
:1021D80000000000000000000000000000000000F7
:1021E800000000000000000000000000842001083A
:1021F80000000000000000000000000000000000D7
:1022080000000000000000000000000000000000C6
:1022180000000000000000000000000000000000B6
:1022280000000000000000000000000000000000A6
:102238000000000000000000000000000000000096
:102248000000000000000000000000000000000086
:102258000000000000000000000000000000000076
:102268000000000000000000000000000000000066
:102278000000000000000000000000000000000056
:102288000000000000000000000000000000000046
:102298000000000000000000000000000000000036
:1022A8000000000000000000000000000000000026
:1022B8000000000000000000000000000100000015
:04000005080041109E
:00000001FF
